:020000040800F2
:10000000F8FF012001E70A089DE70A08CD780408F7
:100010009DE70A089DE70A089DE70A08000000001E
:100020000000000000000000000000009DE70A083A
:100030009DE70A08000000009DE70A0875590408BA
:100040009DE70A089DE70A089DE70A089DE70A0858
:100050009DE70A089DE70A08691604089116040836
:10006000B9160408E116040809170408BD030000C6
:10007000D1030000E5030000F90300000D040000B7
:1000800021040000350400009DE70A08A97B04084C
:10009000B17B04089DE70A089DE70A0831170408A8
:1000A0009DE70A08613B04089DE70A08513B0408E4
:1000B000713B0408813B0408913B04088D1304083C
:1000C0008913040895130408911304089DE70A088E
:1000D0009DE70A089D3A0000E53B0000593D0000FD
:1000E000711704089DE70A08000000004D3C040851
:1000F000253C04085D3C0408153C04084904000044
:100100009DE70A085D230408A13B04089DE70A084F
:10011000CD3E000041400000B13B040829EB090836
:100120005D040000710400008504000099040000D3
:10013000AD0400009DE70A089DE70A089DE70A084C
:1001400000000000000000000000000000000000AF
:10015000C1040000D5040000E9040000B54100001E
:100160009D130408991304089DE70A089DE70A08EF
:100170009DE70A089DE70A089DE70A0800000000BD
:100180009DE70A089DE70A08294300009D440000F6
:100190009DE70A089DE70A089DE70A089DE70A0807
:1001A0009DE70A089DE70A089DE70A089DE70A08F7
:1001B0009DE70A089DE70A089DE70A08A5130408B9
:1001C000A11304089DE70A089DE70A089DE70A08AD
:1001D0009DE70A0869E109089DE70A089DE70A0802
:1001E0009DE70A089DE70A089DE70A089DE70A08B7
:1001F0009DE70A089DE70A089DE70A089DE70A08A7
:100200009DE70A089DE70A089DE70A089DE70A0896
:100210006D3C04087D3C04088D3C04089DE70A08F9
:100220009DE70A089DE70A089DE70A08000000000C
:10023000612304089DE70A08000000009DE70A0802
:100240009DE70A089DE70A089DE70A089DE70A0856
:100250009DE70A089DE70A089DE70A089DE70A0846
:100260009DE70A089DE70A089DE70A089DE70A0836
:100270009DE70A089DE70A081146000000000000FB
:100280009DE70A08000000009DE70A080000000042
:08029000000000009DE70A08D0
:020000040804EE
:10000000114A037A0168D35C10B4CC58CA1824F0A2
:100010000104CC501368DB07FCD4037D1F2B09D9E6
:10002000203B20225DF8044B02FA03F343F018034F
:10003000CB60704720225DF8044B02FA03F343F0D3
:1000400018038B60704700BF2CC50B084368426DD6
:1000500030B49A61EFF31182502383F31288416820
:10006000D2B2856C0B68046D23EA050323430B6051
:1000700082F31188436981681A68096822F00102D5
:10008000D0E908541A60826A1D605C615A60D0E948
:100090000B429C60DA600023B0F86C2030BCCA626E
:1000A00003777047002A4FEA014C034630B508BF7A
:1000B000E64600F1C00514BF8E468C460024196840
:1000C0000C3353F8042C43F8084C41EA0C0142EA83
:1000D0000E02AB4243F80C1C43F8042CEFD1D0F8CD
:1000E000C03043EA0E03C0E93144C0F8C03030BD2F
:1000F00010B40C4C6368002B11DD002004F1080CD7
:100100000146DCF8AC3003F1C00259600C33934275
:10011000FBD1013063680CF5867C8342F1DC5DF82D
:10012000044B704704000020F0B5404C04EB401332
:1001300093F8543403B9F0BD3D4B42011D7893F858
:1001400001C065450CD00CEB4C0E03EBCE0E9EF8B7
:1001500004604FEA4C0E771E012F5AD9032E52D05D
:100160002244A2F83814EFF31181902383F312880C
:1001700092F83A34C9B2B2F8380443EA4003002096
:100180009BB282F83A0481F311881909207881EA38
:1001900013215940D8B1C9431B01D2F8505401244E
:1001A000D2F83C049BB201F00F01D5F8AC2084409A
:1001B0000B4302F1C000590013F4004F8BB202D17F
:1001C0005168214351600C329042F4D1F0BDD2F815
:1001D0003C041B01D2F8502401F00F0110309BB2F7
:1001E0000124D2F8AC200B43844002F1C000590036
:1001F00013F4004F8BB202D15168214351600C328D
:100200009042F4D1F0BD0CF1010606F00306AE42B7
:10021000A6D0E64403EBCE030344597C00299FD0CB
:10022000A318012083F83A049AE700BF04000020D5
:10023000901E0024704700BF024B03EB401393F85D
:100240005504704704000020426A806A131A58421D
:100250005841704790F84F3830B53BB990F84D1879
:10026000012490F84E38DAB2914200D830BD04FA39
:1002700003F2B0F8565801332A43A0F85628F2E7A3
:100280000379024613F0010005D0D369D068116AE2
:1002900001385B1A1840704710B503790446DB0734
:1002A00001D4002010BDFFF7EBFF0028F9D0236A2E
:1002B0006269D05C236AE268C0B20133B3FBF2F139
:1002C00002FB11332362EDE703799B070AD5436AEA
:1002D0008269D154436A02690133B3FBF2F102FB34
:1002E00011334362704770470171704703790246CA
:1002F00013F0020007D0536A1069916A01385B1A43
:100300000340DBB2C01A704707280AD84FF4B47212
:10031000054B02FB0033B3F83805B0FA80F0400912
:1003200070470020704700BF04000020072807D84E
:10033000044B4FF4B471012201FB003383F83A25DA
:10034000704700BF0400002010B584464FEA810EBC
:10035000102312F4004F4FEA420214BF0E24072468
:10036000013B92B2CCF80040F444F2D100EB811290
:100370008C010351122042F8213010BD10B5844683
:100380004FEA810E0424130B013C4FEA021203EBE7
:10039000430392B203F11803CCF80030F444F2D1D5
:1003A00000EB01130A018450062043F8214010BDE0
:1003B000704700BF704700BF00EB4000024B03EBEB
:1003C000C00313F8670C7047FC100020064B93F82D
:1003D0004820824206D900EB400003EBC00353F8EB
:1003E000640C704700207047FC100020072808D8D4
:1003F000044B03EB401393F8542412B1012283F809
:100400003A24704704000020072808D8054B03EB66
:100410004013B3F83804B0FA80F040097047002068
:10042000704700BF04000020064B93F84830834219
:1004300005D9054B03EB4013D3F844047047002063
:10044000704700BFFC100020040000202DE9F04F91
:100450004FF49A754A4E85B000FB05F506EB050E84
:100460009EF87D219EF87C31DEF864909A4273D02C
:10047000444B05F11C0B4FF0010A03EB00289FEDE4
:100480003E7BD9F8C44014F4001265D19EF87D116A
:10049000C4F304448B1C2701C9B205EB0310009779
:1004A00008EB041C304490F86900002857D005EB95
:1004B00001103044C06F20F0604040F0804047F8A9
:1004C0000800080105EB0313334493F868703F04F8
:1004D000CCF8047093F868708DED027B3FB328442C
:1004E000012F304490F8803002931ED01023012059
:1004F00013FB01B1244B19440346CDE9008403F0FA
:10050000FC0203F0030311F8018F01301032DB000D
:100510006A4408FA03F352F8084C234342F8083CB3
:10052000C3B2BB42EBD3DDE90084DDE902270AFA5E
:1005300004F4CCF80820CCF80C70C9F8D0409EF830
:100540007D31013303F00F038EF87D319EF87D215C
:100550009EF87C319A4294D105B0BDE8F08F05EB4E
:1005600001100A4F3044C06F07EA8040009F47F8EF
:1005700008000801A6E700BF00000000000000001E
:10058000901E002430AC0040F41E00240000FC1F2C
:100590002DE9F04FDFF8F0B04FF49A7985B00746B7
:1005A00009FB00B9D9F864502C6DE6070FD4220777
:1005B00008D508232B654FF49A7303FB07B39A6F92
:1005C00001329A67A3054CD405B0BDE8F08F012332
:1005D0002B65D5F8A4305806E9D02A4E01943E4444
:1005E0003602D5F8A430C3F3052A06EB0A134FEA06
:1005F0000A1290595A6810F080489968C2F3034271
:10060000D3F80CE014BF20F06040C0F38A40082A01
:10061000134628BF08239AB100240DF1070C00955A
:10062000224602F00302032C8CBF75460D460134AE
:10063000D200D540E2B293420CF8015FF1D8009DA0
:10064000D9F87440C5F8A8A02CB1B8F1000102AAED
:1006500018BF0121A047D5F8A4305906C1D1019C8B
:10066000A5E74FF49A724FF40073384602FB07BBBC
:100670002B65DBF884310133CBF8843105B0BDE85C
:10068000F04FE3E6AC004000901E00241B4B93F8B3
:100690004C2092B353F8781C09B100200860012A5D
:1006A0002BD053F8601C09B100200860022A24D026
:1006B00053F8481C09B100200860032A1DD053F8E4
:1006C000301C09B100200860042A16D053F8181C09
:1006D00009B100200860052A0FD0196809B100206F
:1006E0000860062A09D0996909B100200860072A24
:1006F00003D01B6B0BB100221A607047FC10002066
:100700001B4B93F84C2092B353F8781C09B100208E
:100710000860012A2BD053F8601C09B10020086042
:10072000022A24D053F8481C09B100200860032A8B
:100730001DD053F8301C09B100200860042A16D0DF
:1007400053F8181C09B100200860052A0FD0196859
:1007500009B100200860062A09D0996909B1002072
:100760000860072A03D01B6B0BB100221A60704788
:10077000FC100020C04B1B78002B40F04781BF4B82
:1007800093F84C20002A00F0418113F8681C30B522
:1007900000294AD153F8781C0020012A086043D967
:1007A00013F8501C002962D153F8601C0020022A63
:1007B000086039D913F8381C002940F0C38053F879
:1007C000481C0020032A08602ED913F8201C002999
:1007D00040F0DA8053F8301C0020042A086023D946
:1007E00013F8081C002940F0F08053F8181C002072
:1007F000052A086018D9197C002940F00881196879
:100800000020062A08600FD993F82810002957D134
:1008100099690020072A086006D993F84020002A29
:1008200070D11B6B00221A6030BD53F8742C910AF2
:10083000A1F58011522940F20A814FF0FE0CEFF32E
:100840001181502080F312888D4C4FF02C0E556A88
:10085000C9B250690EFB0C4C013540F00100CCF8D8
:100860002854506181F3118893F84C2092E753F893
:100870005C2C910AA1F58011522940F2EC804FF0D6
:10088000FE0CEFF31181502080F312884FF02C0EF4
:10089000556A7B4CC9B2506901350EFB0C4440F0DF
:1008A0000100C4F82854506181F3118893F84C205A
:1008B000002053F8601C022A08603FF67BAFB3E7C4
:1008C000DA69910AA1F58011522900F2E1806D48A0
:1008D00010F801C0EFF31181502080F312884FF01F
:1008E0002C0E556A664CC9B2506901350EFB0C449A
:1008F00040F00100C4F82854506181F3118893F846
:100900004C2085E75A6B910AA1F58011522900F21B
:10091000C2805C4810F801C0EFF31181502080F3D1
:1009200012884FF02C0E556A554CC9B250690135EA
:100930000EFB0C4440F00100C4F82854506181F3D0
:1009400011886EE753F8442C910AA1F580115229C1
:1009500040F285804FF0FE0EEFF31181502080F3BE
:1009600012884FF02C0C556A454CC9B250690135BC
:100970000CFB0E4440F00100C4F82854506181F390
:10098000118893F84C201AE753F82C2C910AA1F502
:100990008011522967D94FF0FE0CEFF311815020DE
:1009A00080F312884FF02C0E556A354CC9B250694D
:1009B00001350EFB0C4440F00100C4F8285450618E
:1009C00081F3118893F84C2004E753F8142C910A12
:1009D000A1F5801152294AD94FF0FE0CEFF3118195
:1009E000502080F312884FF02C0E556A244CC9B267
:1009F000506901350EFB0C4440F00100C4F8285446
:100A0000506181F3118893F84C20EEE670475A68E4
:100A1000910AA1F58011522936D94FF0FE0CEFF35F
:100A20001181502080F312884FF02C0E556A144C1F
:100A3000C9B2506901350EFB0C4440F00100C4F806
:100A40002854506181F3118893F84C20D7E60D4863
:100A500010F801C0F3E60B4810F801C011E709488F
:100A600010F801E078E7074810F801C095E705485D
:100A700010F801C0B2E700BF00000024FC10002005
:100A8000901E0024881B0B08044810F801C0C6E71C
:100A90004FF0FE0C1EE74FF0FE0C3DE7881B0B08E5
:100AA00000EE100AB8EE400A704700BFBCEEC00A64
:100AB00010EE103A98B27047124810B590F894466C
:100AC000ECB100F5D36C4FF0000E05E00EF1010E15
:100AD0000CF1100CA64510D0BCF808009042F5D1DE
:100AE0009CF80A009842F1D1074B012003EB0E134A
:100AF00053E90223C1E9002310BD002010BD2046A8
:100B000010BD00BF901E00243025002470B5104E8B
:100B100096F89446D4B1B1F816E006F5D3630022F6
:100B200003E001321033A24210D0B3F808C0F445FC
:100B3000F7D19D7A91F818C06545F2D106EB0216FF
:100B4000D6F8A43613B1BDE87040184770BD00BF99
:100B5000901E002470B5154C94F818C794F81967C6
:100B60000CF1010505F01F05AE421DD05FFA8CFCAB
:100B7000082B9E4604EB0C1628BF4FF0080EC6F853
:100B80001C0786F8291786F828E75BB1013A06F2B8
:100B90001F710023013312F8010FDBB201F8010FBE
:100BA0009E45F7D884F8185770BD00BF901E0024EA
:100BB0002DE9F047214C6568002D34DD002304F158
:100BC00008024FF4867601271846984606FB034C28
:100BD00001339CF8051101F0FF0E59B9AB4202F543
:100BE0008672F3D120B1164B93F81C29542A1DD0DC
:100BF000BDE8F08791687046B2F810A0D1F8009077
:100C0000D2F814E0D9F80C1021EA0A01C9F80C1046
:100C1000DEF8001021F00101CEF800108CF80581FB
:100C200082F8FE70DAE70020BDE8F087B3F82429E7
:100C30000132A3F82429BDE8F08700BF040000209A
:100C4000901E002410B504466FF0DCF801462046E3
:100C500089B2BDE81040FFF767BA00BF10B500EBDE
:100C60004000084C04EBC00414ED1C7A54ED1B7AD0
:100C7000E7EE007AB0EE670A6FF0C4F854F8783CFB
:100C8000186010BDFC10002002692DE9F843C3680C
:100C900012EA030828D005460E464FF00047B8FA7E
:100CA00088F327FA03F21B3BD24308EA02082A61C1
:100CB000042B16D8DFE803F03B30251A0300B36A93
:100CC000002B3FD003F1FF3900231FFA89F9B362EB
:100CD000746A34B123682046494698476468002CFA
:100CE000F8D1B8F1000FDAD1BDE8F88370680028B8
:100CF000F7D0696B036889B29847B8F1000FCED17D
:100D0000F2E7B0680028ECD0A96B036889B2984775
:100D1000B8F1000FC3D1E7E7F0680028E1D0E96B34
:100D2000036889B29847B8F1000FB8D1DCE73069A1
:100D30000028D6D0296C036889B29847B8F1000F13
:100D4000ADD1D1E7EB6A1FFA83F9C1E710B590F88E
:100D50003DE0BEF1020F76D0144690F83D20844667
:100D6000012A02D1022280F83D200C2921D8DFE897
:100D700001F007202020222020203A2020205200AD
:100D8000DCF824003449DCF80020C1633349C16435
:100D900090F8341001290CD0012180F8341090F81B
:100DA0003510012952D000224FF4006380F834201E
:100DB0004365002010BDDCF828002749DCF800203E
:100DC000C1632649C16490F834100129F1D0012192
:100DD00080F8341090F835100129E4D138322146DA
:100DE0005BF0E8FBE5E7DCF82C001B49DCF80020B1
:100DF000C1631A49C16490F834100129D9D0012186
:100E000080F8341090F835100129CCD13C322146BD
:100E10005BF0D0FBCDE7DCF830000F49DCF80020B8
:100E2000C1630E49C16490F834100129C1D0012179
:100E300080F8341090F835100129B4D140322146A1
:100E40005BF0B8FBB5E75FFA8EF010BD3432214697
:100E50005BF0B0FBADE700BFB18A0908598A090809
:100E6000F8B5A0F668042379DB0725D5657994F8F1
:100E70004C3805F001073D46FBB1D4F848341A68F8
:100E8000D36A5B08536294F8503823B1B4F85A38E7
:100E90000133A4F85A3885F00101606C62F098FFC4
:100EA000012384F84F38002384F84D3884F84E38F5
:100EB000A4F8563884F84C38F8BD94F84F68012EE1
:100EC00003D194F84D3884F84E382046FFF7C2F924
:100ED0004EB9012385EA030184F84F38606CBDE800
:100EE000F84062F075BF0023394684F84F38F5E7C3
:100EF00038B5A0F668040022344D606C03685A626D
:100F0000A1F12903302B31D895F8CF3995F8D019B4
:100F10000133DBB2012B85F8CF3909D9B4F8563843
:100F200085F8CF295B08A4F856384B1C85F8D039D2
:100F300095F8D0290023082AA4F8583815D185F847
:100F4000D039B5F8D23901339BB2032BA5F8D23989
:100F500008D92379DB0705D5E36A94F8560843B32B
:100F6000216B98470023A4F8563838BD5B396C29AB
:100F70000CD8B4F8563885F8CF295B0843F08003C5
:100F8000A4F8563895F8D0390133CFE794F85138A2
:100F9000002BCDD1012185F8CF39A5F8D239802396
:100FA00084F85118A4F8563885F8D01962F010FF6B
:100FB000BEE7E3696269D054E369E2680133B3FBD9
:100FC000F2F102FB1133E361CCE700BF901E002475
:100FD00038B55CF005FA0D490D4CD1F8FC20A4FBA6
:100FE00000400C4D42F080720B4B800CC1F8FC208D
:100FF0004FF060420949C5F8D409C2F8B01F002279
:101000005A601A6842F001021A6038BD00ED00E033
:1010100083DE1B43901E0024001000E055CEACC5BB
:1010200070B505460A26084C013E00D170BD94F902
:10103000000021F017F9031E04DB6178EA185172F1
:10104000A278EA540434EFE7DB1B0B0830B40D4CF4
:10105000BFF34F8F0C4BC3F85C42BFF34F8FBFF30E
:101060006F8F0A4B0A4D03F13000DA792AB15979B2
:1010700034F8112092B225F811200C338342F4D1B8
:1010800030BC70472062012400ED00E06828002495
:10109000804B012400207047704700BF036882B076
:1010A00023F002030360036823F004030360036872
:1010B00023F040030360036823F020030360036808
:1010C00023F010030360036823F080030360836947
:1010D0009B0603D5C36943F02003C36183699A0764
:1010E00001D5002383628369DB0701D40123836177
:1010F00000224260036823F0010303600192019B18
:101100003F2B06DC00BF019B01330193019B3F2B6A
:10111000F8DD03684FF0010C074A43EA0C03036053
:10112000002381F800C04B70B2F82C3A63449BB2A4
:10113000A2F82C3A02B07047901E00242C2170B403
:1011400000FB01F16B4C6318D3F8303A5B681A6806
:10115000D5060CD59A69D20609D5DA692144184614
:1011600042F0100201F6482170BCDA6196E71A6875
:1011700096071ED59A6995071BD52C2202FB0042C3
:1011800092F84D1A21B192F84C1A002940F0938040
:101190002C2202FB004292F84C1A21B192F84D2AFF
:1011A000002A40F086801A6822F0020270BC1A60A1
:1011B00070471A68510722D41A68560638D59A69BA
:1011C000550635D52C2202FB004292F84E1A002912
:1011D0006FD092F84A4A484992F84C0A5A680A4035
:1011E0004649224342EA0042114359601A6822F0FC
:1011F00002021A601A6842F004021A6059E09A6901
:101200005207D9D52C2202FB004292F84E1A19B18E
:1012100092F84C1A00295DD12C2202FB004292F870
:101220004C2A002A45D11A6822F004021A6040E0D4
:101230001A68910625D59A69920622D5D9692C2279
:1012400041F0200102FB00420020D961196821F021
:1012500002011960196821F004011960196821F070
:1012600040011960196821F020011960196821F006
:1012700010011960196821F08001196082F8490A8B
:1012800017E01A6822F002021A601A6822F00402BB
:101290001A601A6822F040021A601A6822F02002CE
:1012A0001A601A6822F010021A601A6822F080028E
:1012B0001A6070BC7047D2F8501A4D1CC2F8505AD0
:1012C0000978C9B2996292F84C1A0139C9B282F808
:1012D0004C1A5DE7596AD2F8545AC9B26E1CC2F86A
:1012E000546A297092F84C1A0139C9B282F84C1A22
:1012F00092E700BF901E0024008000FC00240082C2
:101300002C23014610B41E4C03FB0043D3F8302AB3
:101310005068026812062AD58269D20506D5C269CC
:1013200042F48072C261012283F8482A83699A05D7
:1013300009D5C2692C2342F4007203FB0143C26148
:10134000012283F8482A83695B0509D5C2692C23E9
:1013500042F4806203FB0143C261012283F8482A00
:101360002C2303FB01F1631893F8483A13B95DF895
:10137000044B7047034B5DF8044B19448EE600BFE5
:10138000901E0024D82800240020B9E70020D5E6CC
:101390000120B5E70120D1E60220B1E70220CDE629
:1013A0000320ADE70320C9E62DE9F8430568D5E938
:1013B00004366C68F0611A7DD3F800801F2A4BD97F
:1013C000203A2021376801FA02F242F01802C8F8E8
:1013D0000C20327D1F2A4AD9203A202101FA02F23C
:1013E00042F01802FA6072680020596808601060C4
:1013F0004046116841F01001116093F80890AA6905
:10140000494668F0F5FA367AEA693846314668F0B6
:10141000EFFA2B6A9A6863686FF30F0313436360F4
:10142000164B13F809009A5D58F8003043F0010399
:1014300048F80030BB5843F00103BB50A36843F4A5
:101440004043A360236843F001032360236843F40F
:1014500000732360BDE8F8832021376801FA02F2A7
:1014600042F01802C8F80820327D1F2AB4D8202183
:1014700001FA02F242F01802BA60B4E72CC50B0878
:10148000D3B20F2B1FD8114B00B503F17E0E02E033
:101490000333734514D093F800C08445F8D193F812
:1014A00001C08C45F4D102EB42020948997800EB67
:1014B00082030430D96000EB820019715DF804FBEF
:1014C00000205DF804FB0020704700BF001C0B08E3
:1014D0000000002410B40C4C002304F52E6C01E035
:1014E000152B0CD003EB430201331CF80210814290
:1014F000F6D1144494F9E20A5DF8044B70474FF0BA
:10150000FF305DF8044B7047901E002430B5114D3C
:10151000002305F1F80C02E001331A2B18D05CF817
:1015200033408442F8D10CEBC30EDC009EF804E09B
:101530008E45F1D102EB4202074B254403EB8201B9
:10154000043395F8FD4003EB8200CC600C7130BD94
:10155000002030BD881B0B0800000024F0B10023E0
:1015600010B504460E4894F804E000F52E6C01E036
:10157000152B11D003EB430201331CF80210714507
:10158000F6D183186179206893F9E22AD3B20F2B40
:1015900002D8BDE81040B9E7002010BD0020704718
:1015A000901E00244FF02C0C01380C4B82B00C4ADA
:1015B0000CFB00330B49D3F8C4308B4214BF022319
:1015C0000123D2F8D8101943C2F8D810D2F8D82085
:1015D00013400193019B02B0704700BF000000243C
:1015E0000044025800000240F8B501381E46134C72
:1015F0002C2315460F4603FB0044114BD4F8C400BE
:10160000984214BFA120A02064F092FBC5F3011200
:10161000A909B4F9DC00C4F8D470C4F8E0605AF049
:1016200071FAB4F9DC30002B07DB03F01F00012254
:101630005B090449824041F82320F8BD00000024E2
:101640000000024000E100E060B182884FF0B0414C
:101650004FF00043B2FA82F2D1F88000D340034346
:10166000C1F88030704700BF4FF0B042D2F88030F0
:10167000D2F888100B4003F00103C2F8883023B180
:10168000024BD3F8200B036818477047901E0024C4
:101690004FF0B042D2F88030D2F888100B4003F0FF
:1016A0000203C2F8883023B1024BD3F8240B03683D
:1016B00018477047901E00244FF0B042D2F8803097
:1016C000D2F888100B4003F00403C2F8883023B12D
:1016D000024BD3F8280B036818477047901E00246C
:1016E0004FF0B042D2F88030D2F888100B4003F0AF
:1016F0000803C2F8883023B1024BD3F82C0B0368DF
:1017000018477047901E00244FF0B042D2F8803046
:10171000D2F888100B4003F01003C2F8883023B1D0
:10172000024BD3F8300B036818477047901E002413
:10173000F8B54FF0B043D3F88050D3F88820154067
:1017400005F47875C3F888507DB1084F0126B5FAC5
:1017500085F4C4F11F0407EB840306FA04F4D3F8FC
:10176000200B03689847A543F1D1F8BD901E0024D3
:10177000F8B54FF0B043D3F88050D3F88820154027
:1017800005F47C45C3F888507DB1084F0126B5FAB1
:1017900085F4C4F11F0407EB840306FA04F4D3F8BC
:1017A000200B03689847A543F1D1F8BD901E002493
:1017B00030B1036882881B691A4214BF01200020DF
:1017C000704700BF10B1036882889A61704700BFFC
:1017D00018B1838802681B049361704770B50D4689
:1017E00082B00446164640B101680C4B0C4A0B44CB
:1017F0009B0A02EB4303B3F8C80164F099FAC5F3FE
:101800008101C5F3411305F01302CDE90016A1884B
:10181000206868F0D5FF02B070BD00BF0000FEA7D1
:10182000881B0B0800B1D9E770472DE9F84FDFF8A6
:1018300074832C23074603FB0083D3F8305A002D12
:1018400000F08D81D3F8386A26B196F90630002B66
:1018500040F085812C2303FB0783D3F83C4A24B155
:1018600094F90630002B40F07A817B1CDBB216B174
:101870001522F371B27114B11622E371A2714FF007
:101880002C09288D64F054FA214609FB07F93046EB
:101890006BF08EF8304608EB090AB64E9AF8423AD9
:1018A0009AF8402A002B0CBF4FF01E0B4FF03E0B56
:1018B0005946FFF7B7FF20469AF8412A5946FFF7E5
:1018C000B1FFDAF8303AAC4814225C680021484491
:1018D000DFF8D4926FF0E2FD236823F00103236068
:1018E000A64B9C4215D1D6F8903043F40013C6F8AD
:1018F0009030D6F8903023F40013C6F890305BF0A7
:1019000091FD9C4BDB69C3F30213994499F8DC31D8
:1019100032E09B4B9C420AD1D6F8903043F48003CE
:10192000C6F89030D6F8903023F48003E5E7954B65
:101930009C420AD1D6F8903043F40003C6F89030A8
:10194000D6F8903023F40003D7E78F4B9C42D6D1D2
:10195000D6F89C3043F08003C6F89C30D6F89C3013
:1019600023F08003C6F89C305BF05CFD336AC3F360
:1019700002134B4493F8DC3103F01F039FED837A8D
:101980009FED835AB0EE084AD8402C23F7EE003A78
:10199000002607EE900A03FB078840F2145CF8EE7D
:1019A000677AB8F8448AC7EE275A07EE908A9FED07
:1019B000797AF8EEE77AC7EE274ADFED777AB0EE6C
:1019C000007AE5EE877AA5EE875A25EE844A37EE4F
:1019D000856A74EEE72AB8F5C87F06F10107D5BF1E
:1019E0004FF4967278226423322307EE907AD8BFA0
:1019F0004FF4167E1344A2F13202F8EEE76AC8BF34
:101A00004FF4827E07EE903AD4BF61464FF4FA71EC
:101A100066EEA56AB8EEE77A7144C7EE267A07EE5D
:101A2000102AB8EEC77A37EE447A77EEE37AFCEE06
:101A3000E77A17EE903AC7EE267AFCEEE77A17EED1
:101A4000900A07EE90EAB8EEE73A07EE901AF8EE41
:101A5000E77A23EE243A83EE277A37EE453A32EEE0
:101A6000C77AC3EE267A77EEE37AFCEEE77A17EED2
:101A7000901AC7EE267A77EEE37AFCEEE77A17EE55
:101A8000902A02F1020E0EEB0109B0EE467A07EE43
:101A9000909AF8EE677AA6EEA77AF4EEC74AF1EECE
:101AA00010FA60DC43EA000E5FFA8EFEBEF10F0F03
:101AB0005BD841EA020E1FFA8EFEBEF1FF0F54D82A
:101AC0001B05000403F07F6392B200F47F00034320
:101AD000324843EA067300EA01210B4313432268AC
:101AE0002F4E22F001022260226822F4F852226076
:101AF000002223612368114643F001032360A36899
:101B000023F40043A360A3686FF30A03A360236870
:101B100023F440132360636823F400436360236865
:101B200043F001032360012495F82B0059F0EAFFEC
:101B300095F82B305A0903F01F0304FA03F346F813
:101B40002230002295F82A00114659F0DBFF95F863
:101B50002A305A0903F01F039C4046F82240BDE892
:101B6000F88F3E4637E701318DE70F2FF9D100237B
:101B7000B5E700BF00440258D828002400540040B4
:101B800000580040005C0040001C0058286B6E4E5E
:101B900000001643002474490000704200FFFF005B
:101BA00000E100E0901E0024881B0B0808B1002211
:101BB00014E670470D4B70B593F84860A6B10C4C15
:101BC000002503E001352034B5420DD0237F002BE2
:101BD000F8D0E06800220028F4D00135217DFFF71D
:101BE000FDFD2034B542F1D1012070BDFC10002074
:101BF0003C04002070B590F8723004461D09013D88
:101C0000082D11D81B4E03F00F0306EB4502B2F866
:101C1000EC1141FA03F2D20706D590F87520012A9B
:101C2000D0B205D0012070BD94F875300120FAE7DC
:101C30009840013808406FF03FFF73190E4A93F83F
:101C40000032034402EBC30552F83320AB8810691D
:101C50001840E8D0002394F873200221284684F825
:101C60007530FFF7BBFD226E136843F00803136065
:101C7000D8E700BF881B0B08F029002470B5154B6E
:101C8000BFF34F8F144903F58652C1F868322033F1
:101C90009342FAD1BFF34F8FBFF36F8F0F4C40F2D7
:101CA0002A430C4AB4F87C5904F513602946FFF71F
:101CB0004DF8034618B1002384F87E3970BDD4F87E
:101CC0003069294604F5136001227362BDE8704053
:101CD0006BF0F4BE60B7012400ED00E0901E00241C
:101CE000014B53F82000704750400058014B43F817
:101CF000201070475040005819481A4B01681A4A82
:101D000041F4807130B482B00160D3F8F410FF2444
:101D1000CA2041F48031C3F8F410D3F8F41001F470
:101D2000803101915321019D546250625162D3F878
:101D3000D030DB010CD40C4B00220C495A659A655B
:101D4000DA651A665A669A66196502B030BC704741
:101D5000126D064B9A42EED102B030BC704700BF04
:101D6000004802580044025800400058316665425D
:101D70002DE9F84FD0F85C710446534B00F5967688
:101D8000FDB227F0FF09826800F1E00A103D4846E5
:101D9000D2F80080A3FB05352D09294667F084FEA3
:101DA000D4F81C210023B2F5807F84F820317FD045
:101DB0000DD8102A00F084805DD8012A46D0042A6C
:101DC00016BF6FF400616FF008013C230EE0B2F51E
:101DD000805F71D0B2F5803F3BD0B2F5806F15BF08
:101DE0006FF400616FF008013C230423324608F1D0
:101DF0001806404656F803C001EA0C01F150D4F829
:101E00001CB1594667F010FCBBF5807F2ED024D85A
:101E1000BBF1100F3FD037D8BBF1010F02D0BBF19F
:101E2000040F34D14FF0080C336852462946484617
:101E300043EA0C0333604023C4F8E83067F0D8FD70
:101E40003B6843F010033B60BDE8F88F6FF008017A
:101E5000CCE76FF008013C23C8E7BBF5805F22D0D8
:101E6000BBF5803F1AD0BBF5806F10D108F11C067E
:101E70004FF0080CD8E7402A15BF6FF400616FF0EF
:101E800008013C230023B1E7BBF1400FCAD03C3628
:101E90004FF4006CC8E74FF4006CC5E708F1540636
:101EA0004FF0080CC0E708F11C064FF4006CBBE7CC
:101EB0006FF00801042399E76FF40061042395E7AC
:101EC0006FF4006192E700BFABAAAAAA464A92F853
:101ED000E41F013949B24B1C00F08480434B480198
:101EE00003EB411100B5C2F8E81F811D13F801E0B2
:101EF00003EB010C92F8EC1F8E455BD09CF802E0DE
:101F00008E4555D000F10A0113F801E003EB010CF6
:101F100092F8ED1F8E4546D09CF802E08E4540D0E9
:101F200000F10E0113F801E003EB010C92F8EE1F33
:101F30008E4531D09CF802E08E452BD092F8E21FFE
:101F400031B300F1120113F801E003EB010C92F838
:101F5000EF1F8E4535D09CF802E08E452FD000F162
:101F6000160113F801E003EB010C92F8F01F8E4507
:101F700033D09CF802E08E452DD01A3092F8F11F34
:101F800013F800C003448C4521D0987888421DD0B6
:101F90005DF804FB0CF1020CBCF80010A2F8F41F71
:101FA000CCE70CF1020CBCF80010A2F8FE1FB7E75A
:101FB0000CF1020CBCF80010A2F8FC1FA2E70CF117
:101FC000020CBCF80010A2F8F61FC8E702331B8809
:101FD000A2F8FA3FDCE70CF1020CBCF80010A2F802
:101FE000F81FCAE7704700BF901E0024941D0B081D
:101FF0000120704738B5134D41F20D13124941F2DB
:10200000883255F8B40C55F8F84C0004A060E0682C
:10201000014020460B430D21E3605BF02DFE38B1FB
:1020200055F8C42C03460020134345F8C43C38BD82
:10203000606900F4F050A0F50060B0FA80F040094B
:1020400038BD00BF882F0024C0E0FEFFC24B53E91B
:102050001F1270B58C0F1D7C100EC2F3072C03F8F5
:10206000484CC1F383640001012D03F8474CC1F3D0
:10207000016403F8464CC1F3074403F8454CC1F32F
:102080000724C9B203F8444CC2F3035403F8431CB9
:1020900023F8420CC2F3C03033F8421C89B241EA43
:1020A0000401C2F3034423F8421CC2F3403103F895
:1020B000404CC2F3803403F83F0C4FF0000003F8AB
:1020C0003E4C03F83D1CC2F3003103F83C1C53F8AE
:1020D000741C03F83B0C40F2EC80022D00F0C3802E
:1020E0002A204FEA4C0C03F82F4CC1F3C01201F028
:1020F0007F010CF07E0C03F82ECC4FF0010C13F88E
:102100002E4C144353F8702C03F82E4CD40F03F8C4
:102110002D1C910D03F82C4CC2F3417401F00C01FD
:10212000C2F3815503F82B4CC2F3826403F82A4CA6
:1021300003F8291C13F8291C53F86C4C294303F8A5
:10214000291CC2F3405103F8281C002103F8271C66
:10215000C2F3004103F8261CC2F3C03103F8251C6A
:10216000C2F3803103F8241CC2F3403103F8231C6E
:10217000C2F3003103F8221CC2F3812103F8211CB1
:10218000C2F30121C2F3460203F8201CC4F3074145
:1021900003F81F2C220E090203F81ECC03F81C2C96
:1021A000C4F3072223F81A1C240633F81A1C89B238
:1021B000114323F81A1C53F8681C43F8184C0C0EF2
:1021C00053F8182C42EA044243F8182C0A0A53F830
:1021D000184C02F47F422243C1F30724C9B243F8EA
:1021E000182C53F8185C53F8642C2C4343F8184C03
:1021F00003F8141C110E03F8131C110C090643F804
:10220000101C110253F8104C0A4601F47F012143BF
:1022100092B253F8604C43F8101C53F8101C0A4358
:1022200043F8102CC4F3035253F8101C41EA146114
:1022300043F8101C13F80C1C1143C4F3072203F8D5
:102240000C1C210A01F4706123F80A1C33F80A1CE3
:1022500089B21143C4F3460223F80A1C03F8082C80
:1022600003F807CC70BD1204C1F3072C0D0E02F465
:102270007C1243F8382CC1F3074253F8384C44EA37
:10228000052443F8384C53F8384C22434FF400747B
:1022900043F8382C53F8382C9C60013240F100048C
:1022A000A40244EA925492025C60C1F380341A6042
:1022B00017E74FEA8C2CC1F3C26594000CF440621E
:1022C000C1F3072C04F47F7443F8382C53F8382CEE
:1022D0001443CA0B43F8384C02F0060253F8384C4A
:1022E00044EA917443F8384CC1F3026403F8345C57
:1022F000012503F8334CC1F3425403F8324CC1F3C7
:10230000824403F8314CC1F3C03403F8302C13F885
:10231000302C224303F8302C53F8384C13F8302C6F
:1023200013F8406C023205FA02F2B540D617A2FB50
:10233000052E9D6005FB06EE04FB0EEE0134A2FBAC
:102340000424A644520AC1F3803442EACE521A60F1
:102350004FEA5E225A60C4E6882F002462F0F8BA81
:1023600062F0F6BA2DE9F04F067991B00546046E99
:1023700016F0020940D090F87280B8F1000818BF3A
:102380004FF001084FEAC802236823F4F873236072
:10239000A36823F00103A360236823F001032360F3
:1023A000B34B9C4200F05581B24B9C4227D0B24BBC
:1023B0009C4200F08981B14B9C4200F0B681B04B49
:1023C0009C4200F07381AF4B9C4200F0BC81AE4B4D
:1023D0009C4200F0C681AD4B9C421DD1AC4BD3F862
:1023E000901041F00041C3F89010D3F8901021F004
:1023F0000041C3F890100FE04A46C846C4E7A44B1A
:10240000D3F8901041F40031C3F89010D3F8901035
:1024100021F40031C3F890102368D5F808A0D9073B
:102420006F794AD4BB022068390206F0010603F432
:10243000805301F480610B43964901400B4343EA0A
:102440008603134323603B03626803F4005322F4C2
:10245000405213436360904BA4EB030BA36823F437
:102460004073BBFA8BFBA3604FEA5B1B804B4FEAC8
:102470008B0B9C4200F036817E4B9C4220D07E4BE1
:102480009C421DD003F580639C4219D003F5806304
:102490009C4215D003F544439C4200F02381A3F5F0
:1024A0001C439C420CD003F580639C4208D0E36A35
:1024B00023F00F0343EA0B03E36211B0BDE8F08F92
:1024C00076485BF0A7FC0028F1D0BAF1000FEED0FF
:1024D000734B03EB8B03D3F84C32B0FBF3F000EB00
:1024E0005A00B0FBFAF080B2E060E36A23F00F0319
:1024F00043EA0B03E362FB070BD51EB1636843F4A9
:1025000080336360B9F1000F03D0636843F4003394
:10251000636095F874301BB1636843F400436360F3
:10252000A3683F0743F48053A360236823F000535C
:102530002360636823F490436360A36823F02A0355
:10254000A36003D5A36843F00803A360236843F0A6
:1025500001032360002E3FD0EF6B002F00F0D480EA
:102560006B6CFEB227F0FF090022099304F12403EB
:10257000103E484600934FF4806305934FF48073F8
:1025800003934FF480330A93464BA3FB0636002394
:102590000293360904933146CDE90B33CDE90D336F
:1025A0006B690193EB6808930023CDE9062367F07C
:1025B0007BFA6A463146484667F01AFA3B6843F0B0
:1025C00001033B60384BA2689B5D42F040024B44E4
:1025D000A2605B689BB26B65B8F1000F3FF46DAF12
:1025E0002E6C002E00F08580F1B2AA6C2D4B26F0E7
:1025F000FF07A1F1100509923846A3FB053500231A
:1026000001932D0908932946CDE90333CDE906331B
:10261000CDE90B33CDE90D334023029304F12803B8
:1026200000934FF4806305934FF480330A9367F06F
:102630003BFA6A462946384667F0DAF9336843F0D0
:1026400010033360236843F04003236011B0BDE8FA
:10265000F08F0F4BD3F8981041F01001C3F8981089
:10266000D3F8981021F01001C3F89810D4E600BFF9
:10267000001001400044004000480040004C004071
:10268000005000400014014000780040007C0040F1
:1026900000440258F369FFEF000C005808000007DF
:1026A000881B0B08ABAAAAAA2CC50B08344BD3F87D
:1026B000901041F48011C3F89010D3F8901021F4D9
:1026C0008011C3F89010A7E62D4BD3F8901041F479
:1026D0008021C3F89010D3F8901021F48021C3F822
:1026E000901099E627485BF095FB00283FF4DFAE99
:1026F000EBE6236843F080032360236843F0400344
:10270000236011B0BDE8F08F236843F48073236029
:10271000A36843F00103A360236843F02003236010
:10272000236843F01003236056E7154BD3F890104D
:1027300041F40021C3F89010D3F8901021F4002147
:10274000C3F8901068E60E4BD3F8981041F02001C2
:10275000C3F89810D3F8981021F02001C3F898100E
:102760005AE6074BD3F8901041F08041C3F890101F
:10277000D3F8901021F08041C3F890104CE600BFD0
:10278000004402580803000738B50409013C082C2E
:102790001AD80F4D00F00F0305EB4402B2F8EC011C
:1027A00040FA03F212F0010210D00122254402FA8D
:1027B00003F3013B18406FF07FF995F80032054AAA
:1027C000034402EBC30038BD002038BD104638BDBD
:1027D000881B0B08F02900242DE9F047944D05EBE8
:1027E00000135C69002C00F08880DF8B06464FEAFE
:1027F0000019384663F09CFA01227B0907F01F0795
:10280000023BBA40082B0FD8DFE813F0B900C10033
:10281000C900D100D9000900E100E900B1008549F3
:10282000CB6F23EA0203CB6705EB09030136187E61
:10283000F6B2FFF7A9FF074610B11223C6718371E4
:1028400005EB0903587EFFF79FFF824610B1132363
:10285000C671837105EB0903987EFFF795FF8046EB
:1028600010B11423C67183714D4450462E212A7F26
:10287000FEF7D8FF6A7F40460E21FEF7D3FFEA7EBF
:102880002E213846FEF7CEFF23686B4A23F0010362
:102890009442236033D0694B9C423ED1654BD3F8C0
:1028A000902042F48042C3F89020D3F8902022F484
:1028B0008042C3F89020E36843F00043E360A368DC
:1028C00023F4F073A3602368DA0716D4A1685C4A86
:1028D0005C4B0A401343A360E368DB0042D5E26827
:1028E000594B134043F0E863E360236823F400632B
:1028F0002360236D23F001032365BDE8F0874D4B72
:10290000D3F8982042F48052C3F89820D3F8982046
:1029100022F48052C3F89820CDE74C4B9C4213D050
:102920004B4B9C4263D04B4B9C426ED1414BD3F8F6
:10293000982042F48012C3F89820D3F8982022F40B
:102940008012C3F89820B6E73A4BD3F8902042F4AF
:102950000042C3F89020D3F8902022F40042C3F83C
:102960009020A8E7236843F480532360B7E73149F8
:10297000D1F89C3023EA0203C1F89C3054E72D497A
:10298000D1F8983023EA0203C1F898304CE729497E
:10299000D1F8903023EA0203C1F8903044E725498A
:1029A000D1F8943023EA0203C1F894303CE721497E
:1029B000D1F8803023EA0203C1F8803034E71D49A2
:1029C000D1F8843023EA0203C1F884302CE7194996
:1029D000D1F88C3023EA0203C1F88C3024E7154982
:1029E000D1F8883023EA0203C1F888301CE7114B84
:1029F000D3F8982042F40052C3F89820D3F89820D6
:102A000022F40052C3F8982055E7134B9C427FF400
:102A100052AF03F50C33D3F89C2042F02002C3F8E8
:102A20009C20D3F89C2022F02002C3F89C2042E78F
:102A3000882F002400440258003001400038004034
:102A4000E0FFBF8F07000020FFFF39D8003C0040A7
:102A500000340140005001400014005808B51D200A
:102A6000FFF792FE10B190F9063053B11E20FFF728
:102A70008BFE10B190F9063003B108BD5523C38019
:102A800008BD5523C380F1E72DE9F04FDFF810931F
:102A90009BB099F8741031B1B54B93F8844320463C
:102AA0001BB0BDE8F08F0124B24D7C22A9F1F800E3
:102AB00089F874406EF0F2FCD5F8E86F4FF480525C
:102AC00095F8E27F346849F8F02C49F8F84C1FB1CA
:102AD0004FF4804249F8EC2C01224FF4003C49E9C4
:102AE0003AC219F8C82C002A00F0F1800321A24A4A
:102AF0000AAB09F8C81CD26C18460093D50340F104
:102B0000E2805AF0C9FC0C989C4A010A6668A2FB54
:102B100001219B4A090932400A434D006260A842E4
:102B2000226842F00302226057D39649B0FBF5F0C9
:102B3000B1FBF0F1D9F878000231D9F878301B1ADE
:102B40009942FAD800228A4E0492A2608E4AE16825
:102B50000A408E4942F48052E260D6F88823A1FBF5
:102B6000021B41F288324FEA5B2B02FB0BFB5A46F9
:102B7000002A00F09780636B013A1806F8D5844A62
:102B80008149A2634FF4D572A260E268114041F21C
:102B900008120A43E260BBF1000F09D05A46636B8A
:102BA00013F0450F02D0990440F1FC80013AF6D1B0
:102BB000002249F8BC2CA260734AE1680A4042F442
:102BC0008052E2605A46002A6CD0636B013A1D06BF
:102BD000F9D56F4A0025A26303E1D9F87810D9F836
:102BE00078305B1A022BFAD9ACE7636B590700F116
:102BF000B282C4F838806169049B002903F10103A3
:102C00000493049B04DB4FF6FE72934240F2F6807D
:102C100004984FF6FE722B465D4690429B4600F2AA
:102C20002F834A0040F1198122680127930749F850
:102C3000C07C00F098820022DFF84C812046A26020
:102C400041F20232E16801EA08010A43E2605BF006
:102C5000B5F848BB626904F1200304F1180A49F889
:102C60008C2CA269019349F8882CE26949F8842CDC
:102C7000226A49F8802C41F20312A060E16801EA5F
:102C8000080104F11C080A43E260BBF1000F09D0FF
:102C9000636B13F0450F02D0990440F1F482BBF14D
:102CA000010BF5D14FF00040012209F8C82C59F86A
:102CB000C42C024349F8C42C2A24204686F88443B5
:102CC0001BB0BDE8F08F5AF081FC0B981CE7314A2D
:102CD000944200F08B82304A944200F0A38295F82F
:102CE000FC0FFFF751FD824695F8FE0FFFF74CFDF4
:102CF000804695F8F40FFFF747FD95F8F63F044638
:102D000095F8FABF009395F8F83F0193BAF1000FD8
:102D100005D0504695F8FD2F0E21FEF75FFDB8F166
:102D2000000F05D0404695F8FF2F0E21FEF756FD07
:102D30002CB1204695F8F52F0E21FEF74FFD002F00
:102D400040F014820022B6F90400114658F0DAFE71
:102D5000B6F90420002A07DB02F01F040121520902
:102D60000E48A14040F8221059F8F84CBEE600BFCA
:102D700000000024901E002400440258598B4F018B
:102D8000002CC0FF10210100C0E0FEFFD34D6210F7
:102D9000C5002000007000520024024800E100E05D
:102DA000882F0024626B520700F1AD82626BD3075B
:102DB0004CD4626B570601D54022A2630022012544
:102DC000CD49204649F8BC5CA260E268114041F25E
:102DD00037120A433721E26041F288325AF04CFF41
:102DE00088BB04994FF6FE72914232D85B46DFF8F9
:102DF00008A3AB46C14FDFF808831D4600233721E7
:102E00002046A36041F23713E26802EA0A02134344
:102E100041F28832E3605AF02FFF00287FF444AF7C
:102E2000A76041F22913E26802EA0A021343E36051
:102E30004DB12B46626B12F0450F02D090047FF526
:102E4000D4AE013BF6D14FF080502DE70122A263B2
:102E5000AEE60499914200F213822268900700F0D6
:102E6000828159F8C07C032F7FF4E5AE59E927121F
:102E7000A069000D49F8B80C880F8DF82800C1F33F
:102E800083608DF82900C1F301608DF82A00C1F339
:102E900007408DF82B00C1F30720C9B28DF82C0034
:102EA0008DF82D10110DADF82E10C2F303418DF8E1
:102EB0003010C2F3C0318DF83110C2F380318DF87B
:102EC0003210C2F340318DF83310C2F300318DF867
:102ED000341000218DF83510002F40F0718140F63C
:102EE000FC7101EA820259F8941C42EA91720E9236
:102EF000C1F3C2628DF83C20C1F302628DF83D201F
:102F0000C1F342528DF83E20C1F382428DF83F203A
:102F1000C1F3C2328DF8402001220E989DF840C0C6
:102F200010440CF0070C0CF1020C00FA0CF09DF8A8
:102F300030C00CF00F0C49F8B00C02FA0CF249F852
:102F4000AC2C520A00FB02F249F8A82C59F8B40C38
:102F50004FF4007A59F8902C4FF001034FEA0048E3
:102F6000C1F3803049F8A4AC8DF84100C1F3C6101C
:102F700001F07F01DFF880B18DF8420020468DF826
:102F80004310D10F8DF84410C2F341718DF84510F4
:102F9000C2F382618DF84610C2F383518DF8471059
:102FA000C2F340518DF8481000218DF84910C2F34A
:102FB00000418DF84A10C2F3C0318DF84B10C2F3B6
:102FC00080318DF84C10C2F340318DF84D10C2F3B2
:102FD00000318DF84E10C2F381218DF84F10C2F3ED
:102FE0000121C2F346028DF850108DF8512041F2B4
:102FF00007128DF85230C4F80880E16801EA0B012D
:103000000A430721E26041F288325AF035FE002877
:103010007FF44AAEC4F808A041F21013E268102110
:10302000204602EA0B021A43E26041F288325AF06B
:1030300023FE41F21013002840F0B680D9F878A0A2
:103040006269900100F18C80402210212046A2602C
:10305000E26802EA0B021A43E26041F288325AF057
:103060000BFE00284ED1C4F8088041F23712E16807
:10307000204601EA0B010A433721E26041F288321F
:103080005AF0FAFD00283DD14FF0FF324023626232
:10309000A36201301F28FCD9E26A2046164922F0BB
:1030A000FF0242F06302E2620022A260E268114085
:1030B00041F20D120A430D21E26041F288325AF0CA
:1030C000DBFDF8B9009A06E0D9F87830A3EB0A03E3
:1030D000013300F01B81636B13F4957F40F019817D
:1030E000636B1904F0D502F12001D4F8803042F866
:1030F000043B9142F9D1E7E7C0E0FEFF000010C1B8
:10310000C500200059F8C42C49F8C42C874A012175
:10311000A26359F8C42C0243204649F8C42C09F88C
:10312000C81C4FF40071824AA160E1680A4041F274
:103130001011114341F28832E16010215AF09CFDD8
:1031400000283FF4B9AD794AA263012249F8C40CC2
:1031500009F8C82CB0E504224FF08050A263A3E523
:103160004FF40060D2E74FF080609DE50098FFF7D4
:103170000BFB20B195F8F72F0E21FEF72FFB0198DE
:10318000FFF702FB20B195F8F92F0E21FEF726FB81
:103190005846FFF7F9FA95F8FB2F00283FF4D2AD17
:1031A0000E21FEF71BFBCDE5604A4FF00103A26341
:1031B00059F8C42C024349F8C42C09F8C83C7BE5F3
:1031C000012F4FD1120459F8941C02F47C1242EAE8
:1031D00011420E924FF4007249F8AC2C0E9A013253
:1031E000920249F8B02C49F8A82CAFE6514AD2F81F
:1031F000D41021F48031C2F8D410D16F41F4803161
:10320000D167D16F21F48031D167D2F8D41041F465
:103210008031C2F8D410D2F8D42002F48032039264
:10322000039A5CE5434AD2F8DC1021F40071C2F83D
:10323000DC10D2F8841041F40071C2F88410D2F886
:10324000841021F40071C2F88410D2F8DC1041F42B
:103250000071C2F8DC10D2F8DC2002F40072029295
:10326000029A3CE5314A01214FF08050A26359F89F
:10327000C42C42F0805249F8C42C09F8C81C13E54C
:103280004FF0807010E5626B520700F10782626BAD
:10329000D30700F1FE812269D2B2032A40F0FB81FC
:1032A000254AA263626912F4604F0AD0540400F107
:1032B000038212F4004F14BF4FF480504FF480305B
:1032C000F2E4120C1A49204649F8B42C1204A26008
:1032D000E268114041F209320A43E2605AF06EFDA1
:1032E00000287FF4E1AC6169019B49F89C1CDAF885
:1032F000002049F8982CD8F8000049F8940C186878
:1033000049F8900CB4E50422A26351E44FF0004068
:10331000FCE6616B0B0700F1C981616B880700F166
:10332000C981616B890613D5C2E100BFFF0FE01FA1
:10333000C0E0FEFF00440258C5002000D4F8801011
:10334000D9F8783042F8041BA3EB0A030133DDD02F
:10335000636BDB04F2D4DDE90C02DDF828C00B99C5
:103360004FEA104E5FFA82FB0BBA4FEA1C212EF097
:10337000FF0E21F0FF014EEA0B0EDFF854B341EAD5
:103380001C61C4F838B0CCF3811B89B2CCF3401C6B
:103390008DF814B04FF4007B8DF815C0ADF8161001
:1033A000C1B206938DF81C10C0F30721C0F303507F
:1033B0008DF81D10C2F385218DF81E002046ADF852
:1033C00020E08DF82210C2F301218DF82310C2F302
:1033D000031102F00F028DF824108DF825209DF8BE
:1033E0003B20B7498DF82620C4F808B0E2681140A8
:1033F00041F210120A431021E26041F288325AF081
:103400003BFC00287FF49FAE9DF82420012F9DF8FF
:103410002510D2B259F8ECACC9B200F0B380032247
:1034200049F8A00C09F8C82CBAF5004F00F0C38089
:10343000BAF5804F00F00381BAF1000F00F0C280AE
:1034400059F8C42C42F0006249F8C42C59F8C42C35
:10345000FAB19C494FF400722046A163A260984AD9
:10346000E1680A4041F21011114341F28832E160F3
:1034700010215AF001FC002800F0DC80914AA26380
:10348000012259F8C41C084349F8C40C09F8C82C97
:1034900012E459F8E40C59F8E81C032859E93D23D3
:1034A00009D859F8A0ECBEF5007F04D0BEF5807FA6
:1034B00014BF042002201A436368DFF804B20A43F1
:1034C000814919400A4342EA0A02024320466260E7
:1034D0004FF40072A26041F21012E16801EA0B01A0
:1034E0000A431021E26041F288325AF0C5FB0028FD
:1034F000C4D10122009541F20D1A254609F8C82CC5
:103500004446D9F8783098460AE059F8C42C02436A
:1035100049F8C42CD9F87820A2EB0802013241D036
:10352000AC600D21EA68284602EA0B0242EA0A0270
:10353000EA6041F288325AF09FFB0028E5D16A69BF
:1035400002F4F052B2F5006FE4D1002F5F4F4FF05C
:103550000101009DA7F1200249F8C40C18BF022503
:1035600049F8CC0C044609F8C81C89F8105007F13A
:1035700010050FCA87E80F0017E90F0085E80F0054
:10358000FFF79BBB0A4305D0032249F8A0BC09F80A
:10359000C82C49E74FF4807249F8A02C032209F89F
:1035A000C82C41E74FF00041012249F8C41C09F83A
:1035B000C82CFFF781BB59F8C42C42F0805249F85F
:1035C000C42C43E76269002000219201CDE90A0181
:1035D0005CD4009861F0ACFC024628BB0B9AD30384
:1035E00061D5C4F8088041F23712E1682046DFF85F
:1035F000D0B001EA0B010A433721E26041F2883280
:103600005AF03AFB024678B9C4F808A0E16841F2E2
:103610000612204601EA0B010A430621E26041F24C
:1036200088325AF029FB024659F8C41C0A4349F86B
:10363000C42C0BE7012209F8C82CFFF73DBB002082
:1036400062690021CDE90A0190011FD4009861F060
:103650006FFC02460028E7D10B9A510323D5C4F82A
:10366000088041F23712E1682046DFF854B001EAE1
:103670000B010A433721E26041F288325AF0FCFA2A
:1036800002460028D0D10222A260BFE74FF40062B8
:10369000CAE70122A2630120FFF706BB04221046FD
:1036A000A263FFF701BB4FF08062BDE708202DE564
:1036B00020202BE5022029E54FF40050FFF7F4BA53
:1036C000C0E0FEFFFF0FE01F002CC0FF0C2F002406
:1036D0003A0F00182DE9F047344C94F8FC0FFFF72F
:1036E00053F8064694F8FE0FFFF74EF8054694F897
:1036F000F40FFFF749F894F8E28F074694F8F8AF13
:1037000094F8F60F94F8FA4F0EB11823F3800DB128
:103710001923EB800FB11A23FB80B8F1000F15D1EC
:1037200038460121FEF74EF8FEF740FA30460121F7
:10373000FEF748F82846FEF745F83046FEF736FA19
:1037400028460121BDE8F047FEF730BAFFF71CF824
:10375000814608B11B23C3805046FFF715F8804609
:1037600008B11C23C3802046FFF70EF804463846F4
:103770000CB11D23E3800121FEF724F8FEF716FAB1
:103780004846FEF71FF84046FEF71CF82046FEF7B5
:1037900019F801214846FEF709FA40460121FEF7D3
:1037A00005FA01212046FEF701FABFE7901E00242A
:1037B000F8B50E4B93F848709FB10D4DC7F109074E
:1037C0000924013C0FD0AE683079FEF7DDFF95F893
:1037D000DC10F27908B1FEF701F8A74205F5B475DF
:1037E000EFD10120F8BDA368FFDE00BFFC10002070
:1037F0003C050020F0B4046EEFF31183502282F3F5
:1038000012880279920702D590F872203AB9012203
:1038100080F86420DBB283F31188F0BC7047026C3F
:10382000116801F001010029F4D1466A856AAE42AF
:10383000EDD0856A476A866AB74220D8866A816277
:103840000169891B1FFA81FC8169DBB229440025CB
:1038500080F8645040202062D16051686FF30F01FE
:1038600041EA0C015160116841F001011160A26848
:1038700042F08002A26083F31188F0BC7047416A75
:10388000866AA1EB060C416A1FFA8CFC8162DBE7B9
:10389000027D0346C0691F2A1B6805D9203A2021F2
:1038A00001FA02F2DA60A5E7202101FA02F29A6039
:1038B000A0E700BFBFF34F8F0549064BCA6802F46B
:1038C000E0621343CB60BFF34F8F00BFFDE700BF43
:1038D00000ED00E00400FA0519484FF6FF0C194A04
:1038E00084B0C168184B01EA0C010A43C260D3F8E6
:1038F000D020D3F8DC2042F00052C3F8DC20D3F80B
:10390000DC2002F000520192019AD3F8DC2042F050
:103910008042C3F8DC20D3F8DC2002F0804202921F
:10392000029AD3F8DC2042F00042C3F8DC20D3F83E
:10393000DC3003F000430393039B04B0FDF748BB66
:1039400000ED00E00005FA050044025808B51D48E6
:103950000023C0F88430BFF34F8F436923F48033D2
:103960004361BFF34F8FD0F8803043F6E074C3F368
:103970004E3CC3F3C90E4FEA4C1C0CEA04017346DB
:1039800041EA8372013BC0F874225A1CF8D1ACF1B1
:10399000200C1CF1200FF0D1BFF34F8FBFF36F8FBE
:1039A000BFF34F8FBFF36F8F4369002223F40033BF
:1039B0004361C0F85022BFF34F8FBFF36F8F72B6D1
:1039C000FFF778FF00ED00E003689B0AA3F5801382
:1039D000522B54D8F0B5374CE35C0D2B4ED8364DF6
:1039E0004C2440794FF0020E04FB0354E66F840828
:1039F00003EB83000EFA04FE03EB40002044002991
:103A000043D0F7682D4C47EA0E0704EB800CCCF846
:103A10000414CCF81424F760EFF31186502282F3DB
:103A200012882C2101FB0340D0F8002442B3111D61
:103A3000C0F82424224A03EB8300224F03EB40000A
:103A4000800007441030024452F8040F08B10860A7
:103A5000011DBA42F8D10022F6B20A6086F311883D
:103A60002C2202FB0344D4F82424D2B14C2202FBC2
:103A70000353DA6FD36843F00103D360F0BD70479E
:103A80000F4A01FB03212431D5E7F46824EA0E0430
:103A9000F4600A4C04EB8006C6F80414C6F814243B
:103AA000BAE74C2202FB0355EA6FD36823F0010307
:103AB000D360F0BD881B0B08882F0024901E0024C3
:103AC00090220024B022002403689B0AA3F58013EF
:103AD000522B00D970470E4AD35C0D2BFAD84FF009
:103AE0004C0C10B40B4C42790CFB03400223C06F0A
:103AF000DA409340C26829B922EA03035DF8044B17
:103B0000C360704713435DF8044BC360704700BF48
:103B1000881B0B08882F002403689B0AA3F58013D9
:103B2000522B0FD8084AD25C0D2A0BD840790223B9
:103B300006494FF04C0CD8400CFB02128340D26F68
:103B4000DB431361704700BF881B0B08882F0024DC
:103B500001490248FDF798B8902200240000014076
:103B600001490248FDF790B890220024000001406E
:103B700002494FF08040FDF787B800BFBC22002407
:103B800001490248FDF780B8E82200240004004003
:103B900001490248FDF778B81423002400080040CA
:103BA00001490248FDF770B840230024000C004092
:103BB000F8B5164D164E2A69EB681A404FF00040D2
:103BC000B2FA82F3EAB120FA03F3012A6FEA03039F
:103BD00002EA03012B610A46F2D1D6F804758FB1CF
:103BE000013F0023BFB2C6F80435D6F8004534B112
:103BF00023682046394698476468002CF8D1002293
:103C0000DCE7F8BDEF6ABFB2EFE700BF001000408D
:103C1000901E002401490248FDF736B8C423002451
:103C20000004014010B5064C064804F23451FDF77B
:103C30002BF804F28C510448BDE81040FDF724B87D
:103C4000901E002400040140001C0040014902486D
:103C5000FDF71AB8F023002400180040014902487B
:103C6000FDF712B848240024002000400149024812
:103C7000FDF70AB8742400240040014001490248BD
:103C8000FDF702B8A0240024004401400149024885
:103C9000FCF7FABFCC240024004801402DE9F04194
:103CA0004FF425728EB0002173486DF0F7FB734B13
:103CB000734D4FF00008D3F8F02040F27D27A5F5B2
:103CC000277605F6F41442F00102C3F8F020D3F889
:103CD000F02002F001020092009AD3F8E82042F0AE
:103CE0000102C3F8E820D3F8E82002F001020192B3
:103CF000019AD3F8E82042F00202C3F8E820D3F892
:103D0000E82002F002020292029AD3F8E82042F080
:103D10000402C3F8E820D3F8E82002F0040203927A
:103D2000039AD3F8E82042F00802C3F8E820D3F859
:103D3000E82002F008020492049AD3F8E82042F046
:103D40001002C3F8E820D3F8E82002F01002059230
:103D5000059AD3F8E82042F02002C3F8E820D3F80F
:103D6000E82002F020020692069AD3F8F02042F0F2
:103D70000202C3F8F020D3F8F02002F0020207920A
:103D8000079AD3F8E82042F04002C3F8E820D3F8BD
:103D9000E82002F040020892089AD3F8E82042F0A6
:103DA0008002C3F8E820D3F8E82002F080020992EC
:103DB000099AD3F8E82042F48072C3F8E820D3F8D7
:103DC000E82002F480720A920A9AD3F8F02042F4B2
:103DD0008032C3F8F020D3F8F02002F480320B9246
:103DE0000B9AD3F8F02042F40032C3F8F020D3F855
:103DF000F02002F400320C920C9AD3F8F02042F436
:103E00008022C3F8F020D3F8F03003F480230D9320
:103E10000D9B55F82810002354F83320914226D0EA
:103E200001330E2BF8D1002008F1070861F080FF64
:103E3000B845EED14FF0000840F27D2755F8281024
:103E4000002354F8332091420CD001330E2BF8D1CB
:103E5000002008F1070861F06BFFB845EED10EB005
:103E6000BDE8F08106EBC303B3F8940CF1E706EB71
:103E7000C303B3F8940CD7E79022002400440258FF
:103E8000241E0B081F4B984210B50ED003F580631B
:103E900098420AD01C4A03F58043984218BF9042CA
:103EA00003D003F5806398421BD159F0BBFA174B3E
:103EB0001749DC69DA69C4F3022CC2F3022201EB70
:103EC0000C0393F8DC3103F01F03D8400F4B11496A
:103ED0001B69C3F3C03342EAC303CB5C03FB00F0AE
:103EE00010BD59F09FFA094B0949DC69DA69C4F33E
:103EF0000214C2F302120B1993F8DC3103F01F0312
:103F0000D840E3E70000014000400140004402586F
:103F1000881B0B0808C50B082DE9F0470468A30AA5
:103F2000A3F58013522B6FD815466E4AD65C0D2E22
:103F30006AD84C27DFF8C481013907FB06FA89B239
:103F400008EB0A09C9F888100068FFF79BFF08F121
:103F50007C03B0FBF5F0013807FB0637C9F8800099
:103F6000391DD9F87C00A04200F0B7800AF1080A98
:103F70000022C9F87C405344C9F88420C3E90222D6
:103F800099F8B93003F0FF02002B00F0A3804C2514
:103F90000223204605FB068585F8B93059F018FD47
:103FA0000123B4F1804F85F8C43085F8BA3085F824
:103FB000BB3085F8BC3085F8BD3085F8BE3085F85B
:103FC000BF3085F8C03085F8C13085F8C23085F83B
:103FD000C33085F8B930444BA4EB0303B3FA83F341
:103FE0004FEA531356D0002B54D1404A94420DD07F
:103FF00002F58062944209D002F5806294422BD08F
:1040000002F57842944227D0BDE8F0874C2303FBA9
:10401000068393F8B820012AF6D00221344A83F8A7
:10402000B910A0680240A260012283F8B92083F889
:10403000B9106268A16822F0700221F080014C235F
:1040400062600022A160012103FB068383F8B9109E
:1040500083F8B820BDE8F0874C2202FB068292F874
:10406000B8100129D0D0022182F8B9102049A068E7
:1040700001402048A1600121201A82F8B9100021D6
:10408000B0FA80F082F8B8101B4A4009944213D06D
:1040900090B9B9E74C2202FB068292F8B8100129C8
:1040A000B2D0022182F8B9101149A0680140002065
:1040B000A160012182F8B9104C22022102FB068284
:1040C00082F8B9106268A1680BB90028B3D022F455
:1040D0007002B0E789F8B82059E7BDE8F04759F019
:1040E00077BC00BF881B0B080000014000040040A3
:1040F0008800CEFF00040140000C0040882F0024FF
:1041000003689B0AA3F58013522B07D82DE9F041D1
:104110002F4DEE5C0D2E02D9BDE8F08170470446AC
:10412000FFF7FAFE4C222B4B02FB063393F8B92023
:10413000012A12D020680023274951F833209042E9
:104140001CD001330E2BF8D101220020114657F06C
:10415000D9FC224B01221A60DEE70221DA6F83F8D4
:10416000B9101F4B91680B40062BE3D0B3F5803F8D
:10417000E0D0136843F001031360DBE705EBC305F0
:104180000126164F95F8964C3246314604F01F052D
:10419000204657F0B7FC1B2C4FEA541806FA05F5D9
:1041A00047F828500AD02E2CB6D1324631462C2062
:1041B00057F0A8FC4FF480537B60ADE732463146A0
:1041C000192057F09FFC4FF000733B60A4E700BF3D
:1041D000881B0B08882F002418280B0800E100E03A
:1041E000070001002DE9F04F002391B0DFF8EC92B9
:1041F0000093B04BB04DA3F55E6AB04EB04C27684B
:1042000099F80225BB0AA3F58013522B00F2CC804B
:104210001AF803300D2B00F2C780012A16F903B0FB
:1042200000F00181022A02D1BBF1080F3CD14FF00E
:1042300000084146584617F0CDFF18F055F890F9A0
:1042400000C0BCF1000F18BFBCF1540F14BF4FF0F9
:10425000010C4FF0000C40F0DC8008F104081FFA5C
:1042600088F8B8F1100FE4D1009B002B00F0A78074
:10427000914A0BE01AF803300D2B0ED8F3565B452C
:104280000ED002F58672AA4200F0958091680B6804
:104290009B0AA3F58013522BECD900235B45F0D188
:1042A0004B7961799942ECD11C34824B9C42A6D166
:1042B000009B05F586750133042B00939ED1814B3D
:1042C0004FF0010ADFF818B293F848300133029337
:1042D000029B534565D099F81635DBF80C600393C3
:1042E0009BF810300093002E5BD0774A33685568F6
:1042F0007648B288002D184401924FEA902040F38E
:104300009F806D4A002405E0013402F58672AC42BC
:1043100000F0938011688142F6D1674A4FF48671AC
:10432000019F01FB0424009ACBF80C608BF810204D
:10433000019ACBF81840B2FA82FC0322CCF11F0597
:104340006800CBF80450B27186F807A002FA00F6B4
:10435000A16C0122D4F854E0314302FA00F002FAD1
:1043600005F5A164216D0143D4F8AC0021655649DF
:104370000E78A9B2002E00F0408145EA0E05656571
:104380009F61FBF78FFE0AF1010A2046FBF75EFEF4
:104390000BF1200B40F20113BAF1090F2BF8043C8A
:1043A00096D111B0BDE8F08F013A012A7FF67CAFBB
:1043B0004FF0000B3BE7BCF1000F7FF475AFA06836
:1043C0000022434B04E001320C33102A00F06183D9
:1043D00059688842F7D152B261793846FDF796F8AC
:1043E0003C4A0023416804E0102B02F12C023FF408
:1043F0005BAF576818460133B942F5D12C23364AD2
:1044000003FB002090F9E430002B7FF44DAFAC604B
:104410004EE7009B002B7FF42BAF1C34254B9C42B6
:104420007FF4EDAE44E7BBF1010F3FF400AF1C3465
:10443000204B9C427FF4E3AE3AE7042C00F0438229
:104440004FF48671204A01FB05221169059100296C
:1044500000F0F1829060013054211D4FC4B29E469D
:1044600082F8101182F811416A1C17494A60059AB6
:1044700010685179D2F808C0002204E001320C37EC
:10448000102A00F006837B689C45F7D152B2CDF824
:1044900010E0FDF73BF80C4B4FF48672DFF83480E8
:1044A00002FB05310022049BD0E90170C1E90770CD
:1044B00041461CE068290B080C0000201CC50B08B5
:1044C00088280B08FC100020040000200000FEA734
:1044D00004000024C400002400000024882F0024CD
:1044E0003C040020102A01F12C013FF45AAF486827
:1044F000944601328742F5D12C22824902FB0C1CE2
:104500009CF9E420002A7FF44CAF4FF486728CF8BB
:10451000E54054217C4802FB05F28CF8E410144677
:104520007A4AA11006947A4C02F5607C00FB01F1F6
:1045300006982018C360C1EBC10302EB431201EBE4
:10454000C10304F10801C0F8B4200CEB4313069A30
:10455000C0F8FC3033238C18C0F8B8308C23C0F876
:104560000031059B1B6818460493FFF78BFC039BE7
:10457000062B00F0AE81072B6649674B674A18BFD0
:104580001A46674B18BF0B464FF48671B0FBF3F326
:10459000B0FBF2F2013B5E48013A01FB05019BB220
:1045A000A1F8BC20A1F874302366069B03F15801E2
:1045B00000F10803049819440023A4F858306366F6
:1045C000E36565F0AFF9049A136843F08003136064
:1045D000059B5B791A4603930C2A1BD8DFE812F07F
:1045E000F3011A001A001A00D1011A001A001A0069
:1045F000AF011A001A001A008C01CCF12F0C3F04F5
:1046000002FA0CF242EA0E02626532469F61FBF743
:1046100049FDB8E63E4A4FF4867304984FF0020C09
:1046200003FB0523602208924FF4807259690368E6
:104630000E92012223F00103079109920A220360DE
:104640000023CDE90B2C08AA0A930D930F9364F075
:10465000EBFF07990023B1F5807F00F0128240F252
:104660003B81B1F5805F00F00882B1F5803F00F03A
:10467000FF81B1F5806F15BF4FF4006208223C2323
:10468000042304991831C8580243CA50059B18796D
:10469000002840F0BE81049A136843F001031360C0
:1046A000002304E0102B08F12C0800F0AE81D8F8AC
:1046B0000420194601339742F4D105932C22114B63
:1046C00002FB0132D2F8C400164A904214BFA12066
:1046D000A02061F02DFB0399059B0C2900F293812A
:1046E000114A02EB4102B2F8E01D09484FF486720C
:1046F000DFF838E002FB0502DDF810C0002011836E
:104700001DE000BF000000246B4CA40760AF012433
:1047100004000020D0DD060044950800105522005A
:1047200040771B0000000240881B0B083018002057
:10473000944500F0A0810130042800F0AD815EF8BE
:104740003020002AF4D1BF4A1746D2F8542701324C
:10475000C7F8542707EBC002049FC000C2F83477A3
:104760000EEB0007902218462346B7F804C041EA32
:104770000C01B9800027B449FCF736FFB34A4FF467
:1047800086734FF0400C4FF4403EB14803FB0523C5
:104790004FF48052DD690793296841F010012960C8
:1047A000296841F014012960C4E91F77C4E927771B
:1047B000C4E92977196AC4F878C04FF4806CC4F84A
:1047C00094100391E9B2C4F898E01039C4F884C099
:1047D00025F0FF0CA0FB0101D3F8B800CDF810C004
:1047E000C4F890000909D3F80C80C4F8882008F1B7
:1047F00018029848059108F110082267069A70324D
:104800000244D3F8B40060674FF48040C4F88C00D1
:10481000604665F0EDF8D5F800E0069AC4F820E0AF
:10482000D5F814E0B8328B4BC4F824E0D5F804E096
:104830001A44039BC4F828E0D5F808E0C4F82CE03B
:10484000D5F80CE0C4F8DC304FF48063C4F8C870CD
:10485000C4F8CC30079BC4F830E0C4E93077C4E931
:104860003977C4E93B77DDE904C14FF4003760468E
:104870004FF4006CC4F8E070D3F80071C4F8B8804D
:10488000C4F8D8704FF48047C4F8D0C0D3F8FC30D7
:10489000C4F8D470C4F8BC3065F0AAF82B68B788A7
:1048A00063636B69A3636B68E363AB682364EB6862
:1048B00063642B6843F010032B602B6843F01403F0
:1048C0002B6033682FE5032389F8173511B0BDE855
:1048D000F08F614A614B57E6102900F0D78000F253
:1048E000BF80012900F0D080042915BF4FF4006279
:1048F00008223C230023C4E604984FF486725349EF
:10490000036802FB05124FF4805123F0010351614B
:104910000222036000230A930D930F9360230893F0
:104920004FF480730E93012309930A23CDE90B32D0
:1049300008AA64F079FE4FF400620423A1E604980B
:104940004FF4867241494FF0600C03684FF0020E3D
:1049500002FB05124FF4807123F00103516108AA94
:10496000036000230E910A930D930F930123CDE969
:1049700008C30A23CDE90B3E64F056FE0822042347
:104980007FE632494FF48672049802FB051210212B
:1049900003685161602223F0010308924FF4807292
:1049A000036000230E9201220A930D930F930223BA
:1049B00009920A22CDE90B2308AA64F035FE0023F0
:1049C0004FF400625DE604984FF486721F49036855
:1049D00002FB0512012123F00103516160220360F3
:1049E000002308924FF480720A930D930F930223D1
:1049F0000E920A220991CDE90B2308AA64F014FE55
:104A0000002308223DE600216FE64FF0FF3100232E
:104A100053E6FDF7B9FE079038B1059B0221DA791C
:104A2000FCF7DCFE5422079BDA80049A536C43F4B3
:104A3000004353642FE6022389F8173511B0BDE80F
:104A4000F08F00BFFC1000200100000004000020D7
:104A5000ABAAAAAA0C000020882A1100A0BB0D0056
:104A6000402915BF4FF4006208223C23002308E6CA
:104A700008223C2305E6C00072E64FF400620423DE
:104A8000FFE508220423FCE50822FAE54FF4006262
:104A9000F7E500235B68FFDE00239B88FFDE00BF95
:104AA0002DE9F04FB24D8FB095F81885B8F1000F91
:104AB00003D100200FB0BDE8F08F00222F21404627
:104AC00017F068FC06460028F3D0036890F80590BC
:104AD000A84F0193A7F87C99FCF740FD0028E8D087
:104AE000D0E901430293002CE3D0DFF8C0B20022EA
:104AF000594601E0102ADCD04B6894462C31013233
:104B00009C42F7D12C229C4B02FB0C3C9CF9E4A06C
:104B1000BAF1000FCDD1019B2F221846ACF8E4204A
:104B2000C7F83039FFF7AEF9944A904280F0FC8024
:104B3000012303930198FFF7A5F9039B9049C7F858
:104B400034A9B0FBF3F2120A8E48A1FB0221002225
:104B5000C7F84029C7F838290A090909A0FB020249
:104B6000C7F83C195208A5F81C255200A5F81A25CB
:104B700097F86D2902F0FF01002A00F0E780022279
:104B80000198814987F86D2958F022FF012240469B
:104B900087F8782987F86E2987F86F2987F87029B0
:104BA00087F8712987F8722987F8732987F874299B
:104BB00087F8752987F8762987F8772987F86D2986
:104BC000FDF7E2FDC5F8200528B12F21C1804E2157
:104BD000F279FCF703FE6D4A0021029BB9F10C0F3C
:104BE000C5F83015C5F82835C5F84015C5F848157D
:104BF000C5F85015C5F85415D2F8D800C5F82445A5
:104C000040F00100C2F8D800D2F8D80000F001004E
:104C100004900498D2F8D80040F00200C2F8D800FE
:104C2000D2F8D82002F002020592059A4FF0400215
:104C3000C5F82C254FF48062C5F834254FF4805216
:104C4000C5F838254FF48042C5F83C254FF40032B2
:104C5000C5F844254FF00302C5F84C2579D84C4AD5
:104C600002EB4902B2F8FC8DC2464A4A08F1080834
:104C70004949C5F85C2507EB8802C2F830195A4645
:104C8000002101E0102969D0536808462C32013117
:104C90009C42F7D1384B2C2202FB0032D2F8C400E0
:104CA0003E4A904214BFA120A02061F041F80020AC
:104CB00001E0102850D0DBF8043001300BF12C0B50
:104CC0009C42F6D107EB8807534660223449FCF733
:104CD0008BFCD7F8300957F0CDFA00287FF4E9AE05
:104CE000B479002760260C9063004A4606A929483B
:104CF00003F002030893E300CDE9066703F008031D
:104D0000002600270993CDE90A6760F0A1F9002881
:104D10007FF4CFAEA30749461E4822D558F062FF64
:104D2000B0FA80F04009C5E60198FFF7ABF81D4ADC
:104D30001D490244A1FB021A4FEA9A5A0AF1FF3AAE
:104D40001FFA8AFA0AF101030393F3E687F86C1954
:104D500015E78A46884688E70020B3E74FF0FF3022
:104D600098E758F0A9FDB0FA80F04009A2E600BF2C
:104D7000882F0024901E002400000024006CDC0218
:104D8000598B4F01ABAAAAAAC42700240044025899
:104D9000881B0B08C0270024AC340024000002400C
:104DA000D502000000366E01819F5E16C40000240B
:104DB000F8B5134C94F8CE3903F0FF05002BF9D168
:104DC000104B012693F89C3584F8CE6903B9F8BDE1
:104DD0000D4AB4F8CC79138E34320C483946FBF7BF
:104DE000B5FF034610B184F8CE59F8BDD4F8804918
:104DF0003246394605486362BDE8F84068F05EBE59
:104E0000901E0024882F00242062012410280024F2
:104E100037B590F85F380446032B2FD10023204D7F
:104E20008DF807309DF8073094F860289A4201D831
:104E300003B030BD9DF8073005EBC30393F8A435EC
:104E40008BB181F0010383B19DF8073005EBC303FB
:104E5000D3F8A005FCF7B6FC9DF807300133DBB2B0
:104E60008DF80730DEE70B46EDE79DF8073005EBE0
:104E7000C303D3F8A005FCF7ABFCEDE7D0E91003C2
:104E80009B7903F00103994204D003B0BDE83040A0
:104E9000FCF798BC03B0BDE83040FCF799BC00BFFC
:104EA000882F002438B5044600790D4650B1FDF72F
:104EB0006BFC08B10323C380E2792946BDE8384082
:104EC000FCF7B0BC38BD10B504462221FFF7EAFF5D
:104ED0002046FEF721FE20460121BDE81040FEF7E6
:104EE000F3BD10B504460121FFF7DCFF0021204689
:104EF000BDE81040FEF7E8BD38B510F8133CA0F649
:104F0000640433BB94F85028002A33D1616AA36A41
:104F100099421ED0A36AA169581CA062CB5CA06A0A
:104F20002169DBB2884200D3A2625B0043F40073C4
:104F3000A4F854380A2384F85238012384F85038EE
:104F400094F85F38012B01D0042B02D1606CFFF77D
:104F5000C8FF94F84C38002B6DD194F84D380133CC
:104F6000DBB2092B84F84D3825D12046BDE8384006
:104F7000FBF770B994F952586DB1B4F85418013D6B
:104F800020464B0801F00101A4F85438FFF740FF18
:104F900084F85258DDE7626AA36A84F850589A424E
:104FA000D7D194F85F38012B01D0042BD1D1606C9C
:104FB000FFF789FFCDE70A2B3DD194F84F382BB985
:104FC000B4F8563843F00103A4F856382379D907CA
:104FD0000AD5B4F85608820501D4C30718D4B4F82A
:104FE0005C380133A4F85C380122002384F84C2893
:104FF00094F84F2884F84D38012A1CD16179606CEF
:1050000084F84F3801F00101BDE838405EF0E0BEA1
:10501000E36AC0F3470013B1216B9847E4E7E36903
:105020006269D054E369E2680133B3FBF2F102FB39
:105030001133E361D8E738BD2DE9F84310F8133C8C
:10504000A0F664047BB1B4F8583801339BB2082B46
:10505000A4F858381BD90021606C84F85118A4F8C2
:1050600058185EF0B5FE394F97F8E085B8F1000F9B
:1050700003D101212046FFF7CBFE94F850385BBBEB
:10508000626AA36A9A4204D1002387F8E035BDE83A
:10509000F883B8F1020F12D808F1010814BFFF23FA
:1050A0007F2387F8E085A4F854380823606C84F8DF
:1050B0005238012384F85038BDE8F84311E7A36A59
:1050C000A269591CA162D35CA16A2269DBB2914238
:1050D000E9D30022A262E6E794F952685EB3B4F81D
:1050E000549897F8E15519F001010BD0012D01D822
:1050F000012103E0AB1E012B09D800212046FFF758
:1051000087FE04E015F0FD03F2D0012BF6D0013547
:10511000EDB2032D87F8E155B9D9013E4FEA59099F
:10512000002376B2A4F8549887F8E13584F85268E1
:10513000002EA5D0ABE7626AA36A9A42A7D1606C41
:1051400084F85068BDE8F843BDE600BF882F00240E
:105150002DE9F047BEB0BFF35F8FA14A0020516A2E
:105160000346044621F4803151620146C2F894009E
:10517000C2F898300133C2F89C10112BC2F8A0106D
:10518000F6D10523C2F89430536A43F48033536256
:10519000BFF34F8FBFF36F8F9248934A9349121A10
:1051A0006CF01EF99248934A9349121A6CF018F960
:1051B000924BDA6D042A00F0FB8005D8012A00F03A
:1051C0009D83022A00F0B083854A00238C4C012085
:1051D000D2F888108B4E41F470018B4DC2F88810C4
:1051E00020602361216841F0800121602168014332
:1051F0002160216841F480312160216841F48051AF
:105200002160A361E3612362A362E36223636363BA
:10521000A363E36323646364216821F48021216034
:105220007A492366C1F808014FF000614FF6FF008C
:10523000774B9160D16801400B43D36058F0D0F8B0
:10524000A36902460F20C3F30323A169334493F8F3
:10525000DC3103F01F0322FA03F3C5F8883356F05C
:105260008DFC6C4AD36813F0040FD36840F0A28021
:10527000694B0021674A0591D96A21F00101D96281
:10528000DB6A03F001030593936943F440439361A0
:10529000936903F440430593059B93699B04FCD5F4
:1052A0004C2200210EA85D4C6CF0F8F85C4A42F2EA
:1052B00003031268B3EB124F4FF000030793A4F1FE
:1052C000140308BF1C46E268002A4DD0524B5149D6
:1052D000D86A20F00100D862DB6A03F0010307936B
:1052E0008B6923F4404313438B618B6903F4404380
:1052F0000793079B474A93699F04FCD5404B4FF4A3
:10530000403748480321D3F8E02042F08002C3F838
:10531000E0200122D3F8E03003F080030693069BDF
:1053200087610D9B00910193002365F049FA0223E8
:1053300022690EA8CDE91733A3781E920122199392
:10534000A3881A93A3791B93E3791C93237A1D9363
:1053500000231F934FF48033CDE90E2357F088FDCF
:10536000032839D098B1FEE72A4A2B4B916941F4C2
:1053700040419161926902F440420792DA6A42F038
:105380000102DA62DB6A03F001030793B1E7264BFF
:105390001A6812F00E0F4BD11A6822F00F0242F079
:1053A00002021A601B6803F00F03022B40D0FEE7D5
:1053B000DC6509E723F007031C4C43F00203D360CC
:1053C000A16F05E0A36F5B1AB3F57A7F3FF650AF8C
:1053D00053689804F6D54BE772B6FEF76BFA00BF38
:1053E00000ED00E00000000070480000086C0C08B0
:1053F000000000200400002081E10C08004000585B
:1054000000440258881B0B08000000240080005153
:105410000003FA050048025800040058A0030024C5
:105420000010005C001C025800200052882F00244D
:105430006D4A936903F070033F2B05D8936923F0FD
:10544000700343F040039361674AD36903F070032C
:105450003F2B05D8D36923F0700343F04003D36199
:10546000614AD36903F4E063B3F5806F05D2D36971
:1054700023F4E06343F48063D3615B4A136A03F06F
:1054800070033F2B05D8136A23F0700343F04003E9
:105490001362554B9A69140705D49A6922F00F02DA
:1054A00042F008029A61504A936923F47063936151
:1054B000136898017FF57BAF136941F288304B4C3C
:1054C00023F0070343F003031361A16F04E0A36F0C
:1054D0005B1A834200F2C881136903F03803182B6A
:1054E000F5D1936903F00F03082B05D9936923F0D5
:1054F0000F0343F0080393613D4A136803F00F0361
:10550000022B0BD9136823F00F0343F0020313603F
:10551000136803F00F03022B7FF449AF324A9369FB
:1055200003F07003402B05D9936923F0700343F017
:10553000400393612C4AD36903F07003402B05D9D3
:10554000D36923F0700343F04003D361264AD36943
:1055500003F4E063B3F5806F05D9D36923F4E06306
:1055600043F48063D361204A136A03F07003402B35
:1055700000F272811C4F57F033FF0346D5F8B40395
:10558000BA69B969C2F30322164496F8DC2102F025
:105590001F02D340C5F8883356F0F0FA002840F0D7
:1055A00066811023159017900EA80E9357F060FC9B
:1055B000002840F050813B680E4A43F080033B6076
:1055C000D7F8F43043F00203C7F8F430D7F8F430DA
:1055D00003F002030493049B136A43F00103136274
:1055E000054BA16F0DE000BF00440258882F002436
:1055F000002000520004005800E20400013B3FF488
:10560000EBAEA26F9142F9D0A26FA36F9B1A0A2B47
:10561000FBD9C94C23689904FCD54FF480224FF480
:1056200040130EA84FF000080E9203262F9364F04B
:10563000FDFAD4F8EC300EA8C04A022743F002036A
:10564000BF49C4F8EC30D4F8EC3003F00203039304
:10565000039BD4F8943043F00203C4F89430D4F898
:10566000943023F00203C4F8943041F2030312682B
:10567000B14CB3EB124FB34BB34A28BF0A465A6042
:105680001A6822F47C5242F400521A601A6842F0FE
:1056900060021A600E96CDE92B8864F0C7FA4FF4C9
:1056A000E0430EA8CDF8E4800E93CDE9258864F0A0
:1056B000BDFA18230EA8CDF8B8800E93CDF8CC8093
:1056C00064F0B4FAD4F8D4304FF4803205210EA837
:1056D0001343C4F8D430D4F8D43021921340CDF819
:1056E0005480CDF850800293029B4FF4FA73CDF8AA
:1056F00058801296CDE910370423CDE90E2113937B
:1057000064F094FA4FF400230EA80E934FF4003384
:10571000369364F08BFAD4F8E0303A464FF4807157
:105720008A4843F00103C4F8E030D4F8E03003F0D5
:1057300001030993099B4346CDE9006865F040F8F1
:1057400023693A46824823F0FE7343F0887323614D
:10575000D4F8E03043F00403C4F8E030D4F8E0308B
:1057600003F004030893434608994FF40071CDE910
:10577000006865F025F8236923F07E4343F0FC437D
:10578000236157F02DFE734B734A4146C5F88803D9
:105790001846D21A6BF082FE7048714A7149121A8B
:1057A0006BF01EFEBFF35F8F6F4D46466F4C0127B7
:1057B0006B6A23F480336B62C5F8948022E0002981
:1057C00051D02268637A103414F8060C1B0643EAA1
:1057D000007343EA410314F8051C43EA814314F8BB
:1057E000041C43EA414314F8031CC5F898600136D1
:1057F00043EA0143C5F89C20032E43F00103C5F89A
:10580000A03035D0D4F80480217AB8F1000FD6D07A
:1058100022680029D6D122F01F09A8EB090ABAF1A3
:10582000200F38BF4FF0200A50466BF017FE411E84
:1058300007FA01F39A4518D0431C014607FA03F30F
:1058400001E05B0001315A4202EA090298188045E2
:10585000F7D8C9B2B6E7FEE7136A23F0700343F046
:105860004003136286E6FEE7A1E50346E6E79EE510
:105870000523C5F894306B6A43F480336B62BFF341
:105880004F8FBFF36F8FBFF34F8FBFF36F8F002228
:10589000C5F85022BFF34F8FBFF36F8F6B6943F48E
:1058A00000336B61BFF34F8FBFF36F8FC5F8842058
:1058B000BFF34F8FD5F8805043F6E0762A49C5F301
:1058C0004E34C5F3C905640104EA06002B4640EADC
:1058D0008372013BC1F86022F9D2203C14F1200F01
:1058E000F2D1BFF34F8F4B6943F480334B61BFF369
:1058F0004F8FBFF36F8F3EB0BDE8F0870E4A022096
:105900001B49D865D2F8F4300343C2F8F430D2F81A
:10591000F43003400E930E9AD1F8003883F30888D0
:10592000D1F804389847FEE704210320FCF7DEF99C
:1059300072B6FDF7BFFF00BF004402580010005CC4
:105940007FBB2200008400407FBB22300000025851
:1059500000080258804B012420620124E046012403
:10596000804B012485E10C0800ED00E0B803002421
:105970000090F01F10B4EFF31182102383F312880C
:105980000B4B4FF0E0200024D2B2D3F8E4150131E4
:10599000C3F8E4158169C3F8E815C3F8EC4501695B
:1059A00082F311889A6F5DF8044B01329A67704751
:1059B000882F002410B4EFF31183102282F3128891
:1059C0004FF0E0218C690A6912F4803F0E4A03D03F
:1059D0000120C2F8EC058C69D2F8E415DBB2D2F8EC
:1059E000EC2583F31188094B0A444FF47A70D3F8FD
:1059F000D41900FB01F31B1B5DF8044BB3FBF1F35F
:105A000000FB0230704700BF882F0024901E002446
:105A1000B0F1FF3F7DD003282DE9F04704463CDC80
:105A20003D4F2C2505FB0075D5F8346A002E34D087
:105A3000984695F8493A914603F0FF026BBB012363
:105A40008A4685F8493A85F8482AFFF7B3FFC5F832
:105A5000580AFFF7AFFF73680546304A1340304AD3
:105A600043EA4A031A437260B3699A0718D5C6F825
:105A70002890B36998071ED4B369D90641D52C2361
:105A8000F269284904FB03F342F010021F44194451
:105A9000F261D7F8340AFBF701FB0020BDE8F0877C
:105AA000B369DB06EBD4FFF785FF42F20F73401BAF
:105AB0009842D9DD0EE0C6F82880B3699A0614D45E
:105AC000B369DB06DBD4FFF775FF42F20F73401BAF
:105AD0009842F2DD2C23134904FB03F31F441944BD
:105AE000D7F8340AFBF7DAFAD7E7F3692C2201205A
:105AF00002FB047743F020030022F36187F8492A70
:105B0000CCE7FFF757FF42F20F73401B9842B0DD1E
:105B1000E0E70020704700BF901E0024008000FCDA
:105B200000200282D8280024B0F1FF3F00F0A680B8
:105B300003282DE9F84F044641DC514F2C2606FB83
:105B40000076D6F8345A002D39D0984696F8493A5E
:105B5000914603F0FF0293BB01238A4686F8493A37
:105B600086F8482AFFF726FFC6F8580AFFF722FFF3
:105B70006B688346434A134002F1044243EA4A03F6
:105B800002F520424FEA4A0A1A436A60AB69990754
:105B900018D5C5F82890AB695B061FD4AB69DE0643
:105BA0004DD52C23EA69384904FB03F342F0100277
:105BB0001F441944EA61D7F8340AFBF76FFA002052
:105BC000BDE8F88FAB69DA06EBD4FFF7F3FE42F2DB
:105BD0000F73A0EB0B009842D8DD38E06B68294AC0
:105BE0000A9E1340294A43EA0843B04443EA0A03A1
:105BF0001A436A60AA6950070DD4AA69D106D0D4A5
:105C0000FFF7D8FE42F20F73A0EB0B0098421EDCA8
:105C1000AA695007F1D56A6A06F8012BB045E9D1A7
:105C2000AB699A061ED4AB69DB06BAD4FFF7C2FE95
:105C300042F20F72A0EB0B039342F1DD07E0FFF796
:105C4000B9FE42F20F73A0EB0B009842A3DD2C23A8
:105C50000D4904FB03F31F441944D7F8340AFBF73A
:105C60001DFAACE7EB692C22012002FB047743F01C
:105C700020030022EB6187F8492AA1E70020704742
:105C8000901E0024008000FCD828002400240082FC
:105C9000274B5B68C3F3080310B403BBEFF3118316
:105CA000EBB9244B4FF0E02CD3F8E425DCF81800D6
:105CB000D3F8E4158A42F7D1D3F8E8158842F3D82F
:105CC0001D4B4FF47A71D3F8D44901FB04F3181A31
:105CD000B0FBF4F05DF8044B01FB02007047EFF3FA
:105CE0001182102383F312884FF0E0218C690B6935
:105CF00013F4803F0F4B03D00120C3F8EC058C69EF
:105D0000D3F8E415D2B2D3F8EC3582F311880B4402
:105D100009494FF47A72D1F8D41902FB01F0001B43
:105D20005DF8044BB0FBF1F002FB0300704700BFCD
:105D300000ED00E0882F0024901E00242DE9F04F94
:105D4000994D87B02B781BB9012007B0BDE8F08FC3
:105D50006E68964B002ED3F8E47518DD05F1080443
:105D600000209349D4F8F430BFF34F8F03F59072BD
:105D7000C1F85C3220339342FAD1BFF34F8FBFF3A7
:105D80006F8F01306E6804F58674B042EADB894A91
:105D90004FF00008884BA2FB0712DFF838920596F7
:105DA0005209A3FB0213DB0803EB8303A2EB4303BB
:105DB000DAB20492814A02F5EB6B0BEB830A1346CD
:105DC00092F8482003F638240092009B984500F092
:105DD0005581D9F8183093F8FE20002A40F041810F
:105DE000D9F80460D3E93D75FFF752FF6F4B01907E
:105DF000012293F8F005724BB240724993F81CE906
:105E000007EB40036918BEF1540F07EB410102D1C3
:105E10006B4EA6F82609994240F26E811E88164202
:105E200000F063815E88164200F075819E881642FC
:105E300000F07681DE8808331642ECD1DF1B9942F0
:105E40004FEA670740F25881E81B452828BF4520E4
:105E500003EB4000834280F0548100251E46AC468F
:105E60002946CDE9028EB3F800E00EEA020E8E4517
:105E70001CD1B3F802E00EEA020E714540F0318108
:105E8000B3F804E00EEA020E714540F02C81B3F83D
:105E90000680083308EA0208414508D1984209D92A
:105EA000B3F800E00EEA020E8E45E2D002339842CB
:105EB00000F2FC80BCF1110FDDE9028E40F221817D
:105EC000DCF1150200F11D813F49019ED1F8E83354
:105ED0009F42364BD3F8F40538BFC1F8E873331A44
:105EE000002B15DB394B03449E4201D93346053361
:105EF0002E48C0F8F435D1F8E833052B00F20D81B7
:105F000000232A4880F8F0354FF0FF33C1F8E8331A
:105F10003AB105FA02F2CCF1140C012505FA0CF5A0
:105F200015432B4BC5F3C43203EB8202D2F8180E93
:105F300005F01F0203EB8202D2F8181EC5F34412CB
:105F4000C5F3842503EB820203EB850541EA0031AA
:105F5000D2F8183E41EA0311D5F8183E41EA032170
:105F6000164B81EA1122D3F8403A82EA1212013329
:105F700002F00F020F2A2FD1B1F5803F2CD2BEF1D3
:105F8000540F4FEA111105D10D48B0F82029013204
:105F9000A0F82029094AB1F5606FC2F8403A00F034
:105FA000C180A1812BE000BF04000020882F0024C5
:105FB00000ED00E01F85EB51CDCCCCCCFC100020D7
:105FC000901E0024C7FFFF7F0000002420A10700CF
:105FD000881B0B083C040020BEF1540F05D1584922
:105FE000B1F820290132A1F82029564A4FF6FF7155
:105FF000C2F8403AD2F83C3A0133C2F83C3A9BF836
:1060000058300498834214D0DAF80820DBF80030C6
:106010009B1ACBF80030DBF80430DAF830209B1AFA
:10602000CBF804300023CAF80830CAF830308BF8B7
:106030005800DBF800300133CBF80030DAF80830D4
:106040000133CAF808304FF6FF73994209D1DBF8E3
:1060500004300133CBF80430DAF830300133CAF8B9
:10606000303008F101080BF15C0B0AF15C0A1434C2
:10607000B8F1080F09F120097FF4A7AE059E0123AE
:10608000304A002E82F83C3B7FF75EAE2E4B4FF439
:106090008671002201FB063683F8FE2003F5867325
:1060A000B342F9D1012007B0BDE8F08FA3EB060E93
:1060B000264E33F8021C4FEA6E0E11400EF1010E0F
:1060C00086FB0E86A6EBEE764FF0010E012EB8BFD2
:1060D0000126B540B444013E0EFA06F635431E468D
:1060E000C1E60433E3E60633E1E60233DF1B9942FF
:1060F0004FEA67073FF6A8AE18B10138144B83F892
:10610000F005BEF1540FACD10D4AB2F8223901337B
:10611000A2F82239A5E7043390E6053BDBB2F0E6AE
:1061200006338BE6064A537803EB430302EBC303C3
:1061300043445B7C0D2B7FF434AF8023A3775EE771
:10614000901E0024FC1000200C00002056555555D0
:10615000882F0024264B70B51A785B789A4242D17A
:10616000244E7368002B22DD06F108000025224C26
:10617000D0F8AC30BFF34F8F03F1E002C4F86832BF
:1061800020339342FAD1BFF34F8FBFF36F8F337831
:1061900013B1037F012B20D042690135716800F5EE
:1061A00086701368A94243F001031360E0DCFFF737
:1061B0006FFD124BD3F85447002C0DDD03F23473FE
:1061C00003EBC4041968083333F8042CC8689C42F4
:1061D00042EA0002CA60F5D170BD002380F8FC30AD
:1061E000F9F734FFD8E766F063FC0028B8D170BD3A
:1061F000901E00240400002000ED00E0FC100020B0
:106200002DE9F04FDFF868A287B09AF800301BB98B
:10621000012007B0BDE8F08F8E4B8F4DD3F8E445D9
:10622000FFF736FD95F84820002A00F0D2818B4B0D
:1062300005F5EB678A4E05F63828A3FB04130AF52B
:10624000A76402925B09CDF80480A6FB0316F6084A
:1062500006EB8606A3EB4606D5F8483B0025C31A95
:106260000393F3B207EB86060593B1460FE0204691
:106270000135FBF77DFD019B04F5B4745C371433E5
:1062800009F15C090193029BAB4200F0F380039A91
:10629000002A04DBD4F82431934200F387814FF4C1
:1062A000B47303FB05A393F85836002BDFD0D4F862
:1062B0005C11A3686B481A68CBB221F0FF01103B58
:1062C000A0FB030368481B09C35C0B44A1895E68FB
:1062D000D368B6B223EA0103C6F11606D360072ECF
:1062E000C5D95D4A0020D4F864B1D2F8403A80465E
:1062F000844604940133C2F8403A0123DBF80010CD
:1063000021E05BF82320BCF1140F88F00108A2EB18
:10631000010E11462EDC1EF1080248BF0EF11702D5
:10632000BEF1070F4FEA221202F1FF3E00FA02F01F
:1063300040F3838001240133944404FA0EFE9E420C
:106340004EEA000016D39E42DBD8CCF11502CCF108
:10635000140E0124002A00FA02F204FA0EFE09DDEE
:1063600018F0010F06D001334EEA02004FF0150C71
:106370009E42E8D2BCF1150F049C5FD13B49C0F3AB
:106380008423C0F3441201EB830301EB8202D3F8B0
:10639000983ED2F8982E1B0243EA021300F01F0227
:1063A000C0F3C43001EB820201EB8000D2F8982EDA
:1063B0001343D0F8982E43EA023383EA132282EA89
:1063C000121202F00F020F2A38D1C3F30F134FF647
:1063D000FF72934232D0B3F5606F00F0EB80019A08
:1063E000938197F858200598824210D0D9F8081068
:1063F0003A68521A3A607A68D9F83010521A7A60BC
:106400000022C9F80820C9F8302087F858003A68F7
:1064100001323A60D9F808200132C9F808204FF655
:10642000FF7293427FF423AF7B6801337B60D9F81E
:1064300030300133C9F8303019E7049C064AD2F8ED
:106440003C3A0133C2F83C3A002D00F0A9804FF6E7
:10645000FF73C6E7882F0024FC1000201F85EB5136
:10646000CDCCCCCCABAAAAAA2CC50B08881B0B0898
:10647000040000205A481A4600230121C0F8483B76
:10648000DAF8403580F83C1B9AF810161B6811F0BA
:10649000020FDAF85406196A0CBF014341EA800181
:1064A000012A19623FF4B4AEDAF8A8369AF87817E0
:1064B0001B6811F0020FDAF8BC07196A0CBF014320
:1064C00041EA8001022A19623FF4A2AEDAF81038DC
:1064D0009AF8E0181B6811F0020FDAF82409196A1B
:1064E0000CBF014341EA8001032A19623FF490AED8
:1064F000DAF878399AF8481A1B6811F0020FDAF8BE
:106500008C0A196A0CBF014341EA8001042A19620E
:106510003FF47EAEDAF8E03A9AF8B01B1B6811F04F
:10652000020FDAF8F40B196A0CBF014341EA80014B
:10653000052A19623FF46CAEDAF8483C9AF8181D47
:106540001B6811F0020FDAF85C0D196A0CBF0143E9
:1065500041EA8001062A19623FF45AAEDAF8B03DEA
:106560009AF8801E1B6811F0020FDAF8C40E196A3F
:106570000CBF014341EA8001082A19627FF448AE4A
:10658000DAF8183F9AF8E82F1B68164912F0020F44
:106590001A6AC96A14BF42EA81020A431A6237E6DC
:1065A0005946582210486AF01BFF50E7002007B0F8
:1065B000BDE8F08F0D4A517801EB410102EBC102B9
:1065C0002A44527C0D2A7FF40AAF802201998A77EF
:1065D00007E703490123C1F8482B81F83C3B17E644
:1065E000FC10002004100020E01B0020901E00245E
:1065F0002DE9F04F2DED048B97B00C4600250020BF
:106600000EAB002138228DF8145000930023099519
:106610000893079306932B468DF813508DF812506C
:10662000CDE90E01CDE90C01CDE90A011146204664
:1066300066F076FF05A92B460322204600917021C3
:1066400066F06EFF0CA901232522204600918821C7
:1066500066F066FF0AA90123252220460091AD219C
:1066600066F05EFF09A901231B2220460091ED215F
:1066700066F056FF08A92B462022204600914FF4D1
:10668000847166F04DFF07A92B4620222046009119
:106690004FF4947166F044FF06A92B462022204651
:1066A00000914FF4A47166F03BFF0DF113012B46EE
:1066B0000622204600914FF4B47166F031FF0DF1CF
:1066C00012012B460222009120464FF4B77166F06A
:1066D00027FFA68AF600B6F5C07F80F0FA812E4625
:1066E00010ADB146CDE9026600231093C5E9013330
:1066F0009DF81430022B00F086819DED070ADDED38
:10670000080A20EE008A9FEDDE7ADDED067AA0EE23
:10671000A08AB4EEC78AF0EE488AF1EE10FAE7EEEE
:10672000A78A10DD69F0FAFADFEDD67A60EE279AD3
:10673000F5EEC09AF1EE10FA00F14C81F2EE047A17
:1067400029EEA79A03E09FEDD09AF0EE499ACF4C3C
:10675000D4F8F8350133C4F8F83594F8FC35002B3B
:1067600040F07C810027B8462A220021C8486AF000
:1067700095FEC848DDE90A2C130F22F070414FEA5C
:10678000EC7E43EA0C130EF0030A2EF0030E23F006
:1067900070430B444FF0CC3103EB1C635344A0FB1C
:1067A00003AB2BF0030A0AEB9B0AA3EB0A03734427
:1067B000D21A6CEBE37C02FB01F100FB0C11A2FB93
:1067C0000020091802D5013241F100015208B148F8
:1067D00042EAC172C4F80426DDE90C2C130F22F042
:1067E00070414FEAEC7E43EA0C130EF0030A2EF0E0
:1067F000030E23F070430B444FF0CC3103EB1C63CA
:106800005344A0FB03AB2BF0030A0AEB9B0AA3EB58
:106810000A037344D21A6CEBE37C02FB01F100FB28
:106820000C11A2FB0020091802D5013241F1000130
:106830005208DDED087A9FED987A42EAC172099B11
:10684000F4EEC77AC4F80826944AF1EE10FA82FBF7
:1068500003124FEAE373C3EBA203C4F80C3600F152
:10686000FB809FED8F7AF4EEC77AF1EE10FA00F319
:10687000AE809FED8C7A67EE877AFDEEE77A17EEB1
:10688000903A1BB2DDED077A9FED837AA4F82836A3
:10689000F4EEC77AF1EE10FA00F1DC809FED807A19
:1068A000F4EEC77AF1EE10FA00F374819FED7D7A71
:1068B00067EE877AFDEEE77A17EE903A1BB2DDEDD0
:1068C000067A9FED757AA4F82A36F4EEC77AF1EECF
:1068D00010FA00F196809FED727AF4EEC77AF1EE2D
:1068E00010FA00F3C9809FED6F7A67EE877AFDEEAC
:1068F000E77A17EE903A1BB29FED6B7AA4F82C362C
:10690000B4EEC78AF1EE10FA78DCB1EEC87ADFEDAA
:10691000657A27EE277ABCEEC77A17EE103A9BB25B
:106920009FED617AA4F83036F4EEC78AF1EE10FAE2
:1069300059DCB1EEE87ADFED5B7AB5EEC09AF1EEA4
:1069400010FA27EE277ABCEEC77A17EE103A9BB200
:10695000A4F82E3650D4DFED557AF4EEE79AF1EE36
:1069600010FA00F3B380FCEEC97A17EE903A9BB2AE
:10697000A4F83236029BC4F82096C4F81836039B5C
:10698000A4F81066C4F81C36494BA4F81276A4F893
:10699000148695E8070083E807009DF81230022B63
:1069A0009DF8133098BF002384F83436FFF770F950
:1069B0000123C4F84C0684F85036D4F8F835013376
:1069C000C4F8F83517B0BDEC048BBDE8F08F47F67E
:1069D000FF7357E79FED377AF2EE047A79EE879AE4
:1069E00029EEA79AB3E6B5EEC09A4FF6FF73A4F866
:1069F0002E36F1EE10FAAED50023B9E74FF6FF734D
:106A00008EE72D4B78E7DDE90E7457EA04033FF477
:106A100074AE38462146294A002367F0E7FD034655
:106A20008846384621461F464FF47A72002367F0A5
:106A3000DDFD4FF47A72002367F0D8FD144643461B
:106A40003A46A4B22846009442F096FB01238DF802
:106A50004A3052E6184B32E7174B13E7FFF718F9A5
:106A6000D4F80036C01A164B98423FF77BAEB4F804
:106A70001276B4F8148677E647F6FF733CE700BF5A
:106A800018B7D138E02E654200000000882F00249E
:106A90009E350024CDCCCCCC0AD7A3C367666666EE
:106AA000C3D5A3430000C84274B5D14800CCCC453F
:106AB000C83500240000B4430080FFFF40420F00AF
:106AC0007F841E00000080770000800F4FF6FF7368
:106AD0004EE70DF115022B464FF4BD712046009292
:106AE00006228DF8155066F01BFD9DF815301F012C
:106AF00007F5C078B04550D8152B00F0478100F25B
:106B00000C81012B00F08980062B46D110AD4FF48B
:106B1000C07B0DF116030296A9465E465FED178A0B
:106B2000AB461FED178A1D46DFF8D0A200231022C6
:106B30003146204600951036ADF8163066F0F0FC70
:106B4000BDF816300AEA43321B0407EE902A03F020
:106B50000043F4EEC87A27EEA87AF1EE10FA17EEA9
:106B6000102AA8BF42F0FF42B6F5F07F43EA0203C5
:106B700049F8043BDAD1029E5D46DDED107ADDED89
:106B8000115A9DED137A9DED146A9DED155ADDEDB8
:106B9000126A73E047F6FF7391E6A94610ADCDE99E
:106BA000029907F5C877B74201D900269CE50DF197
:106BB000160200234146204600921022ADF81630FE
:106BC00066F0AEFCBDF816308C4ADFED8D6A02EA45
:106BD0004332DFED8C7A1B0407EE102A03F00043EA
:106BE000B4EEE67A67EE277AF1EE10FA17EE902A05
:106BF000A8BF42F0FF42134307EE903AF5EEC07A89
:106C0000F1EE10FAD1DD9FED807AF4EEC77AF1EE65
:106C100010FA6FDD4FF6FF7666E52B46ADF8405073
:106C200010AD10224FF4C0712046009566F078FC3C
:106C3000BDF84030714ADFED726A02EA43329FEDDF
:106C4000717A1B0407EE902A03F00043F4EEE67A13
:106C500027EE877AF1EE10FA17EE102AA8BF42F05D
:106C6000FF42134307EE903AF0EE676AB0EE675AC0
:106C7000B0EE676AB0EE677AF0EE675A77EEA57A03
:106C8000F6EE005A37EE067A9FED606A67EEA57A57
:106C900037EE057AF5EEC07A27EE067AF1EE10FAB5
:106CA00038DDB1EEE76ADFED5A7A66EE277AFCEE60
:106CB000E77ACDED027AF5EEC06AF1EE10FA26DD44
:106CC000F1EEE67ADFED526A67EEA67AFCEEE77A3D
:106CD000CDED037AB5EEC07AF1EE10FA14DDF1EEE7
:106CE000C77A9FED4B7A67EE877AFCEEE77A17EE6C
:106CF000909A56E79FED477A67EE877AFCEEE77A3F
:106D000017EE903A9EB2EFE44FF0000949E70023F6
:106D10000393DFE700230293CDE7242B7FF43DAFFD
:106D200010AD4FF4C07B0DF116030296A9465E46E6
:106D3000DFED348AAB469FED328A1D46DFF8BCA0FA
:106D4000002310223146204600957036ADF81630EB
:106D500066F0E6FBBDF816300AEA43321B0407EE84
:106D6000902A03F00043F4EEC87A27EEA87AF1EEF9
:106D700010FA17EE102AA8BF42F0FF42B6F5846F52
:106D800043EA020349F8043BDAD1F4E610AD0DF111
:106D900016030297DFF88490AA46DFED1A8A1F4691
:106DA0009FED178ADFF854B019F8010B10224FF449
:106DB000C0710023009702FB00112046ADF8163089
:106DC00066F0AEFBBDF816300BEA43321B0407EE4B
:106DD000902A03F00043F4EEC87A27EEA87AF1EE89
:106DE00010FA17EE102AA8BF42F0FF4213434AF8E8
:106DF000043B094B9945D7D1029FBEE600E0FF0F47
:106E00000000800F0000807766D62344ABAAAA3E1C
:106E100000007A440000C842A62A0B08A02A0B08EA
:106E200030B52DED028B85B00D46002310220DF1FB
:106E30000E0428462021ADF80E30009466F070FB59
:106E4000BDF80E30444A2846DFED446A302102EA9C
:106E50004332DFED437A009407EE102A1A04002330
:106E6000B4EEE67A02F0004267EE277AADF80E3013
:106E7000F1EE10FA17EE90CAA8BF4CF0FF4C42EAB0
:106E80000C0208EE102A102266F04AFBBDF80E3004
:106E9000314ADFED326A02EA4332DFED317A1B0418
:106EA00007EE102A03F00043B4EEE67A67EE277A85
:106EB000F1EE10FA17EE902AA8BF42F0FF421343FA
:106EC00007EE903AFEF7E4FE264A0121D2F8F835A3
:106ED000C2F800060B4482F8FC15C2F8F835B5EE8E
:106EE000C08AF1EE10FA11DD9FED1F7AB4EEC78A69
:106EF000F1EE10FA2DDC9FED1D7A28EE078ABCEE2C
:106F0000C88A18EE103A9BB2A2F81236F5EEC07A93
:106F1000F1EE10FA11DD9FED147AF4EEC77AF1EE7E
:106F200010FA13DC9FED117A67EE877AFCEEE77AB0
:106F300017EE903A9BB2A2F81436D2F8F835013326
:106F4000C2F8F83505B0BDEC028B30BD4FF6FF73CB
:106F5000F1E74FF6FF73D7E700E0FF0F0000800F67
:106F600000008077882F002466D623440000C842A2
:106F7000F0B585B00024102205460DF10E030E4633
:106F8000ADF80E400DF10A0700932346ADF80C4012
:106F9000ADF80A4066F0C4FA03AA234628460092D8
:106FA0001022B11866F0BCFA234606F120012846EB
:106FB0001022009766F0B4FABDF80E30604ADFED9B
:106FC000616A02EA4332DFED607A5D4907EE102A1A
:106FD0001A04BDF80C30B4EEE67A02F0004267EE17
:106FE000277A01EA43319FED576AF1EE10FA07EE76
:106FF000101A17EE900ADFED547AB4EEC67A5049B3
:10700000A8BF40F0FF4067EE277ADFED4E5A0243FB
:10701000F1EE10FA17EE900ADFED4B7A06EE902AA9
:107020004FEA0342BDF80A30A8BF40F0FF4002F02B
:107030000042464C01EA433102431B0406EE101A9B
:10704000D4F8541607EE102A03F00043B4EEE56AB4
:10705000013166EE277AC4F85416F1EE10FA17EEF5
:10706000902AA8BF42F0FF42134307EE903A9FEDEB
:10707000386AF4EEC66AF1EE10FA54D49FED356A20
:10708000F4EEC66AF1EE10FA4ADC9FED336A66EE62
:10709000866AFDEEE66A16EE903A1BB2DFED2C6AC8
:1070A000A4F85836B4EEE67AF1EE10FA3FD4DFEDEC
:1070B000296AB4EEE67AF1EE10FA3DDCDFED266ADD
:1070C00027EE267ABDEEC77A17EE103A1BB29FED77
:1070D000207AA4F85A36F4EEC77AF1EE10FA24D4E6
:1070E0009FED1C7AF4EEC77AF1EE10FA21DC9FEDE9
:1070F0001A7A67EE877AFDEEE77A17EE903A1BB2BE
:10710000A4F85C36FEF7C4FD0123C4F8600684F8D9
:107110006436D4F854360133C4F8543605B0F0BDA3
:1071200047F6FF73BAE70D4BB8E70C4BE8E70B4B9C
:10713000CDE747F6FF73E3E747F6FF73C7E700BF06
:1071400000E0FF0F0000800F00008077882F0024F0
:107150006F1203C26811034200007A440080FFFFEF
:1071600010B584B000230C4608220DF10F0019461B
:107170008DF80F300090204666F0D2F90C4B93F852
:10718000652662B99DF80F10012283F8661683F810
:1071900065260821204604B0BDE81040E8E69DF8C9
:1071A0000F2093F866369A42F3D004B010BD00BFAA
:1071B000882F002408460021DAE600BF4B4B5B68AD
:1071C000C3F308032DE9F0470546002B67D1EFF321
:1071D0001183002B63D1464B4FF0E024D3F8E42514
:1071E000A069D3F8E4158A42F8D1D3F8E8158842AB
:1071F000F4D8404E4FF47A71D6F8D47901FB07F4F5
:10720000241AB4FBF7F401FB0244384F4FF0100886
:107210004FF0E02C4FF47A7E4FF001097A68C2F308
:107220000802E2B9EFF31182CAB9D3F8E425DCF819
:107230001800D3F8E4158A42F7D1D3F8E81588424C
:10724000F3D8D6F8D4A90EFB0AF1091AB1FBFAF16A
:107250000EFB0212121BAA42E0D3BDE8F087EFF347
:10726000118288F31288DCF81800DCF81010C903CA
:1072700003D5C3F8EC95DCF81800D3F8E415D2B2C6
:10728000D3F8ECA582F311885144D6F8D4A90EFBAB
:107290000AF2121AB2FBFAF20EFB0122DAE7EFF35E
:1072A0001181102383F312884FF0E022976913694C
:1072B00013F4803F0E4B03D00120C3F8EC0597690F
:1072C000D3F8E405C9B2D3F8EC2581F31188094E4F
:1072D00002444FF47A71D6F8D40901FB00F4E41BA0
:1072E000B4FBF0F401FB02448FE700BF00ED00E0C7
:1072F000882F0024901E00242DE9F0473F4B00F119
:10730000FF383F4E10273F4D4FF0E0204FF47A7C7E
:107310004FF001096A68C2F30802002A5AD1EFF35C
:107320001182002A56D1D3F8E4258469D3F8E415F4
:107330008A42F8D1D3F8E8158C42F4D8D6F8D4199B
:107340000CFB01FEAEEB040EBEFBF1FE0CFB02EEED
:107350006A68C2F3080202BBEFF31182EAB9D3F8FC
:10736000E4258469D3F8E4158A42F8D1D3F8E81506
:107370008C42F4D8D6F8D4A90CFB0AF1091BB1FB56
:10738000FAF10CFB0212A2EB0E02B2F57A7FDFD308
:10739000B8F10108BED2BDE8F087EFF3118287F3A0
:1073A000128884690169C90302D5C3F8EC95846920
:1073B000D3F8E415D2B2D3F8ECA582F31188514486
:1073C000D6F8D4A90CFB0AF2121BB2FBFAF20CFBA2
:1073D0000122D8E7EFF3118187F3128884690269EB
:1073E000D20302D5C3F8EC958469D3F8E4E5C9B2B9
:1073F000D3F8EC2581F3118872449FE7882F00248D
:10740000901E002400ED00E001302DE9F04F964C75
:1074100083B0964E01F1FF39954D5FFA80FA10273F
:107420004FF001085BF0DEFF4FF4FA734FF0E022FB
:107430004FF47A7C01936B68C3F30803002B40F090
:10744000D680EFF31183002B40F0D180D4F8E435DF
:107450009169D4F8E4058342F8D1D4F8E805814273
:10746000F4D8D6F8D4090CFB00FBABEB010EBEFB45
:10747000F0FE0CFB03EE6B68C3F30803002B40F037
:107480009680EFF31183002B40F09180D4F8E4351F
:107490009069D4F8E4158B42F8D1D4F8E815884205
:1074A000F4D8D6F8D4B90CFB0BF1091AB1FBFBF1F7
:1074B0000CFB0313A3EB0E03B3F57A7FDBD3019B25
:1074C000013B0193B7D150465CF05EF94FF47A73FB
:1074D0004FF0E0229C4601936B68C3F30803002B36
:1074E00040F0A380EFF31183002B40F09E80D4F88E
:1074F000E4359169D4F8E4058342F8D1D4F8E8057D
:107500008142F4D8D6F8D4090CFB00FBABEB010E9A
:10751000BEFBF0FE0CFB03EE6B68C3F3080333BB4A
:10752000EFF311831BBBD4F8E4359069D4F8E4156C
:107530008B42F8D1D4F8E8158842F4D8D6F8D4B9FB
:107540000CFB0BF1091AB1FBFBF10CFB0313A3EBD2
:107550000E03B3F57A7FDFD3019B013B0193BBD1CF
:10756000B9F10109BFF45EAF03B0BDE8F08FEFF3EE
:10757000118387F31288D2F818B01169C90303D5B3
:10758000C4F8EC85D2F818B0D4F8E405DBB2D4F82E
:10759000EC1583F311880144D6F8D4090CFB00F3F1
:1075A000A3EB0B03B3FBF0F30CFB0133CFE7EFF3DB
:1075B000118387F31288D2F818B01169C90303D573
:1075C000C4F8EC85D2F818B0D4F8E405DBB2D4F8EE
:1075D000EC1583F311880144D6F8D4090CFB00F3B1
:1075E000A3EB0B03B3FBF0F30CFB013362E7EFF308
:1075F000118087F3128891691369DB0302D5C4F8FF
:10760000EC859169D4F8E435C0B2D4F8ECE580F3A8
:107610001188D6F8D40973440CFB00FEAEEB010EC2
:10762000BEFBF0FE0CFB03EE25E7EFF3118087F3C2
:10763000128891691369DB0302D5C4F8EC8591695E
:10764000D4F8E435C0B2D4F8ECE580F31188D6F86C
:10765000D40973440CFB00FEAEEB010EBEFBF0FE42
:107660000CFB03EE58E700BF882F0024901E002477
:1076700000ED00E02DE9F043144C83B0DFF85090AA
:10768000DFF8508004F5906602E00834B44219D067
:1076900094F90650002DF8D12768083407EB080349
:1076A0009B0A09EB4303B3F8C8015EF041FB34F8D1
:1076B000041C01232A463846CDE9005563F080F8C2
:1076C000B442E5D103B0BDE8F08300BFF029002447
:1076D000881B0B080000FEA72DE9F04F4C484FF027
:1076E000010A4C494FF002094B4B4FF004080827A0
:1076F0001026202540244FF0800EDFF820C130F8FE
:10770000022F12F0010F03D01960083323F804ACE4
:1077100012F0020F03D01960083323F8049C12F012
:10772000040F03D01960083323F8048C12F0080FFB
:1077300003D01960083323F8047C12F0100F03D033
:107740001960083323F8046C12F0200F03D019607D
:10775000083323F8045C12F0400F03D0196008339B
:1077600023F8044C12F0800F03D01960083323F87B
:1077700004EC12F4807F05D04FF4807B196008334D
:1077800023F804BC12F4007F05D04FF4007B19608D
:10779000083323F804BC12F4806F05D04FF4806BDB
:1077A0001960083323F804BC12F4006F05D04FF4BD
:1077B000006B1960083323F804BC12F4805F05D015
:1077C0004FF4805B1960083323F804BC12F4005FA7
:1077D00005D04FF4005B1960083323F804BC12F4A1
:1077E000804F05D04FF4804B1960083323F804BC58
:1077F000D20B05D04FF400421960083323F8042C53
:1078000001F5806161457FF47AAFBDE8F08F00BF7C
:10781000721D0B0800000258F029002400240258B1
:10782000704700BF10B4284C94F8303763B3226D12
:10783000904234D0012B27D0D4F82C21824236D06C
:10784000022B21D0D4F80822904232D0032B1BD037
:10785000D4F8E42290422ED0042B15D0D4F8C023C3
:1078600090422AD0052B0FD0D4F89C24904226D0E9
:10787000062B09D0D4F87825904222D0072B03D0CC
:10788000D4F85426824210D0DC22591C02FB034259
:1078900084F83017106518465DF8044B70470023D4
:1078A000DBB25DF8044B184670470723F8E7012365
:1078B000F6E70223F4E70323F2E70423F0E70523C6
:1078C000EEE70623ECE700BFFC10002015F078BAC5
:1078D0002DE9F04FAC4F4FF49A7585B005FB00755C
:1078E0006C6E4CB195F86890B9F1000F04D095F822
:1078F00069A0BAF1000F02D105B0BDE8F08F0646CD
:10790000B5F86E0088465EF013FA4846FAF73CFF79
:107910008346504606F1010AFAF736FF81465FFAC0
:107920008AFABBF1000F00F08C805F238BF807A070
:1079300058468BF8063095F86B20B9F1000F00F02F
:1079400018816023022189F807A089F80630F9F729
:1079500045FF95F86C2048462221F9F73FFF4FF488
:107960009A7303FB067393F86A00002852D1A36947
:1079700043F00103A361854B01E0013B02D0A26902
:10798000D107FAD5A56915F00105B5D0A36943F073
:107990000203A361A36923F44073A361B8F1000F4C
:1079A000AAD07B4B1B6D03F04053B3F1805F43D0F3
:1079B000B3F1005F00F0E180002B764818BF002093
:1079C0002B4640F2EE29DFF8DCE140F2012CB0FB5F
:1079D000F3F203FB1201C9B9B2FBF8F108FB112263
:1079E000A1F1080A92B9BAF1110F0FD809FB01F2FF
:1079F00002F5FA72AEFB02A24FEA921AB1EB921FA5
:107A0000A1EB0A0226D9802A40F2BC8001336345EB
:107A1000DDD171E7FAF7B8FE05460028A7D061234B
:107A20000022012180F807A08371F9F7D7FEAB8807
:107A30002A681B0493619AE701A855F0C7FD0298D4
:107A4000BEE700288BD0602380F807A0837195F8EB
:107A50006C2080E701F1FF3A691E013B042DAAF179
:107A6000020A41EA03434C4A43EA0A212B4628BF53
:107A7000042332440025013B120241EA436302F52C
:107A800080704649E361131D984234BF01204020B5
:107A900000EB86100144B00189008B4215601A4644
:107AA00003F10403F9D1D4F8801000F10C02830033
:107AB0004FF49A7821F03C01920008FB0678C4F854
:107AC000801042F04072C4F88430C4F8883043F427
:107AD0004033C4F8A030C4F8B050C4F8AC50C4F877
:107AE000BC50C4F8C020C4F8F050C4F8C85088F89E
:107AF0007C51C8F8885188F87D51C8F88051C8F881
:107B00008451FEF7C5F8C8F8905140F20923626D20
:107B1000012198F870501343C8F88C0102222846BE
:107B20006365E36D43F00103E3650723C4F8E030C8
:107B300053F0E8FF0123690905F01F05184AAB401F
:107B400042F82130A269114B22F00102A26101E04A
:107B5000013B02D0A269D207FAD4A369DB073FF543
:107B6000CBAE4FF49A72012302FB067787F894316B
:107B7000C2E60221F9F732FEF1E601A855F08CFCCD
:107B800002981DE7154667E7901E0024A1860100B4
:107B90000044025800127A00AC004000002B001094
:107BA00000E100E0D34D62100020F8F7F1BC00BF07
:107BB0000120F8F7EDBC00BF0246074B02209A42B5
:107BC00008D801335B0840009A4280B202D2FF28F5
:107BD000F8D97047704700BF7FF0FA022DE9F04FE7
:107BE000012385B0DFF804A30026BB4A99460AF1B9
:107BF000F00BBA4FA2F1040801960BE0019B09F1CA
:107C000001090AF1280A0BF1050B0133062B019338
:107C100000F0F1809AF80030022BEFD19BF903209D
:107C2000511C00F0EB80D2B2964602EB4204AA4B04
:107C30009DF8041003EB84040F2A5ED8A84802E0E4
:107C40000330B84259D00378002BF9D145788D42E2
:107C5000F6D18678D8F8C8506068A660A842267029
:107C600000F04681D8F8F450A84200F06081D8F8BE
:107C70002051A84200F06581D8F84C51A84200F08C
:107C80006581D8F87851A84200F07181D8F8A451E4
:107C9000A84200F08981D8F8D051A84200F07E8136
:107CA000D8F8FC51A84200F08A81D8F82852A8429E
:107CB00000F07F81D8F85432984200F09981D8F8CA
:107CC0008032984200F08D81D8F8AC32984200F0B2
:107CD000B481D8F8D832984200F0A881D8F804339B
:107CE000984200F0B881D8F83033984200F0BA8159
:107CF000D8F85C33984200F0A78101320C34D2B23C
:107D0000724599D9002303939BF90420531C79D021
:107D1000D2B2964602EB42046F4B9DF8041003EB7F
:107D200084040F2A5DD86E4802E00330B84258D070
:107D30000378012BF9D145788D42F6D18578D8F8B2
:107D4000C8606068A560B04225705FD0D8F8F46064
:107D5000B04200F0F180D8F82061B04200F0FB8022
:107D6000D8F84C61864200F0FC80D8F87861B042C7
:107D700000F00281D8F8A461B04200F00981D8F87F
:107D8000D061B04200F0FE80D8F8FC61B04200F053
:107D90002281D8F82862B04200F01781D8F85462E6
:107DA000B04200F03281D8F88032984200F027814A
:107DB000D8F8AC32984200F03381D8F8D8329842E3
:107DC00000F02881D8F80433984200F05E81D8F89A
:107DD0003033984200F05381D8F85C33984200F079
:107DE000488101320C34D2B296459AD20022002347
:107DF000CAE9042302E705B0BDE8F08F4FF00F0E8B
:107E0000002212E74FF00F0E002283E74FF0000C24
:107E100063466046CDF808C02C2606FB008090F92A
:107E2000E460002EDDD1324680F8CC3066462D4B22
:107E3000029CAC46334480F8E5900134C0F8D0C0D1
:107E4000CAF814301323154680F8E4302046F9F7B9
:107E5000A9FB039B002BC9D0DAF814603046F8F771
:107E6000CFF8DAF81000F8F7CBF8DAF81830C16874
:107E7000DAF80420596240215D60996002F1200126
:107E80009D631960C3E90355C3E90555C3E9075567
:107E9000C3E90A55C3E90C55A6B1DAF81C303032F3
:107EA000F1681D625962C3E900254FF48032C3E9CD
:107EB0000255C3E90455C3E90655C3E90B55C3E9A7
:107EC0000D559A620023204607491A46F9F78CFBA4
:107ED00001238AF80C3091E6040000247E1C0B0874
:107EE000001C0B08C4000024B9060000F035002473
:107EF0009C4602932C2000FB0C8595F9E400002899
:107F00007FF4FBAE029A604685F8CC30624B0130BC
:107F1000C5F8D060134485F8E590CAF810301423F2
:107F200085F8E430F9F73EFB01230393ECE60123E7
:107F30002C209C460290DDE74FF02C0C1846029353
:107F40006AE7022358209C460290D3E7032384204B
:107F50009C460290CEE702234FF0580C184602933D
:107F60005AE703234FF0840C1846029354E7042386
:107F7000B0209C460290BDE704234FF0B00C184699
:107F8000029349E706234FF4847C1846029343E7A3
:107F900005234FF0DC0C184602933DE706234FF40F
:107FA00084709C460290A5E70523DC209C46029045
:107FB000A0E74FF4B0704FF0080C02909AE7072347
:107FC0004FF49A709C46029094E708204FF4B07CDE
:107FD0000023029020E707234FF49A7C184602936F
:107FE0001AE74FF4DC7002234FF00A0C029081E78D
:107FF0004FF4C6734FF0090C029301237AE70A206D
:1080000002234FF4DC7C029006E709204FF4C67C83
:10801000029001E70C204FF4047C04230290FBE65D
:108020000B204FF4F27C03230290F5E64FF4047327
:108030004FF00C0C029304235CE74FF4F2734FF003
:108040000B0C0293032355E74FF425734FF00F0CED
:10805000029307234EE74FF40F734FF00D0C02937A
:10806000052347E74FF41A734FF00E0C02930623D3
:1080700040E70F204FF4257C07230290CCE60E202A
:108080004FF41A7C06230290C6E60D204FF40F7CB5
:1080900005230290C0E600BFC4000024800AA0F5BA
:1080A000801052286ED838B50C4611461A466E4BD1
:1080B0001D5C0D2D4ED805EBC5036C48490005EB42
:1080C000430300EB830023465EF0D0FF684A102C88
:1080D00059D8DFE804F0405858588A585858095879
:1080E000585870585858A4004C2303FB052393F8A4
:1080F000BC0093F8C2100128C9B22BD1012929D1A3
:10810000022183F8BC104C23022103FB052383F8D2
:10811000C210D96FCB6843F00803CB604C21012318
:1081200004F01F0401FB0521524A03FA04F4CB6F4B
:10813000196A21EA04011962196A0C431C629968E0
:108140000A40062A06D0B2F5803F03D01A6842F0F2
:1081500001021A6038BD4C2303FB052393F8BA00D3
:1081600093F8C0100128C9B2F4D10129F2D102213B
:1081700083F8BA1083F8C010D96FCB6843F00203BC
:10818000CB60CBE770474C2303FB052393F8BF106C
:1081900093F8C3300129DBB2DCD1012BDAD1231FE4
:1081A0000C2B51D8DFE803F02D505050595050504F
:1081B0001350505047004C2303FB052393F8BD1088
:1081C00093F8C3300129DBB2C4D1012BC2D14C23B7
:1081D000022103FB052383F8BD1083F8C310D96F78
:1081E000CB6843F01003CB6098E74C2303FB0523D7
:1081F00093F8BB1093F8C1300129DBB2AAD1012B4F
:10820000A8D14C23022103FB052383F8BB1083F87C
:10821000C110D96FCB6843F00403CB607EE74C23D9
:1082200003FB052393F8BE1093F8C330C9B2012BAA
:1082300090D101298ED14C23022103FB052383F821
:10824000BE1083F8C31069E74C23022103FB05230A
:1082500083F8BF1083F8C31060E74C23022103FBAF
:10826000052383F8BC104EE7881B0B08043000245C
:10827000882F0024070001002DE9F0470C4619461D
:1082800088B02368BDF840804FEA932C9DF8449055
:10829000ACF5801CBCF1520F58D82F4B13F80C6072
:1082A0000D2E53D806EBC6032C4F0546204606EB91
:1082B000430307EB8307FBF72FFE94F805A0A37990
:1082C000B9F1000F01D083F001035A004FF480711F
:1082D000DB00384602F00202CDF8088003F0080304
:1082E000039252460493602301934FF40073CDE947
:1082F0000613002301A905935CF0AAFEA379384672
:1083000051469F0725D455F0D7FA4C22144B02FB57
:10831000063393F8B920012A0FD10221DA6F83F8CE
:10832000B910104B91680B40062B06D0B3F5803F77
:1083300003D0136843F0010313602168637901F1EE
:10834000340269600021D0182860D15008B0BDE81F
:10835000F08755F047FCD8E7881B0B080430002451
:10836000882F0024070001002DE9F84F614CD4F854
:108370009C37002B00F08F805F4E04335F4FDFF897
:10838000889197F9EC031968C2B21D7B022A00F2AA
:1083900082804FF49A7200FB02F206EB020898F812
:1083A00094C1BCF1010F76D1082D74D898F87CA146
:1083B00098F87DE10AF1010C5FFA8AFA0CF00F0CD3
:1083C000F44552D00AF1020E02EB0A1821F0604B7C
:1083D000C90F02EB0E1EB044B644C8F87CB08EF84C
:1083E00068508EF8691065B11B32D91C444B02EB02
:1083F0000A120D44134411F8012FA94203F8012F6A
:10840000F9D14FF49A754FF0010805FB006595F816
:10841000703085F87CC15A0903F01F03203208FA36
:1084200003F349F82230BFF34F8FBFF36F8FF8F794
:108430000DF895F87020B4F88E07D4F89C5702F028
:108440001F01D4F888C752092B6808FA01F10138D6
:1084500049F82210C4F89C37C5F800C0C4F8885702
:10846000A4F88E07BBB104338BE70546FDF710FC7B
:10847000D8F88421D8F888319A420ED0D8F88431BF
:10848000C8E962304FF49A7303FB0566D6F8803171
:108490000133C6F88031BDE8F88FD8F88C31194A1D
:1084A000C31A9342EEDD98F870300122164C590938
:1084B00003F01F03D8F86470203102FA03F344F884
:1084C0002130BFF34F8FBFF36F8F0723C7F8D4302E
:1084D00088F87DA1D8F8901198F870301144C8F848
:1084E0008C01C8F8901103F01F015B098A4044F821
:1084F0002320C7E7882F0024901E002400000024BA
:10850000F41E00249F86010000E100E02DE9F04701
:10851000794F8CB097F8A43713B90CB0BDE8F08749
:10852000764C054694F8192794F818379A4230D0BB
:1085300004F21C7A00264FF010094FF0040894F85A
:108540001917059604EB011309FB018193F829071C
:108550005144D3F81C2742EAC07203A8029293F850
:108560002827CDE903668DF8142068F039FF2A46E4
:10857000002302A85EF02EFE94F81937013303F0B1
:108580001F0384F8193794F8192794F818379A427A
:10859000D5D15B4B5B4E03F1240103F1200403E0D2
:1085A0009C4201F1100115D053F8042FA81A002A9B
:1085B000F6D0B042F4DD0A78FF2A02F1010204D0BD
:1085C00001200A70504A82F8ED039C4201F110012B
:1085D0001D60E9D197F848382BB1D7F84C384B4A91
:1085E000EB1A934209DCD7F85438494AEB1A934204
:1085F0000EDC0CB0BDE8F047B6E60023444A87F82D
:10860000483887F85038D7F85438EB1A9342F0DDE1
:10861000D7F858380026282202A801333146C7F877
:108620005458C7F858380093ADF804608DF80660C8
:1086300068F034FF0223374802A9CDF824D08DF822
:1086400008300790E4382AA3D3E90023CDE90423B6
:1086500040F25513ADF8183018238DF82030072359
:10866000ADF8283065F07DF8D7F89887B8F1000F9D
:10867000BFD04446DFF8A090D4E90223AA1A63EBE6
:108680004303914576EB030317D2D7F8983720467A
:10869000A34217D05EF08AFD2168B7F88E37D7F86D
:1086A0008827C8F80010013B2260C7F888470C46AD
:1086B000A7F88E37002CDFD19BE7A0462468002C5A
:1086C000DAD196E75EF072FDD4F80080B7F88E3705
:1086D000D7F88827013BC7F898872260C7F88847F2
:1086E0004446A7F88E37002CC6D182E7AFF300804E
:1086F000F1C6A7C1D068080F882F0024901E00245F
:108700002C3700249F860100000000241FA10700D1
:108710003F420F00E437002480841E002DE9F0471B
:108720006B4C94F9613894F86168002B05DD94F87E
:108730006278013FFFB2022F01D9BDE8F087002126
:10874000DFF8CC81634B2C2204F5EF6088F8181712
:1087500083F8EC7304F6680588F8941688F81917FE
:1087600068F09CFE5C4B04F66841C4F89457C4F86A
:1087700080375A4BC4F87C3704F5F1631A462B4610
:10878000156020358D42F9D14FF0200A84F87867C2
:1087900000265348C4F88CA7C4F8486CA4F8906726
:1087A000C4F8846765F018F8314648224D4884F8CB
:1087B0005C68C4F8586868F071FE4B48DFF8549163
:1087C00084F85066C4F80066C4F84C6684F8FC650A
:1087D00065F002F8454864F0FFFF454884F8646698
:1087E000C4F85866C4F8606684F8656684F86666FE
:1087F000A9F8046064F0F0FF3E4864F0EDFFB4F8BF
:1088000064383D4AB3F5FA7FC4F8686C84F8786C34
:10881000A8BF4FF4FA73EE60322BB8BF3223B2FB1D
:10882000F3F3C5E90166C4F87C3CFDF731FA524622
:108830003146C4F8800C09F5A87068F02FFEFF23BC
:108840002E4884F8C83784F8D83784F8E83784F895
:10885000F83784F8083884F8183884F8283884F809
:10886000383864F0B9FF94F86638C4F8886C84F836
:10887000506884F84868C4F84C6884F8846CC9F877
:108880003466C9F83866C9F83C6693B94FF49A73F0
:108890001B4A03FB078894F8F2340A2BC8F87420AB
:1088A0000ED0FDF7F5F90123C4F8540884F8A43775
:1088B00043E7144864F090FF134864F08DFFE5E748
:1088C000124B42F21072D3F800371A61E9E700BF89
:1088D000882F0024000000240D0B0408B90A0408A6
:1088E000A82A0B088C350024B82A0B08C82A0B08C4
:1088F000D82A0B08E82A0B0840420F00F82A0B0878
:10890000550B0408082B0B08182B0B08883F002474
:10891000901E0024E035002407280ED89FED077A2A
:10892000DFED077A80FE470A064B80FE270ABDEE80
:10893000C00A10EE102A23F81020704700F8FF45F7
:1089400000000000F03B0024012070470120704728
:10895000B0F5FA6F9FED0A7A9FED0A0AA8BF4FF4AF
:10896000FA60B0F57A7FB8BF4FF47A7007EE900ADC
:10897000F8EE677A77EEC77A27EE800A704700BF75
:1089800000007A44560E034191F91B20CB7E002A49
:108990000ADD580903F01F0204490123934051F8EE
:1089A0002020134341F82030704700BF103C0024C2
:1089B0000E2809D8DFE800F0151515151515151541
:1089C000150A0C0E10121400402070470C2070473E
:1089D00010207047142070471820704720207047DF
:1089E000302070472DE9F043456A35B94162BDE852
:1089F000F083CEF800100B60F9E74E68AE462B46C8
:108A000026F0604CC6F38A47C6F3807817EA26073B
:108A100038BF67465C6894EA060F24F060420CD5C4
:108A2000002C1EDA920CBA4201D0BA420FD99D42F4
:108A3000DFD10D60DAE71346ECE7944505D104F089
:108A40008049C4F38074444507D19445EFD31A6834
:108A50009E46002AEFD11960C9E7B9F1000FF6D0A0
:108A6000E5E7BA42F3D0E0E703460122002083F8AD
:108A700029207047426A08B50346C06B996B0244CF
:108A80005A6201B18847002008BD00BF036B02464F
:108A90001B681B6A5B685B7813F0010008BF82F8F3
:108AA0002900704782634162704700BF704700BF72
:108AB00004307047036B02461B681B6A5B689B7837
:108AC00013F0010008BF82F82900704782634162F9
:108AD000704700BF03460122002083F82920704719
:108AE000426A08B50346C06B996B02445A6201B1F1
:108AF0008847002008BD00BF704700BF04307047A2
:108B0000094B1A79196802440144D2B219601A71EA
:108B10001A79120603D51A7982F080021A71034B72
:108B200001221A70704700BFB8470024F0030024E8
:108B30002DE9F84F154FBD68ED0A22D00026DFF869
:108B400050A007F10C09B0467419F9684FF01003F2
:108B5000524648BF0134D1F828B04846C7F844808F
:108B60006410E102D8470F280BDD094B03F1100117
:108B700053F8042B013207D18B42F9D12546B54277
:108B8000E2DCE802BDE8F88F661CF8E7B84700248D
:108B9000E0460124164B174A1968D36CCB1A322BC6
:108BA00004DC136ECB1A002B0FDC7047116D49B13A
:108BB00092F85C30888803F0010309681B0100FA11
:108BC00003F38B61002313667047136D63B118685C
:108BD00032319B8810B44469116623425DF8044B1E
:108BE00018BF1B048361704732311166704700BFA4
:108BF0006C350024B8470024074A136D4BB192F836
:108C00005C209988186802F001031B0101FA03F344
:108C100083610020704700BFB8470024044B4FF425
:108C2000007C00201B6FA2F800C00B60704700BFE3
:108C3000B84700240020704701207047012070478A
:108C40000020704710B41C6994420CD394460A4625
:108C500061448C42996938BFA4EB0C0261445DF811
:108C6000044B68F0BDBB5DF8044B704738B5074B4B
:108C700014460D46D3F8A0301B6A984702464FF4BD
:108C80000073002012682A60238038BDB847002492
:108C900008B5064BD3F8A03023B15B69984701387B
:108CA00040B208BD4FF0FF3008BD00BFB8470024F8
:108CB000002070472DE9F0410BB316460F4603EB39
:108CC0000208104CD4F8A050002339463046AD6855
:108CD0001A46A8470028F5D0D4F8A030002BFBD0C6
:108CE0005B6998470028F7D0013607F50077B04553
:108CF000E8D1054B00201B68E364BDE8F081014C1E
:108D0000F7E700BFB84700246C3500242DE9F04197
:108D10003BB316460F4603EB0208134C04E0D4F8AD
:108D2000A01019B14B699847D4F8A01000230D6921
:108D3000304639461A46A8470028F0D1D4F8A0306A
:108D4000002BFBD05B6998470028F7D0013607F568
:108D50000077B045E8D1054B00201B68E364BDE80F
:108D6000F081014CF7E700BFB84700246C350024C0
:108D7000002070470020704708B5F9F73BF9A0B113
:108D80000B4BD3F8F80058B1026893F8F53080889F
:108D9000126910402BB9003818BF0120013840B2C9
:108DA00008BDB0FA80F04009F8E74FF0FF3008BD89
:108DB000B847002400207047034B93F8C8000038E0
:108DC00018BF0120704700BFB8470024816D0346DB
:108DD0000A6A52681278FF2A09D090F8F020013A06
:108DE00052B2002A80F8F02006DD012070470822E8
:108DF000002083F8F02070470B6A002202205B6895
:108E00001A707047836D1B6A5B681B78FF2B0AD151
:108E100090F9F030002B03F1FF3280F8F020D4BF3E
:108E20000220012070470020704700BF836D1B6A3D
:108E30005B681B78FE2B0CD0FF2B08D190F9F0302B
:108E40005A1E002B80F8F02001DD0120704702201F
:108E500070470020704700BF034B93F8C8000328F9
:108E600094BF002001207047B84700240048704795
:108E700084480024034B93F8C800003818BF012031
:108E8000704700BFB847002470B5144C05460E4625
:108E900094F8C830042B10D0082B1CD1D4F8C03063
:108EA00083420FD0002394F89C21C4F8C4300AB147
:108EB000C4F8A031F9F79EF830B10823C4E9305660
:108EC00084F8C830022070BD054B09221B6884F865
:108ED000C820C4F8B830012070BD00BFB8470024D6
:108EE0006C350024034B93F8C800032894BF00207E
:108EF00001207047B8470024004870478448002488
:108F0000164B002030B493F82A4014B1DD698D422D
:108F100005D0013010330B28F5D130BC7047104B11
:108F2000BAB1D3F8BC1101EB40218A4201D1022C25
:108F300008D093F88C2312B9012283F88C230122E4
:108F400083F8A52103EB0013012283F8CE2130BC66
:108F5000704703EB001383F8CE21DEE75C49002461
:108F6000B847002430B400231A4C04F5D27084F8BA
:108F7000783203E0013310300B2B19D0C5698D42D4
:108F8000F8D190F82AC0BCF1030FF3D192B1D4F814
:108F9000BC1101EB43218A4205D094F88C23A2B185
:108FA000012284F8A52104EB0314012384F8CE31B7
:108FB00030BC7047D4F8742204EB0313042101324F
:108FC00083F8CE11C4F87422F2E7012284F88C23CE
:108FD000E6E700BFB8470024C0B1836823B10F4B58
:108FE000072283F8A62170470C4A042192F8A401B5
:108FF00082F8B831032882F8A611C2E96C3314BF95
:109000004FF480738023C2E96A337047034B012217
:1090100083F88C2383F8A521704700BFB84700244C
:10902000704700BF70B58CB000240D46202207A801
:1090300023462146ADF8164000902846ADF814406E
:1090400004AEADF8124006948DF811408DF8104032
:1090500064F066FA0DF116012346102228460091AD
:10906000202164F05DFA05A92346102228460091CC
:10907000302164F055FA0DF11201234610222846E2
:109080000091402164F04CFA06A9012312222846DF
:109090000091502164F044FA0DF11101234607229A
:1090A00028460091622164F03BFA2346052269219B
:1090B0002846009664F034FA9DF81040072C01D938
:1090C0000CB070BDBDF81630714ADFED726A02EA6D
:1090D0004332DFED717A6E4907EE102A1A04BDF8AB
:1090E0001430B4EEE67A02F0004267EE277A01EA25
:1090F00043319FED686A1B04F1EE10FA07EE101A77
:1091000017EE900A6249DFED647AB4EEC67AA8BF22
:1091100040F0FF40DFED5F5A67EE277A9FED5E7A01
:109120000243F1EE10FA03F0004306EE902ABDF878
:10913000122017EE900A01EA4231A8BF40F0FF402A
:10914000120406EE101A08A9034302F0004226EEAC
:10915000077AB4EEE56A9FED516A07EE903A002374
:1091600026EE866A17EE100AF1EE10FA0893B5EEB5
:10917000C06AA8BF40F0FF40F1EE10FA42EA0002D8
:10918000C1E9023307EE102A08D4DFED455AF4EEA8
:10919000E56AF1EE10FA68DD4FF6FF73DFED416A24
:1091A000ADF82230F4EEE67AF1EE10FA63D4DFED9A
:1091B0003E6AF4EEE67AF1EE10FA53DCDFED376A40
:1091C00067EEA67AFDEEE77A17EE903ADFED377A92
:1091D0000993B4EEE77AF1EE10FA51D4DFED346A78
:1091E000B4EEE67AF1EE10FA4FDC37EE677AFCEE79
:1091F000C77ACDED037A9DF80C30DDED067A9FED50
:109200002D7AF8EEE77A8DF82130F4EEC77AF1EE98
:1092100010FA33D49FED287AF4EEC77AF1EE10FA03
:1092200030DC9FED267A67EE877AFDEEE77A17EE5F
:10923000903A1BB2ADF82C300122214E4FEA041CAB
:10924000204B4FF0000E06EB04151A700FC985E88D
:109250000F0006F80CE0FCF71BFD1B4B43F8240045
:109260000CB070BD6FF00043B0E7BCEEC66A16EEFE
:10927000103A9BB292E74FF00043A7E7134BD9E7B0
:109280000023BAE747F6FF73D4E7FF23B5E700BF33
:1092900000E0FF0F0000800F000080770000C84250
:1092A00066D623440AD7A3CB0AD7A34B339388436C
:1092B0009A090444000048CA70FE474A0AD7233C72
:1092C00050370024ED030024303700240080FFFFD6
:1092D0009FED067ADFED067AE0EE077A08B5B0EE8C
:1092E000670A66F08FFD80B208BD00BFD007FA3D67
:1092F00000007A442DE9F04FCC7EA7B014B127B01E
:10930000BDE8F08F0F460DF11701234607223846BE
:10931000009121468DF817408DF8164064F000F951
:109320000DF116012346012238460091072164F011
:10933000F7F8BB8A012B40F2C88003F1FF399DF892
:1093400016301FFA89F9B9F1060F28BF4FF0060948
:10935000002B40F0CE807E4B03931B78002BCED0A9
:109360007C4E3478A1447C4B08254FF0000B5FFA0B
:1093700089F903EB04080DF1180A0FE00134CDF868
:1093800000A08DF818B064F0CBF8E4B29DF8183066
:1093900008354C4508F8013B347007D00F2C4FF0CE
:1093A00000034FF0080229463846E7D90123039A03
:1093B0001370FCF76DFC3178684B0F29186040F290
:1093C000A680DFF8AC8108F588794446A8F1100A38
:1093D000257C1022514620461DB168F0B3F90028C3
:1093E00068D011344C45F3D18022002106A89DF8A5
:1093F000175068F053F85A4B93F901205B78002A14
:1094000004DD983301226B4403F8802C434601208D
:109410001A7C113313F9011C983200296A44C8BF21
:1094200002F8800C4B45F3D10DF1980E0DF11902A5
:109430004C4C0120CEF1800C0CEB02030132C3F343
:10944000421103F01F0354F8211000FA03F30B42FA
:1094500018BF02F8010C7245EED16B1EDBB27D2BFA
:1094600006AB28BF7D2558192B46024603E0013381
:10947000D9B27E2937D012F8011B0029F7D1DDB20D
:10948000394991F82D3513F0010308D198F81020CF
:1094900008F11108002A40D00133102BF6D1C5F392
:1094A000471205F01F0101238B4054F822100B4393
:1094B00044F822301021284659F06EFB0023039A0D
:1094C0003370137027B0BDE8F08F9DF81630ABB93C
:1094D0001F4B03931B78002B3FF411AF1D4E65E724
:1094E00013F0FF050FD010F801296B1E002AF7D1E9
:1094F000C6E7184E164B3470039333E7154E144BE2
:109500003470039352E7039B35701D70F7E600201B
:1095100027B0BDE8F04F59F03FBB03EB0313134AEC
:10952000DFF834E001EB030C012381F82A351370D6
:109530008CF81C54BEE80F00CCF80C04CCF81014C6
:10954000CCF81424CCF8183407F0DEF8A7E700BFF5
:10955000D0370024D8370024B44B0024D43700245B
:10956000E8370024103C0024B84700244C1C00209D
:10957000C44B002438B590F834300446012B08D091
:1095800090F8290008B9012038BD002384F829305B
:1095900038BD006B03681A7B9AB994F82930002B08
:1095A000F1D00A4D022305F1200205F140014EF0F1
:1095B000CDF895F82130D84303F0010300F0010005
:1095C000E4E71B6A002BE8D0002038BDE046012408
:1095D00038B5044694F83430012B09D094F829307A
:1095E00013B1002384F82930012038BD1B6A23B150
:1095F000206B03681A7B002AF8D194F82930002BDD
:10960000F2D0084D022305F1200205F140014EF091
:109610009DF895F8213003F00102DB0784F829203A
:10962000E2D5D7E7E0460124F0B511F0010583B09B
:109630000BD190F834600446012E08D0C368B3F112
:10964000807F02D9012380F8283003B0F0BD0B4B96
:10965000076BD3F83005FEF7AFFAE368B880B3F1D3
:10966000807FF2D9B7212A46384633468DF8041058
:1096700001A984F828604EF069F8E6E7B8470024AD
:1096800010B5164CD4F8F8306BB1196894F8F52081
:109690009B8809690B4022B12BB1002384F8C830A4
:1096A00010BD002BF9D094F8C830032B0FD894F8D4
:1096B000BC300133DBB2072B84F8BC30EDD8084A4C
:1096C0000123126884F8C830C4F8B82010BD0548DA
:1096D000FEF772FAA4F80001E9E700BFB8470024DA
:1096E0006C350024801A0600F0B5002395B0234E97
:1096F0000446069302200B9306F180021093139305
:109700001193009206F1A00294F828701C4D01926A
:10971000226B04950D460290CDE90E3301238DF89E
:109720000C3007938DF820308DF834308DF84830A8
:1097300006F1C0030593134B099306F160030A93E6
:109740003B1D10680C9361F0F1FB9FB12A0E06F1EE
:10975000620386F861202A0A9D70280C69465A70B7
:109760001870206B4EF038F8236B186861F0DEFB40
:1097700015B0F0BD06F16103EDE700BFE04601243E
:109780008D8A0408698A040810B594B004465022F2
:109790000649684667F024FE6946206B4EF01CF8C7
:1097A000236B186861F0C2FB14B010BD442B0B088A
:1097B0002DE9F8431F46036B044688461868914616
:1097C00061F0B4FB94F82830606A002B3CD0264E40
:1097D000020E052386F8E120E236244D012FB070F9
:1097E0006B634FEA10434FEA1020337070704FF0F4
:1097F0000000D8F800302B64D9F80030AB64E36384
:10980000A86524D0022F1DD1D9F80420286513445F
:10981000D8F8041085F84C00EA6501226965E36315
:10982000134B85F860206B66124B94F82920A3F146
:109830001401206B002A08BF19464DF0CDFFA36B21
:1098400063B1E06BBDE8F88304230B4EC5E7084B1A
:1098500085F84C706865E8652B65E5E7236B18684B
:1098600061F064FBEDE700BFE0460124F003002453
:10987000758A040808040024C147012400B583B098
:109880004162019201A9049A0093012382636A460E
:10989000FFF78EFF03B05DF804FB00BF2DE9F04138
:1098A0001F46036B94B01446064618680D4661F0D7
:1098B0003DFB0B940022284C069204F590738DF822
:1098C00020201392009304F5A0730C9701930223B8
:1098D000CDE9092202930123CDE90E22CDE9102220
:1098E0001E4A8DF80C308DF834308DF848300492D3
:1098F00004F5807296F8283005921A1D079233B34A
:109900002B0E04F5817404F8013C2B0CA570DFF8D4
:1099100050802D0A23706570D8F83005FEF74CF999
:10992000346B96F82930A080A3B1694620464DF0EB
:1099300053FF346B206861F0F9FAD8F83405FEF76C
:109940003BF903463846A38014B0BDE8F08104F229
:109950000114DAE705A9E9E7E04601248D8A040845
:10996000B847002430B5002299B004469525134627
:109970008DF80C108DF80D5044F040050493012033
:1099800065F307028DF81C300A938DF830308DF89E
:109990004430159317931D4D069010908DF8580084
:1099A00002A8CDE90D33CDE913330B0E099005F173
:1099B000FC0063F30F220B0C090A63F317420DF14D
:1099C0000703059361F31F62114B0292089306236C
:1099D000104A0DEB03010B93082312920F9104A977
:1099E00085F894314DF0F8FED5F8FC20136A002B71
:1099F000FCD19DF80730FF2B00D01CB99DF8060064
:109A000019B030BD4FF0FF30FAE700BFB84700246F
:109A1000CD8D0408058E040830B597B000231E4C88
:109A20000DF107020890084608218DF814300793BD
:109A30008DF828300B938DF83C301593174D84F832
:109A400094116944099004F1FC0006959FED107B88
:109A5000CDE90232CDE910330122CDE912330223E0
:109A600004928DF850200E938DED0C7B4DF0B4FEDA
:109A7000D4F8FC30186A0028FCD19DF80730FE2B82
:109A800003D0FF2B0CBF0120022017B030BD00BF58
:109A90000000000000000000B84700242D8E0408DC
:109AA00030B52C4C9DB0FD25002301220020002163
:109AB0008DF8065004F1FC05C4F8C4308DF83C3034
:109AC00010938DF85030159318931A930E928DF8C9
:109AD0006420CDE912320DF10603CDE90C01CDE988
:109AE00016010CA9284611934DF076FED4F8FC20FF
:109AF000136A002BFCD10DF10701012228468DF8D5
:109B0000143009930B9304928DF8282084F8942143
:109B1000CDE902311049069102A9CDE907334DF094
:109B20005BFED4F8FC30186A0028FCD19DF80730A1
:109B3000FF2B08D0094A0923126884F8C830C4F8FA
:109B4000B8201DB030BD0423022084F8C8301DB0F9
:109B500030BD00BFB8470024058E04086C350024D2
:109B600010B590F834300446012B04D001200023B6
:109B700084F8293010BD006B03681A7B3AB961F094
:109B8000D9F9C24300F0010302F00100F0E71B6ABB
:109B9000002BF4D0002010BD38B5124D044694F8C7
:109BA0003430012B06D0002384F829300023012013
:109BB000E36238BD206B03681A7B72B961F0BAF9B1
:109BC00000F0010384F82930C307EFD52B68E26A5F
:109BD0009B1A002BE3DB002038BD1B6A002BEDD065
:109BE000F4E700BF6C35002410B5FF22044690F85E
:109BF0003410006B63F03CFC104B20461B680233B2
:109C0000E362FFF7C9FF94F83430012B00D010BD98
:109C10000022A021206B63F001FC94F8202094F82E
:109C200034309200012B42F01002D2B2EFD1206BFF
:109C3000B021BDE8104063F0F1BB00BF6C350024DB
:109C4000CB0700D5704710B50446FFF7CDFF94F859
:109C50003430012B00D010BDA069246BFDF7ACFFA0
:109C6000A08010BD38B504460D46FFF795FF0622CB
:109C700094F83410206B63F0FBFB0121E388D822B9
:109C800084F82910206B94F83410B5FBF3F363F0DB
:109C900011FC024B1B680F33E36238BD6C350024A6
:109CA000838853B32DE9F04104460026DFF84C8049
:109CB0000127E3882046258A03FB05F5FFF76CFFA3
:109CC000062294F83410206B06FB05F563F0D0FBF8
:109CD000E388D82294F83410206B013684F8297078
:109CE000B5FBF3F363F0E6FBD8F80030A2880F333E
:109CF000B242E362DDD8BDE8F08170476C350024E4
:109D000070B50F4D95F8383503B970BDC38804465A
:109D1000D5F83C65B6FBF3F60A4BDE67FFF73CFF70
:109D20003346102294F83410206B63F0C3FB064BCB
:109D300000221B6885F838250233E36270BD00BF3E
:109D4000B8470024F00300246C3500242DE9F04FBF
:109D5000DFF870911E46B0F806C099B099F8383512
:109D600004460D461746B1FBFCF823BBDFF858A1AB
:109D7000DAF87C30434536D1DFF840B10CFB18559A
:109D800094F83430ACEB050CB44534BF1FFA8CF6B4
:109D9000B6B2012B58D0DBF8003020460233E36224
:109DA000FFF7FAFE18B394F83430012B40D0304658
:109DB00019B0BDE8F08FD9F83C35DFF80CA1B3FB42
:109DC000FCFBCAF87CB0FFF7E7FE5B46102294F874
:109DD0003410206B63F06EFB384B1B680233E36278
:109DE000002389F838352046FFF7D6FE18B9002041
:109DF00019B0BDE8F08F4FF0FF33DFF8C0B0206B33
:109E00001322CAF87C30434694F8341063F052FBB6
:109E1000DBF8003020460233E362FFF7BDFE002886
:109E2000E5D0B4F806C0CAF87C80B5FBFCF8A5E71D
:109E3000206B61F07FF8C0F30113023B012BB6D811
:109E40002046FFF7D1FEB2E78DF81C3004A98DF84B
:109E500044308DF858301A4B99F84025089303ABDD
:109E60008DF80E502D0A099304238DF8082002AABC
:109E70000B9300238DF80D508DF80A308DF80F30BC
:109E80000A938DF830301793256B049201AA284667
:109E90000F9710960592CDE90D33CDE91233CDE938
:109EA000143303238DF80C300693C0238DF809304A
:109EB0004DF092FC286861F039F86CE76C350024AD
:109EC000B58A0408B8470024F00300242DE9F04FB8
:109ED000434E83B0D0F830A0044696F840350F4684
:109EE000DFF808919046DAF8000089F8603161F0F7
:109EF0001DF896F83835002B3FD0D6F84455E28847
:109F0000DFF8ECB0B5FBF2F302FB135389F88231B2
:109F10001B0A89F881313B685946324F5046C7F8D1
:109F2000203107F59072D8F80030C7F828310023A7
:109F3000C7F830314DF0F8FED8F800200123E18851
:109F4000154486F83835B5FBF1F301FB1353C6F819
:109F5000445513B3244BC7F8303194F829300BB96A
:109F60000BF1140B59465046E2634DF035FCA36BE0
:109F700073B3E06B03B0BDE8F08F656AE288DFF889
:109F800074B0C6F83C55B5FBF2F302FB135389F8E5
:109F9000A2311B0A89F8A131BDE7D6F83C2550460D
:109FA0000193B2FBF1F2110CFA6752BA89F8C111B0
:109FB00007F59071A9F8C22107F5A4724DF0B4FE1F
:109FC000019BD8F8002086F83835C6F83C55C4E720
:109FD000236B186860F0AAFFE06B03B0BDE8F08F58
:109FE000B8470024F0030024E18A0408E046012475
:109FF00070040024C004002433B910B51C46836BE0
:10A0000020469847204610BD60E700BF10B582B0DB
:10A010000C46019201A9049A446282636A46009345
:10A02000FFF754FF02B010BD2DE9F843DDF82080A2
:10A030000F4616460021202204461D4667F02EFAE0
:10A04000B8F1000F0CD0D8F80030B8F80A20E3813E
:10A050001B0C2382D8F804306282E3821B0C23831A
:10A06000384663F065FEF30619D4431EB8B107EB1A
:10A07000000C01E0013B12D31CF801EDBEF12E0FE4
:10A08000F8D1C01A03F10109421EB944032AA8BF3E
:10A090000322082BA8BF082390461A4606E008288A
:10A0A0000246B9464FF00008A8BF08224FF02033FF
:10A0B000394620462360636067F092F9164B04F13D
:10A0C0000800424649462381837067F089F9611E82
:10A0D000E21D11F801CFACF16103ACF1200C192B9A
:10A0E00098BF81F800C09142F3D104F10A0011F841
:10A0F000013FA3F16102203B192A98BF0B708142F6
:10A10000F5D1182365832D0CE6722373099BA58274
:10A11000E361BDE8F88300BF2020200008B554F0BB
:10A12000D9FF1B20F8F730FB08B12923C3801C207E
:10A13000F8F72AFB08B12923C38060F08DFC114891
:10A140005DF0A2FB104B93F84D25012A09D0022A9D
:10A1500005D193F85425012A12D0022A0ED00120ED
:10A1600008BD0A4AD3F83408C3F8302860F002FB6F
:10A170000023074A184682F8233008BD054AF1E754
:10A18000054AEFE7E8050024B8470024C805002485
:10A1900000ED00E088050024A8050024D7482DE93B
:10A1A000F04F006885B0DFF88493C9F84C00002BAD
:10A1B0005ED00C46154601F5FE7603EB020B1DE062
:10A1C000002D62D0D9F87C30AB4200F0C580D9F8C0
:10A1D0007830AB4200F0F780D9E92031AB424BD860
:10A1E0008D42C0F07281691A204658F04BFC01354F
:10A1F00004F5007406F500765D4539D0D9F888205D
:10A20000AA42DDD8AA1AD9F89870D308396B02F09F
:10A21000070802338B4202D3BA6B93420BD93946FB
:10A220001846039358F0FEFB039B0746002800F0F6
:10A230008681C9F898003A79002A40F01D81D7F844
:10A2400028A0BAF1000F00F073813A6B0135204667
:10A250004FF400719B1AFA6804F5007406F5007655
:10A2600008EBC3083B4602EB4822D0475D45C5D109
:10A27000002005B0BDE8F08F8D42B4D24FF40072DB
:10A280000021204667F00AF9B1E74FF40072294631
:10A29000204667F003F98023994A84F8BE310C23E5
:10A2A00084F8C231D9F87810D9F870309142C4F8E6
:10A2B000C611C4F8CA3100F30D81924A013B924F96
:10A2C00082FB0102C81787FB01C70A44C0EB621278
:10A2D000C0EB27308D4F87FB02C7C2EB821C84F88E
:10A2E000C1018010A1EB0C01174420F03F000131A7
:10A2F0000843D117C1EBE71184F8C0010A4484F880
:10A30000BF217F4A934200F3F1807E4A7E4882FB60
:10A310000312D91780FB03701A44C1EB6212C1EB20
:10A3200020317A4880FB0270C2EB821784F8C51195
:10A330008910DB1B104421F03F0101331943D3176F
:10A34000C3EBE01384F8C4111A4484F8C3214AF61D
:10A350005523A4F8FE314AE74FF0FF3300274FF4AE
:10A36000F072201D84F8EC31394684F8ED3184F820
:10A37000EE3184F8EF315223237063706123A370B0
:10A3800084F8E7314123E37084F8E631722384F8DE
:10A39000E43184F8E531D9F89030C4F8E83167F059
:10A3A0007DF85523C4F8F07184F8FE316FF0550341
:10A3B000C4F8F471C4F8F87184F8FC7184F8FD7184
:10A3C00084F8FF3113E74FF400720021204667F054
:10A3D00065F84F4B022203CB45F6EB032274227340
:10A3E00023809023A273A370F82384F82C200822E2
:10A3F000C4F803006273C4F807106375D9F87810C5
:10A40000D9F870305B1A2362D9E920135B1A4AF637
:10A41000552163620023E372E3736377A377E377E5
:10A4200084F82D3084F82E3084F82F3084F83130C1
:10A43000384BA3613E232377012384F830308023F7
:10A4400084F84030344BC4F84230344B84F8462012
:10A45000A4F8FE11324A03CBC4F84B101988C4F893
:10A4600047009B78A4F84F1084F8513003CAC4F811
:10A470005200C4F85610BAE64FF40072002120468C
:10A4800067F00CF83B6CB8F1000F5FD104F1200AC3
:10A49000002B00F09B803B6B112222492046CDE926
:10A4A0000088FFF7C1FD3B6C1A6C002A00F09B800E
:10A4B0001B6B504611221C49CDE90088FFF7B4FD03
:10A4C00004F1400A4FF4E0788BE0E91A204658F096
:10A4D000D9FA8CE6FF22013B84F8C1214FF6FF72C6
:10A4E000A4F8BF21064A93427FF70FAFFF2384F8F9
:10A4F000C5314FF6FF73A4F8C33128E76C3500244B
:10A50000FF03FB00832008829755454181808080AE
:10A5100040C50B083F00FF0029940E0D4CC50B08E9
:10A5200058C50B0838C50B083CC50B08B8470024B4
:10A5300051464FF40072204666F0B0FF57E6231FE5
:10A540002D4A43F8042F9E42FBD150E6002B7F6C2E
:10A5500014BF02230123C3EB0813002F3FF447AEBF
:10A56000013BBF6C002B01DD002FF9D1A2464FF457
:10A570000078002F3FF43BAE0AEB080303959A46A0
:10A580000BE00025A8F12008CDE900E5FFF74CFD20
:10A59000BF6CCFB1B8F11F0F16D93D7907F11C0E72
:10A5A000112239683B6BAAEB0800002DE9D17A79BA
:10A5B000A8F120083D6942F02102CDE900E5FFF74E
:10A5C00033FDBF6C002FE5D1039D10E6CDE9008877
:10A5D00043464FF4F0780822D9F874102046FFF76C
:10A5E00023FD7F6CC5E75046434611220349CDE960
:10A5F0000088FFF719FD63E7DEADBEEF3CC50B0831
:10A6000010B50E4C236D4BB194F85C2099881868F6
:10A6100002F001031B0101FA03F3836158F0C4F94E
:10A62000D4F8A030002BFBD05B6998470028F7D006
:10A63000034B00201B68E36410BD00BFB847002433
:10A640006C35002408B5F8F71FFA58B1114A92F892
:10A65000BC300133DBB2072B82F8BC3003D90023B6
:10A6600082F8C83008BDD2F8F83043B1186892F8C3
:10A67000F5109B880069034049B1002BEFD1064BD0
:10A6800001211B6882F8C810C2F8B83008BD002B41
:10A69000E5D0F4E7B84700246C35002410B5037901
:10A6A0001A4C002B14BF0122002284F8F4201AD087
:10A6B000174BD4F8F8205B78003B18BF012384F8CF
:10A6C0009C31AAB111689388096994F8F5200B4070
:10A6D00062B96BB994F8BC300022013384F8C82009
:10A6E00084F8BC3010BD84F8C83010BD002BF1D107
:10A6F000F8F7CAF90028EDD1064B012284F8BC0016
:10A700001B6884F8C820C4F8B83010BDB8470024CE
:10A71000702E00246C35002410B51C4C94F85105A3
:10A72000F8F732F828B11F210022C1802021F7F765
:10A7300055F8236D4BB194F85C209988186802F0A5
:10A7400001031B0101FA03F38361114B0021032074
:10A7500093F90320F6F794FE60B1436853B1D4F83F
:10A76000F8305BB1196894F8F5209B8809690B40B3
:10A7700012B11BB1012010BD002BFBD0F8F784F9FA
:10A780000028F7D1034B1B68E36410BDB8470024D1
:10A79000702E00246C35002410B58078F7F7F4FF94
:10A7A00090B10A494FF0410C04460022D1F83838E4
:10A7B00080F806C00133C1F838382021C371F7F79B
:10A7C0000DF82368A2889A6110BD00BFB847002425
:10A7D0000E4838B5D0F8F8300D4614463BB119682C
:10A7E00090F8F5209B8809690B4052B15BB9F7F7E7
:10A7F0002DFC074A4FF400730020926C2A602380DE
:10A8000038BD002BF3D14FF0FF3038BDB8470024DE
:10A81000402F0024F8B5914C94F8F460002E00F01D
:10A82000CE8094F8C8506B1E082B20D8DFE803F0C8
:10A83000A89B571F3905AC1F2A00894B5B6A002B68
:10A8400040F09B80874B0722D4F8B0501B6884F8F7
:10A85000C820C4F8B830002D00F08F80D4F8B43090
:10A860000120D4E92921A84794F8C8506B1EDBB217
:10A87000022B7BD9042D18BF082D0CBF0126002602
:10A880003046F8BDF7F7B6FB002840F0CF80754A98
:10A89000D4F8B8301268FA339342EBD2FFF7D2FE05
:10A8A000BFE76F4B1F6A002F40F0B780F7F7A2FB9E
:10A8B0000028B6D00423D4F8B05084F8BC7084F8D3
:10A8C000C830002DDCD0D4F8B4303846D4F8A420F9
:10A8D000D4F8A810A84794F8C8506B1EC7E7F7F73C
:10A8E000B5FB002842D1604BC4F8C40093F82C108B
:10A8F000DA8D84F8D210A4F8D020196B1A6B090EE7
:10A90000120C84F8D31084F8D4201A6B196B120A35
:10A9100084F8D61093F8341084F8D52084F8D71032
:10A9200093F8351093F83520090902F00F0284F8E6
:10A93000DC1084F8DD209A6BD88FC4F8D820DA8F29
:10A94000D98FC2F30B1301F00F02042143EA102345
:10A9500084F8E02003F00F0384F8C81003F5FA63CD
:10A96000A4F8DE305DE7F7F745FB60BB3D4BD4F85C
:10A97000B8201B689B1AC82B44D800263046F8BD67
:10A98000022384F8C8304CE7F7F734FB00283FF483
:10A990007EAFD4F8C4200023012A84F8BC3049D902
:10A9A000D4F8C010013A0131C4E9301294F89C2166
:10A9B0000AB1C4F8A031082384F8C83060E73046F3
:10A9C00084F8C860F8BDF7F741FB0028CED1274BCB
:10A9D0001B78002BA3F10203B3FA83F308BF012510
:10A9E0005B0984F8BD5084F8BE30F7F72FFB0028D0
:10A9F0007FF454AF1C4B03229B6C84F8C820C4F82E
:10AA0000CC300EE7FFF71EFE94F8C860042E18BF86
:10AA1000082E0CBF0126002632E7124AD4F8B830BF
:10AA2000126864339342FFF4FCAE23E7042384F8F6
:10AA3000C83025E7FAD194F89C21C4F8C4300AB193
:10AA4000C4F8A031F7F7D6FA0028EFD1054B092258
:10AA50001B6884F8C820C4F8B8308EE7B8470024D3
:10AA60000C2F00246C350024402F0024982F002444
:10AA70002DE9F8432B4C80468946174694F8C8C008
:10AA80001E46BCF1040F13D0BCF1080F02D0002009
:10AA9000BDE8F883002394F89C21C4F8C4300AB1BF
:10AAA000C4F8A031F7F7A6FA28B3042384F8C83015
:10AAB00019F01F0F27D101251B4A1C4B4146156277
:10AAC0004FF400724846C4F840985A602A469D6088
:10AAD0005AF01CF9B8B9164B05222846C4F8A490C0
:10AAE0001B68C4F8A88084F8C820C4F8B830C4E94A
:10AAF0002C76BDE8F8830E4B09221B6884F8C82029
:10AB0000C4F8B830C3E7FFF79DFDD4F8B050002D6E
:10AB1000BDD00022D4F8B430D4F8A8101046A8470D
:10AB2000B5E700BFB84700240C2F0024F84F0024DD
:10AB30006C3500242DE9F843DFF8AC800846114657
:10AB40001A46D8F8F8403CB12568A3882C69234000
:10AB500098F8F5407CB383BBC3062ED101231F4C6C
:10AB6000C8F8400823624FF40073C8F84828C8F8B2
:10AB700044385AF0CBF800BB236A002BFCD1DFF835
:10AB80006C9041F20D16164FD9F84450D9F8004098
:10AB90002D04A56041F28832E3680D2120463B4038
:10ABA0003343E36053F068F858B1D9F834300343C5
:10ABB000C9F83430EDE7002BCED14FF0FF30BDE8BF
:10ABC000F883636903F4F053B3F5006FE1D1054BEB
:10ABD0001B68C8F84C30BDE8F88300BF0C2F002478
:10ABE000C0E0FEFF6C350024B8470024902E0024FE
:10ABF0002DE9F843DFF8948010460A46D8F8F8406B
:10AC00003CB12568A1882C69214098F8F54084B3AF
:10AC100089BB00215AF0F6F868BB194A536A002B29
:10AC2000FCD1DFF86C9041F20D16164FD9F8445064
:10AC3000D9F800402D04A56041F28832E3680D2167
:10AC400020463B403343E36053F016F828B1D9F86F
:10AC500034300343C9F83430EDE7636903F4F0534B
:10AC6000B3F5006FE7D1084B1B68C8F84C30BDE85E
:10AC7000F8830029CDD14FF0FF30BDE8F88300BF45
:10AC80000C2F0024C0E0FEFF6C350024B8470024E0
:10AC9000902E00242DE9F0473E4C1F4605460E46F7
:10ACA00094F8C8309046042B13D0082B40D1D4F828
:10ACB000C03083420DD0002394F89C21C4F8C430E6
:10ACC0000AB1C4F8A031F7F795F950B3042384F81A
:10ACD000C830D4F8A091C9F34F230F2BC4E92965DC
:10ACE00029D8D4F8C4A0BAF1000F24D094F89C312C
:10ACF0000BB329484FF400723146484466F070FBAC
:10AD000009F50073C3F34F22C4F8A0315B0A102A7F
:10AD100002D0BAF1010F2ED19BB21F4E5A1EAD1AAE
:10AD20000AE01E4B09221B6884F8C820C4F8B8301A
:10AD30000120BDE8F087012306212846012532467F
:10AD400084F8C8100021C4F8B080C4F8B47084F846
:10AD5000AC505AF057F80028EBD0FFF773FCD4F84A
:10AD6000B06036B1D4F8B4300022D4F8A810284628
:10AD7000B0470320DDE7D4F8C0200AF1FF330421F7
:10AD800002200132C4F8C43084F8C810C4F8C020CE
:10AD9000CFE700BFB8470024A06200246C35002430
:10ADA000F0B503798BB02F4D002B14BF0122002288
:10ADB00085F8F42003D185F8C8300BB0F0BD05F15B
:10ADC000FC07044690F9001038464CF079FFA6784D
:10ADD000002E39D1244B2548C5F89031C5F80461BF
:10ADE000FCF7EAFEA5F800014FF47A70FCF784FA4C
:10ADF000D5F8043113B11A689B8893611C4CEC465A
:10AE00000FCCACE80F000FCCACE80F0094E80300C7
:10AE10008CE80300694638464CF0DEFCD5F8FC307F
:10AE20001A6A002AFCD11EB10D213046F6F7D6FC75
:10AE3000104B012100221B6885F8C81085F8BC2042
:10AE4000C5F8B8300BB0F0BD3046F7F79DFC0646AC
:10AE50000028BFD01E2300222C21C380F6F7BEFCA1
:10AE6000B8E700BFB84700245C480024801A0600F9
:10AE7000942B0B086C3500242DE9F041A34C92B0C3
:10AE800094F8F460002E00F0E98194F8C8305A1E5E
:10AE9000082A00F26E81DFE812F033006E00BB007A
:10AEA0006C013F017C011B006C01090057F04CFD57
:10AEB000002840F0C482964AD4F8B8301268FA33B9
:10AEC000934280F05381FEF7DBFB94F8C830DEE755
:10AED00057F03AFD0028EED0D4F8C4300022012B00
:10AEE00084F8BC2040F2C682D4F8C020013B08217F
:10AEF0000132C4F8C43084F8C810C4F8C02001E19D
:10AF000000210846FEF72EFDD4F8FC20C5B2136AD6
:10AF1000002BFCD10A20FCF751F9D4F8043113B10D
:10AF20001A689B889361012D40F02081002740F230
:10AF3000AB11082084F8BD70FEF714FDC0B20528DF
:10AF400000F0E481012800F0C181D4F8FC20136AEC
:10AF5000002BFCD10A20FCF731F9D4F8043113B1ED
:10AF60001A689B88936194F8BD30002B00F06482CE
:10AF7000022384F8C83094F8BD5000213720A5F191
:10AF80000205FEF7EFFC2920B5FA85F56D09AD073E
:10AF90002946FEF7E7FCD4F8FC20C5B2136A002B63
:10AFA000FCD10A20FCF70AF9D4F8043113B11A686D
:10AFB0009B889361002D40F0D98094F8BD30022B1E
:10AFC00000F0EE810021092084F8BE50FEF7CAFC93
:10AFD000002800F0A0810025D4F8FC20136A002B83
:10AFE000FCD10A20FCF7EAF8D4F8043113B11A684E
:10AFF0009B889361002D00F0B98000210A20FEF7A4
:10B00000B1FCC0B2002840F0BA81032384F8C830F4
:10B01000102103A8FEF700FD002840F0A780BDF82E
:10B020000D309DF80C205BBA9DF8111062F30700FB
:10B030009DF80F20A4F8D0309DF8193062F30F204E
:10B040009DF810201B019DF8145062F317409DF8E5
:10B050001A20DBB261F31F60DDF8151043EA12130A
:10B0600002F00F0209BAC4F8D20003F5FA6384F8BB
:10B07000E020C4F8D8102909A4F8DE30BDF8123059
:10B08000D4F8FC20A4F8D63005F00F0384F8DC10C7
:10B0900084F8DD30136A002BFCD10A20FCF78EF80F
:10B0A000D4F8043113B11A689B88936194F8BE30C8
:10B0B000B3B94FF400711020FEF754FCD4F8FC2013
:10B0C000C5B2136A002BFCD10A20FCF777F8D4F83C
:10B0D000043113B11A689B889361002D7FF4F3AE9D
:10B0E0000C48FCF769FD04220021A4F80001134676
:10B0F00084F8C820C4F8C410042B18BF082B0CBF58
:10B1000001260026304612B0BDE8F081B847002481
:10B110006C35002440787D014FF40071D4F8A40010
:10B12000FEF77AFC012800F09F80022800F0A4803E
:10B13000E0B9D4F8FC20136A002BFCD10A20FCF7FC
:10B140003DF8D4F8043113B11A689B889361042345
:10B150000020D4F8B05084F8C83084F8BC00002D2A
:10B16000D0D0D4F8B430D4E92921A84794F8C83015
:10B170005A1ED2B2022ABFD8BA4BD4F8B8201B68E4
:10B180009B1AC82B00F297800026304612B0BDE80B
:10B19000F081D4F8FC20117B136A002946D0526953
:10B1A000002A43D094F88421002A3FD0B3FA83F3D5
:10B1B0005B09002BDAD0002302A90122AA48ADF8CE
:10B1C00008308DF81830079308938DF82C301193C0
:10B1D0008DF84020CDE90313022105910DF10701FF
:10B1E000CDE9091203A9CDE90C33CDE90E334CF0BA
:10B1F000F3FAD4F8FC301D6A002DFCD19DF807301D
:10B2000003F01F03052B00F00181FEF739FAD4F893
:10B21000B070002F3FF439AED4F8B4302A46D4F8D9
:10B22000A8100120B84794F8C83030E6D4F8A4300C
:10B23000002294F8AC108C4803EB01214FF480738A
:10B240004CF084FA94F8AC200132D2B2A2F102039D
:10B2500084F8AC20B3FA83F35B09AAE7304684F89C
:10B26000C86012B0BDE8F0817E4AD4F8B8301268E8
:10B2700064339342BFF47AAFD4F8FC20136A002BF6
:10B28000FCD10A20FBF79AFFD4F8043113B11A68F5
:10B290009B889361FEF7F4F9D4F8B050002D3FF489
:10B2A000F4AD0022D4F8B430D4F8A8101046A84762
:10B2B00094F8C830EBE5FEF7E3F994F8C860082E7F
:10B2C00018BF042E0CBF012600261BE702AB03A902
:10B2D00065480493042303978DF818700797059326
:10B2E0000A978DF82C500C97CDE908774CF074FA3A
:10B2F000D4F8FC20136A002BFCD19DF80B30AB2B4B
:10B300007FF425AE022384F8BD3020E6D4F8FC207B
:10B3100084F8BD501BE610215448FEF77DFB002841
:10B320007FF459AE94F8F33013F001033FF453AEB9
:10B3300094F8E420921100F0B280012A7FF44BAE21
:10B3400094F8EB2016214A4F02259200D2B2C5F1A3
:10B3500008038B4228BF0B46C3F108059840C91A61
:10B3600042FA05F24FF0000540EA020017F8012FFB
:10B37000EDD1013083023546C4F8CC302CE6D4F848
:10B38000FC20136A002BFCD10A20FBF717FFD4F82E
:10B390000431002B3FF497AD1A689B88936192E5C6
:10B3A00029463A20FEF7DEFA02ABC7B203A904939E
:10B3B00004232D480593012303958DF82C308DF837
:10B3C00018500C95CDE90755CDE909554CF004FA14
:10B3D000D4F8FC301A6A002AFCD187B91A6A002A0C
:10B3E000FCD10A20FBF7EAFED4F8043113B11A6845
:10B3F0009B889361029D2DBAC5F38075E2E51A6AB8
:10B40000002AC1D01A6A002AF9D1BDE7154B0722DC
:10B41000D4F8B0501B6884F8C820C4F8B830002DA8
:10B420003FF4B2AED4F8B4300120D4E92921A847C2
:10B4300094F8C8305A1E9CE684F8C830A4E6D4F8C4
:10B44000FC20136A002BFCD10A20FBF7B7FED4F8CE
:10B45000043113B11A689B889361042384F8C830BF
:10B4600050E600BF6C350024B44800249C480024FA
:10B47000A34800245BD00423D4F8FC2084F8C8300F
:10B48000136A002BFCD10A20FBF798FED4F8043194
:10B49000002B3FF46BAE1A689B88936166E694F8C4
:10B4A000E9001146DFF89CC0032500F00F0294F874
:10B4B000ED00062780019340C0B2C7F10802AA42FE
:10B4C00028BF2A46C2F108079140AD1A40FA07F09A
:10B4D0004FF0000741EA00011CF8010FEDD194F88C
:10B4E000EA000231DFF860E00C2780014FF0060C23
:10B4F000C0B2CCF108024FF0000CBA4228BF3A4665
:10B50000C2F108089540BF1A40FA08F045EA000564
:10B510001EF8010FEDD10135D81705FA01F2A2FB93
:10B52000033102FB00125B0A43EAC25323E7FEF732
:10B53000B7FA02287FF41AAED4F8FC301A6A002A4F
:10B54000FCD1A0E7A5480024A24800242DE9F04141
:10B550000546884617461E46304C94F8C800042815
:10B560000BD0082807D1D4F8C030AB4242D0FEF748
:10B5700097FA0228F1D0012038E094F8BE30BBBB26
:10B5800069021820FEF7EEF9C0B2A8BB94F8C830E3
:10B59000082B2FD0FE23D4F8FC2084F84C38117BE4
:10B5A0001F4BC3F8588251B1526942B194F88421BB
:10B5B000002A14BF4FF400724FF4807201E04FF480
:10B5C000807218481849C3F860224CF005F901222E
:10B5D00006230020C4F8A480C4F8A850C4F8B070B2
:10B5E000C4F8B46084F8AC2084F8C830BDE8F081B9
:10B5F0002946C6E7FC23CEE7D4F8FC20136A002BCB
:10B60000FCD10A20FBF7DAFDD4F8043113B11A6833
:10B610009B889361FEF734F80320E7E7B8470024DE
:10B62000F0030024B44800242006002470B5224E04
:10B6300005460C4696F8C830042B09D0082B20D1BB
:10B64000D6F8C03083421AD0FEF72AFA022818D161
:10B6500000213720FEF786F921461720FEF782F9F0
:10B66000C0B2B0B996F8BE306BB969021920FEF7C6
:10B6700079F970B90823C6E9305486F8C830022039
:10B6800070BD012070BD29461920FEF76BF9002816
:10B69000F0D0D6F8FC20136A002BFCD10A20FBF76F
:10B6A0008DFDD6F8043113B11A689B889361FDF7BC
:10B6B000E7FF032070BD00BFB84700242DE9F0412B
:10B6C000224C07468846164694F8C8C01D46BCF171
:10B6D000040F09D0BCF1080F02D00020BDE8F081B2
:10B6E000FEF7DEF90228F8D194F8BE30ABB1394646
:10B6F0001120FEF737F9C0B2B0B9154B0522012071
:10B70000C4F8A4801B6884F8C820C4F8A870C4F8E2
:10B71000B060C4E92D53BDE8F08179021120FEF735
:10B7200021F9C0B20028E8D0D4F8FC20136A002B1D
:10B73000FCD10A20FBF742FDD4F80431002BCCD019
:10B740001A6800209B889361C8E700BFB8470024AF
:10B750006C3500240021032008B5F6F7C7FA72B64D
:10B76000F8F7A8F8154C08B5D4F8503894F85608EE
:10B77000ABB91420FBF7C0FD00BFD4F850385BB163
:10B78000196894F856289B8809690B4012B91BB1B7
:10B79000FFF7E0FF002BFBD0FDF7FCF9ECE71968A1
:10B7A0009A880B69134020B1002BE2D10B6913403A
:10B7B000FAE7002BDDD00B691340FAE7B847002405
:10B7C0002DE9F047089E01F007054FF47F4900EB93
:10B7D000D1014FEAD6082A4406F00706954201D166
:10B7E000BDE8F08705F0070C06F0070A501BEC08CF
:10B7F000D44567460C5D38BF574604FA0CF4C7F1D0
:10B80000080724FA0AF4874228BF074608EBD60047
:10B8100029FA07FC13F800E03D443E445FFA8CFC33
:10B820008EEA04044CFA0AFC04EA0C048EEA040EC4
:10B8300003F800E0D2E700BF314B2DE9F04793F861
:10B84000049090B0B9F1000F02D110B0BDE8F087BC
:10B850000024C9EBC90802AF2A4E4FEA480841F656
:10B86000FF7A25460294BC81C7E9014436F9021FDC
:10B870003B4600940E3451454FF00E02A8BF51468E
:10B8800021EAE17189B2C1F30720CDE90655ADF88F
:10B890001810810006A88DF819100021FFF790FFFD
:10B8A0004445E3D109F1FF392822002106A865F0BB
:10B8B000F5FD15225FFA89F90E23022006A913FB74
:10B8C000092340F206448DF81800DB080E480D9756
:10B8D000ADF83830ADF8284007A3D3E90023CDE90F
:10B8E00008230A4A08230B928DF8303061F039FFA3
:10B8F00010B0BDE8F08700BF1D95ECD7875C7F21B5
:10B900004C1C0020EE3B002400370024003C0024A7
:10B910000E4B9B780A2B00D0704710B5FAF7B8F998
:10B920000B4A0C4913680968C31A8B4203DB0A4CA3
:10B930001060237803B910BDFFF77EFF2378002B3A
:10B94000F9D0BDE81040FCF70FBD00BF78340024EB
:10B95000083C0024043C00242C3700240B4B00221C
:10B9600010B50B4CC3E90022C3E90222FAF790F9A3
:10B97000084A2378106003B910BDFFF75DFF2378F4
:10B98000002BF9D0BDE81040FCF7EEBCF03B0024E2
:10B990002C370024083C00240B4B002210B50B4C24
:10B9A000C3E90022C3E90222FAF772F9084A2378B0
:10B9B000106003B910BDFFF73FFF2378002BF9D0CB
:10B9C000BDE81040FCF7D0BCF03B00242C3700242D
:10B9D000083C002480EA0120082341F2210201B240
:10B9E000013B4000002980B2B8BF504013F0FF0374
:10B9F000F5D1704738B50C468D18AC4200D138BD32
:10BA000014F8011BFFF7E6FFF7E72DE9F843078C71
:10BA10000446072F1DD900254FF6FF73D0E9029881
:10BA2000C5F12006A5F1200029FA05F1083508FA2C
:10BA300006F628FA00F0314301431846C9B2FFF771
:10BA4000C9FF402D0346EBD13A46E169BDE8F84312
:10BA5000D0E74FF6FF70BDE8F8830346406848B171
:10BA6000026899895A605A89013292B291425A8188
:10BA700038BF9A8170472DE9F74F1C465B6907462E
:10BA800088460092002B00F0C580238C2BB1E26920
:10BA9000002A00F0BF80072B49D807F10C00FFF700
:10BAA000DCFF054620B96FF0020003B0BDE8F08F5F
:10BAB0001422002165F0F2FC228CE16905F10800F6
:10BAC00065F08EFC208C013080B208280DD90C283E
:10BAD00023D9102823D9142823D9182823D920287A
:10BAE00023D9312834BF0E200F20FCF761FF431EFD
:10BAF000294638469BB25A1C23842B442A74626917
:10BB0000127802F01F0262F03F021A7248F00043FE
:10BB10006B60FCF767FF0120C7E70920E5E70A2013
:10BB2000E3E70B20E1E70C20DFE70D20DDE7023340
:10BB30000722C18A9BB20633B3FBF2F3828A9BB21F
:10BB4000521A92B29342AED8002500F10C034FF086
:10BB50008009AA462E460193238CB34201D128B214
:10BB6000A3E70198FFF779FF834600289BD01422B2
:10BB7000002165F093FC6EB9009B0222ABF80830FF
:10BB8000B4F820C031460BF1080E8EB2B44503D88C
:10BB900090B20CE00022F3E7E069405C01310EF85E
:10BBA0000200013290B20728EFD10136B6B201305F
:10BBB000B44508BF4FF0400980B2082807D90C28C7
:10BBC00024D0102824D9152834BF0B200C20FCF7D2
:10BBD000EFFE62690138013512781BFA80F10130FD
:10BBE00002F01F0242EA4A128AF0010A49EA0202FE
:10BBF0004FF000090A7248F000428BF810005946D5
:10BC00003846CBF80420FCF7EDFEA5E70920DEE777
:10BC10000A20DCE76FF0010047E700BF3A4A4FF027
:10BC2000D0532DE9F0411268AAB000240E460C93BF
:10BC300006230B920746354A0BADADF83840CDF8D8
:10BC40003A400D93CDF83E40ADF84240D2F800386E
:10BC50001193D2F804182E4B1291D2F808288DF8BF
:10BC60005440CDE9132407CB1B88CDF85500684616
:10BC7000CDF859102146CDF85D202822ADF861306D
:10BC800065F00CFC37230795F57EADF820300123D5
:10BC9000ADF8103006F11903B67E05931F2E8DF80E
:10BCA000186017A3D3E90023CDE9022319D897F828
:10BCB0000080B8F1000F14D02D026846FFF7A5FEF2
:10BCC000144945EA066502466B46384645EA0805CA
:10BCD0002943FFF7D0FEA04203DD9DF80030012B81
:10BCE00002D02AB0BDE8F081059A13780133DBB2A7
:10BCF0001F2B94BF137014702AB0BDE8F08100BFF1
:10BD00009E6AC421818A46EEE037002400E0F11FDC
:10BD100064C50B08800001000448C3681BB1DB6ADE
:10BD20000BB10C3018470248704700BFB8470024D9
:10BD3000BC2B0B0870B5104C4FF0000C234693F849
:10BD400000E00633864512D00CF1010CBCF1060F61
:10BD5000F5D10A4ED6F87C58052D07D00CFB0543CB
:10BD60000135C6F87C58187059809A8070BD06233A
:10BD700003FB0C43F7E700BF10500024B847002432
:10BD800038B51B4CD4F880381A882AB9002384F8B7
:10BD90008C382371236038BDD4F87C180029F5DD78
:10BDA000D4F884089D7B43880DB901290DD000216A
:10BDB0000122A4F88A38002384F8881884F8892896
:10BDC00084F88C382371236038BD81880131C91A09
:10BDD0009142ECD12046002250F80C3F62641B696E
:10BDE0009847012384F8883884F88938CEE700BF63
:10BDF000B84700240548836813B190F889380BB11F
:10BE00000020704750F80C3F5B681847B847002483
:10BE1000144A30B4144D13794560EC1892F88C38FC
:10BE200004601079834214D81079834206D300232A
:10BE30001A46184630BCC1E90032704710791A1E04
:10BE4000C0F180030CBF0120022030BCC1E90032E8
:10BE500070471479002201201B1B30BCC1E900325D
:10BE6000704700BFB8470024A04B01240C4B1A793F
:10BE700093F88C081A7990421A790CD8904203D31F
:10BE80001B680020184470471A791B68C2F18002B1
:10BE9000104418447047801A1B681844704700BF4C
:10BEA000B847002438B5384C94F88938012B00D0B5
:10BEB00038BDE36804F10C0094F888585B68002DE5
:10BEC0002DD198470028F3D0D4F88428B4F88A38C4
:10BED00092889A4235D3D4F8802820465168656408
:10BEE00003FB01F150F80C3FDB689847E3689B685F
:10BEF0002BB104F10C00984708B958F03DFAB4F89A
:10BF00008A38626D0133A4F88A38002AD0D01168CB
:10BF100093884A69134218BF1B048B6138BD984748
:10BF2000F8B9A36B002BC3D0F9F744FD174BA26BF4
:10BF3000A3FB0013D2EB9312BAD4BDE8384058F0FB
:10BF40001BBA626D94F85C3084F88958002AAFD02F
:10BF5000C3F34003918812681B0101FA03F3936154
:10BF600038BD0023616D94F85C20A36384F88838A1
:10BF700084F8893800299BD0C2F340028B88096875
:10BF8000120193408B6138BDB8470024D34D621035
:10BF900010B5154CD4F88028937B012B06D023686C
:10BFA00003F2FF736FF30A03236010BDE3685B6A5B
:10BFB0005BB104F10C009847E3689B681BB104F186
:10BFC0000C00984768B1D4F8802823685288013B58
:10BFD000514213440B4003F2FF736FF30A032360D3
:10BFE00010BD58F0C9F9EEE7B847002470B5194CF8
:10BFF00084B0194B22790393134494F88C1802935C
:10C0000023799942237914D899420BD225790E4687
:10C01000C5F18005D1B92B4601223F2BCDE9005651
:10C020000CD858B92079401AB0FA80F0400904B011
:10C0300070BDCB1A002601221D46EEE7694600239B
:10C0400002A861F099F994F88C18EBE76B180222BA
:10C05000E3E700BFB8470024A04B01242DE9F043DB
:10C06000164685B0002936D0451E254CDFF898804D
:10C070004FF000096F180BE02379084699422379A5
:10C080001AD2C3F1800318443F2818D8AF4222D0F7
:10C0900094F88C0815F8013F411C08F80030C9B22B
:10C0A0000B0684F88C18E7D50020237984F88C9847
:10C0B000014699422379E4D3C01A3F28E6D923796F
:10C0C0009942E3D00F4B1B78002BDFD00020FFF705
:10C0D0008DFFAF42DCD1694602A8FFF799FEDDE98A
:10C0E000003213443F2B00D910B905B0BDE8F083EE
:10C0F0000246334602A861F03FF905B0BDE8F0837F
:10C10000B8470024F0030024A04B012430B585B0CB
:10C11000694602A8FFF77CFE50B9084C04F10C05F3
:10C12000E36828465B6898470028F9D005B030BD21
:10C130000246012302A861F01FF9EEE7B847002488
:10C1400038B5104C0023A36056F012FDC4F88408E3
:10C15000FFF7E2FDD4F88438C4F880088BB1598821
:10C160009A884368521A02FB0333A360FCF7E0FC91
:10C170002379054694F88C289A4201D0FFF7C6FF30
:10C18000256038BDB84700242DE9F0410D4C164616
:10C1900082180546A3680F469A4294F88C2888BFF7
:10C1A0001E1A23799A4201D0FFF7B0FF00203346D0
:10C1B0003A4629466064E068846A0348A446BDE8BC
:10C1C000F0416047B8470024C44700248C4613461A
:10C1D000014662461846D7E72DE9F04F41F62C722A
:10C1E00089B00021B94865F059F90420F5F778FDC8
:10C1F00004460520F5F774FD54EA000340F057812A
:10C20000B34B0193019BE422B249B048D3F8B0424A
:10C2100065F0E6F8AD4B1E465C621C67C3F8B4409F
:10C22000C3F8B840C3F8BC40C3E90744C3E91A44A3
:10C230005BF0F0F9FFF784FF002108460FF0C2FB26
:10C24000FCF776FCB0F1000B40F39D8106F1E40AA7
:10C250000024A14D53462746DA46A14605F5096854
:10C260009E4E9B46009404E009F50069CA4540F3E0
:10C27000AC809B4B1B68EB64FCF78CFC2022414696
:10C280004846FFF781FF12229649404665F0F6F9CD
:10C290000028E9D1B94525D00099934B01EB410223
:10C2A00003EB82034A1C914918460093A9EB07034C
:10C2B0000392029302F04EFD009B5946039A41F807
:10C2C0004C3B029BCBF80C700092CBE90433DBF8BB
:10C2D0001C30CBE908330123CBF80830844BCBF872
:10C2E00028308B46019B4F461222D3F8B032CBF850
:10C2F0001C30A918335D013291F8901899420BD087
:10C300000024202AF5D120374146BA45384653DB70
:10C31000FFF73AFF0022ECE70134152CF1D1D019D8
:10C3200074492022FFF730FF00230A2207A9714831
:10C33000CDF81C8002F05CFF0746079800230A2214
:10C34000013007A9079002F053FF059000230798DA
:10C350000A2207A90130079002F04AFF0490002347
:10C3600007980A2207A90130079002F041FF0390C5
:10C3700007A9079800230A220130079002F038FF2E
:10C380000023029007980A221946013002F030FF7C
:10C3900097B10399DDE9043243EA4212029B5B0143
:10C3A00043EAC123A7F2BC7143EA600342EA412297
:10C3B00043EA0243CBF81C30009B642B46D04F4627
:10C3C00009F50069CA453FF754AF5B46D3469A4624
:10C3D000009B642B1ED0B9451CD00C22424C434913
:10C3E000A9EB070502FB0344013320461A460093DC
:10C3F00002F0B0FCDAF81C20CAF80040CAF8145069
:10C40000CAE908220122CAF80820394ACAE9037594
:10C41000CAF82820009B002B03F1030118DC4FEA27
:10C420004B03B3F1805FC0F2AF80284B986830B9FE
:10C430001A461B791BB11368002B40F0DB800021EA
:10C44000084609B0BDE8F04F0FF0BCBAD3466721EB
:10C450004C261E4BDFF8A8904FF0010806FB01F4B4
:10C4600032460021244F1D19284665F017F8324640
:10C470000021284665F012F81D4E144A04F11003FD
:10C48000009942F804901834C5F8088004312F62EE
:10C49000AE6242F803B013440432C3F804B0019B07
:10C4A000D3F8B0321351144463606B62B7E74FF4B2
:10C4B0007A720023214640F26D1462F0B1F80F4BFE
:10C4C00040F2B272B0FBF3F31EE000BFA082002482
:10C4D000F0030024DC2B0B08B847002498C50B0898
:10C4E0006C35002474C50B086850002488C50B08FF
:10C4F000CDC10408485000240068214C805101003F
:10C50000B0C50B085B1A013212F0030514BF2146B7
:10C510004FF4B7718B42F5DA8449002D64D0019154
:10C520000199D1F880128B42C0F29C80804D012489
:10C530005B1A55F8041F01349942F9DD0133A2F268
:10C54000BC72019D43EA44133C2443EA4223794AE6
:10C55000B0FBF2F102FB11024FF46160B2FBF0F1AB
:10C5600000FB11221C20C5F88402B2FBF4F004FB8E
:10C570001022521042EA401242EAC12242EA034328
:10C58000C5F8B0323EE603214C266B4BDFF8B8917C
:10C59000012706FB01F4324600214FF002081D1965
:10C5A000284664F07BFF32460021284664F076FF7F
:10C5B000614B019A04F1100143F80490CBF1006340
:10C5C000D2F8B00204F11802BB405B4C5B4E85F818
:10C5D0000580AF602E62635021444B60231D98504C
:10C5E0001A445060686220E70C4601911D21C4F88E
:10C5F000841295E7504C0022002301460546A064B2
:10C60000E063C4E910232246D46C02F14C035CB30E
:10C610009C684E1E9D64B442C2E92355DD630DD073
:10C620004E1CB44210D113F8481C00293FF407AF48
:10C630001A6421461A4643F8083CE5E700293FF40E
:10C64000FEAE53F80C2C2146A1427FF4F8AE00292F
:10C650003FF4F5AE146CE66B0136E6631C6493643C
:10C660001A46D1E7012469E7334A0226254613E03A
:10C67000D36B16635B01C2E9045520D003F6FF7348
:10C6800001EB133319465363CB1A916352F84C7F75
:10C690004E1C1C440130C7B11379711E002BE7D129
:10C6A000136916637BB103F6FF7301EB133357690C
:10C6B000536337B107F6FF7701EB1731E4E73346F1
:10C6C000E0E73146E0E73346F1E71D4D01393E260C
:10C6D0003F27C5F89C008A0F1A488B00C5F8904088
:10C6E00068674020C5F88C10C5F88000C5E91E6752
:10C6F000C9B140F2FF101B1842F100025B0A43EA85
:10C70000C25303F140020C481344C5F8842003EBE4
:10C71000C101C5F888304A022967CB0DC5E925005B
:10C72000C5E91A238BE60123EBE700BFF0030024E1
:10C730007006002480510100A08200240068214C72
:10C74000B8470024CCC50B08C0C50B082DE9F04341
:10C750004D4D93B0FFF714FB05F10C0404E0FFF717
:10C76000A1FB6420FAF7C8FDAB68002BF7D095F861
:10C770008938002BF3D1EB6820465B689847074661
:10C780000028ECD02B7995F88C289A4201D0FFF73D
:10C79000BDFC0024D5F808802C60B8F1000F67D0EC
:10C7A0003A4E09E02B7995F88C289A4201D0FFF790
:10C7B000ADFC2034A0451AD922463146684602F025
:10C7C000C9FA684661F0B4FA012201466846FFF7EB
:10C7D00045FCA3B2002BE5D12B6D002BE2D09A884B
:10C7E0001B6859690A4218BF12049A61DAE7FFF719
:10C7F000CFFB2B7995F88C289A4201D0FFF786FC65
:10C800000023DFF888901F461C462B6022464946CD
:10C8100009A802F09FFA21220021684664F03EFE3A
:10C82000202269462046FFF7AFFC2022064609A9D0
:10C83000684664F023FFA3B2203458B9202E09D1F2
:10C840005BB1A045E2D8B7FA87F77F09384613B045
:10C85000BDE8F0830137002BF3D12B6D002BF0D016
:10C860001A689B8851690B4218BF1B049361E8E763
:10C87000FFF78EFB2B7995F88C289A4201D0FFF7B1
:10C8800045FC00232B60E1E7B8470024D4C50B0822
:10C890000A4B93F8B4221AB9094A92F8600D70470E
:10C8A0000849CA6D032AF7D10020054A4FF0010C50
:10C8B00083F8B40282F860CDC865EEE7F003002487
:10C8C000B84700240040005808B503220E4BDA6533
:10C8D00072B60E4B53E9021251EA020306D100234D
:10C8E0001A4609490A664B66F7F730F8084B4EF6C8
:10C8F000602C1B680CFB00F05B1842F10002C318AF
:10C9000042EBE072EDE700BF0040005828550024DC
:10C910006C350024024BD3F8A0301B6A184700BFC7
:10C92000B84700240A4AD2F8F83073B119689888D9
:10C9300092F8F5300A6910401BB1B0FA80F0400956
:10C940007047003818BF012070470120704700BFB2
:10C95000B8470024034BD3F8A00008B183691847F7
:10C96000704700BFB84700240378022B12D00E494D
:10C9700043680269D1F8F003023A184010B4400A43
:10C98000D1F8E843D1F8E41304FB02005DF8044B4E
:10C9900008447047044B4268D3E9F60100EB4100BC
:10C9A00000EB5220704700BFB84700242DE9F04F3C
:10C9B00083B002F00207874E019308B9002F4ED1D1
:10C9C000D6F8E043C4BB4FF0FF3E834C4FF0000C61
:10C9D000F146F246F046E36994F82A50984249D06D
:10C9E00015B3012D06EB0C1B0ED19BF8CF51EB07B5
:10C9F0000AD415F07E0F07D1ED0940F0A380656AD7
:10CA0000A84584BFA846E1460CF1010C1034BCF1E6
:10CA10000B0FE0D1BEF1000F80F2BB80BAF1000F26
:10CA2000C0F29D80D44628E0E6460CF1010C10349B
:10CA3000BCF10B0FCFD1EDE7D6E9F93505FB043496
:10CA4000A042C0D396F88C3313B9012386F88C33F7
:10CA5000012386F8A531002003B0BDE8F08F96F8D9
:10CA60008C33002B77D00123022086F8A53103B048
:10CA7000BDE8F08F002D40F08E80D6F870420CF1AA
:10CA8000020506EB0C18013406EB051EC6F87042D1
:10CA90000EF5D27ECEF80440C8E970040024CEF82A
:10CAA000084006EB051494F8AE41042CD7D80FF2D9
:10CAB000080E5EF824F000BFCDCA040803CB0408BA
:10CAC00057CA040803CB040805CB040812F001047C
:10CAD000D6F8BCE16DD106EB0510019B4FEAE20EE2
:10CAE00090F8AF81032B6EF3C71880F8AF815ED941
:10CAF0004FF6FF70834228BF034606EB0510A0F8EF
:10CB0000AC3197BB500707D506EB051090F8AF3155
:10CB100043F0010380F8AF31D3060AD506EB0515C3
:10CB200095F8AF31C3F34502013262F3460385F84D
:10CB3000AF31D6F8BC31012003EB4C230B6003B0BE
:10CB4000BDE8F08FE2460CF1010C1034BCF10B0F84
:10CB50007FF441AF5EE7012386F88C3383E7B9F1B8
:10CB6000000FFFF678AFCC4687E7D6F87402D6F808
:10CB7000703201300133C6F8740206EB0C10C6F8AF
:10CB80007032C0F8C43106EB0513042083F8AE01FF
:10CB9000B8E7F44671E7D6F870420CF102050134AB
:10CBA00006EB051EC6F87042CEF8A84179E7234689
:10CBB000A3E7D6F8A0300EEB4C21084A9C6800236E
:10CBC000A04700283FF447AF06EB0515022385F880
:10CBD000AE3140E7B84700245C490024018F0408C7
:10CBE00070B5114D82B00E4695F8A431022B16D1C6
:10CBF000020AC4B2D5F8D803002301A910440322C5
:10CC0000FFF7D4FE012808D195F8A431019A022B30
:10CC10000CBF22F8146042F8246002B070BDC0F36B
:10CC2000D41200F07F04E5E7B84700242DE9F04F67
:10CC3000444E0D4683B0174696F8A4112B6803297D
:10CC40003ED0022961D14FEA13294FF4807A5FFA6E
:10CC500083F8421E012A23D84FF0010B9F421AD9B4
:10CC600001288CBF00240124D6F850231AB1D6F82D
:10CC70006C1399424CD0D6F8D8030023092201A99D
:10CC80004844FFF793FE012823D0022814D020B196
:10CC90002B689F42E8D803202F6003B0BDE8F08FD7
:10CCA000B8F1000F13D096F88C3313B9012386F82E
:10CCB0008C33012386F8A531022003B0BDE8F08F44
:10CCC0004FF0800AC3F3D41903F07F08C1E7D346BD
:10CCD000C4E796F8A411022913D00329ECD1019BD3
:10CCE00053F8282022F07042B2FA82F22B685209DF
:10CCF000A2421FD0D8445B44D0452B601DD20229EC
:10CD0000EDD1019B33F81820EEE74FF4807AD9E794
:10CD1000D6F8E813013A02EB41224902B2FBF1F2E4
:10CD20001344B3FBFBF20BFB12320AB15B449B1AB8
:10CD30002B60AEE79F42B0D8ADE709F101094FF093
:10CD40000008A6E7B84700242DE9F04FDFF88491EA
:10CD50008B4685B0174699F8A4C10968BCF1020F4B
:10CD6000D9F8D85340F08280CEB24FF4807305EBEF
:10CD70001125A6EB010890449844B94208F1FF3808
:10CD8000B8FBF3F84AD200F00103A8446FF0404A20
:10CD90000193BCF1030F07EB0604A8EB050328463B
:10CDA00014BF4FF480728022641A03A9944228BFF2
:10CDB0001446944228BF002E14BF012200220A32DA
:10CDC000FFF7F4FD01282AD199F8A4C1DBF800E0AF
:10CDD000BCF1020F0EF1010324D0B44255D90398DF
:10CDE00006EB0A02011F00EB820201EB840142F80C
:10CDF000043F8A4203F10103F9D1DBF80030A11BA3
:10CE000019448F42CBF8001002D1019B002B48D16E
:10CE10008F4205F101054FF00006BAD8012005B098
:10CE2000BDE8F08FB44246D903986FF00042811EEE
:10CE3000324401EB440100EB420222F8023F9142EE
:10CE400003F10103F9D1A11B71448F42CBF800100B
:10CE5000DED1019B002BDBD086466FF000434FF6FE
:10CE6000FF72012023442EF81320D8E701F07F063B
:10CE7000C1F3D413BCF1030FA6EB01081D4414BF8A
:10CE80004FF480738023904476E7AEEB060E0EEBF2
:10CE900004018F42CBF80010BAD1019B002BB7D010
:10CEA00003986FF040434FF0FF32234440F82320B3
:10CEB000DBF80010ACE7AEEB060E0EEB04018F4280
:10CEC000CBF80010A4D1019B002BA1D0DDF80CE021
:10CED000C3E700BFB847002430B50446C06983B03B
:10CEE00010B9012003B030BD0D460023032201A973
:10CEF000FFF75CFD0128F5D1B4F92020002A19DBE9
:10CF0000019B012D4FEA421103EB421203D0022D87
:10CF10001BD1E5205854A368D3612378032B04D197
:10CF20000023137753779377D377636A190C53836E
:10CF30009182D6E7064A92F88C1309B982F88C03DD
:10CF40000123022082F8A531CCE7E368E4E700BFC3
:10CF5000B84700242DE9F041022382B004460E4672
:10CF600094F83C20042A7CD8DFE802F02E03704FAE
:10CF70003F00414D4FF6F777DFF8008118E0BC45E0
:10CF800062D855F0B5FC01284FF00001034638D1B6
:10CF9000206BFFF725FE0128034632D10199D5F811
:10CFA000EC034A1E2163824228BF0246C5F8EC23E7
:10CFB00095F8A40101A9226B03281FFA82FC1046F0
:10CFC000DDD14245DDD93FE07100204601F0FE0190
:10CFD000FFF782FF0128034643D1626B002A14BF8A
:10CFE0000222012284F83C20BAE794F82830042B6E
:10CFF00002D1002384F82830A36B0BB12046984758
:10D000000123184602B0BDE8F0811B4D0021E26A01
:10D01000D5F86C3305F55270C5F86C239B1AD5F81A
:10D02000E82302FB03F3D5F8502302EB4322C5F8B3
:10D030005023D5F8542302EB4322C5F85423FFF7BD
:10D040004BFF012803460CD10422CBE7626B04F1AD
:10D0500030010020FFF778FE0128034601D10322AA
:10D06000C0E7022BCDD194F82820042AC9D1002290
:10D0700084F82820C5E700BFB8470024F7FFFF0F5A
:10D0800038B5044694F83430052B60D8DFE803F057
:10D0900031251D130D0394F82830082B3FD02D4B5C
:10D0A0000122022083F88D2338BD94F82830082B04
:10D0B00030D0012038BD00212046FFF70DFF0128A8
:10D0C00045D1042084F83400DCE7D4E90B01FFF7F4
:10D0D00087FD01283BD10320F4E74FF0FF31206B9F
:10D0E000FFF77EFD012832D1E36A002BF3D0022046
:10D0F000E8E7184D04F130010120D5F8E0230232B1
:10D10000FFF794FD012813D00238C0B201281ED8C1
:10D110000520D7E70023012084F82830CAE7002340
:10D120000122022084F828300A4B83F88D23BBE7C4
:10D13000E368D5F8E813226B03EB4123C5F8EC2331
:10D14000C4E90332E36A002BBCD16262BAE7002073
:10D1500038BD00BFB8470024F8B50446022094F853
:10D160003830032B07D8DFE803F021180B02002129
:10D170002046FFF7B1FE431EDBB2012B40D9F8BDBC
:10D180000120626B04F13001FFF7DEFD01284FF052
:10D190000303F0D184F83830E1E700211D48FFF7A0
:10D1A0009BFE01284FF00203F4D0E4E71A4BE66837
:10D1B00093F8A421D3F8E813032AD3F86C5314BFCF
:10D1C0004FF480728022256102FB01F1AF1A2A44DC
:10D1D00006EB4126E660D3F85063C3F86C23A6EB58
:10D1E0004126C3F85063D3F85463A6EB4121C3F83A
:10D1F0005413E36A2563626353B965620123C9E787
:10D2000094F82830062BBAD1002384F82830F8BDD2
:10D210002763F3E7004B0024B84700244368C3F3B7
:10D2200008020A44B2F5007F2DE9F041054682B0BC
:10D230000C4605D223446B60012002B0BDE8F081AA
:10D2400090F91A10481C0AD0434A02EB011292F8D6
:10D25000CF1121F0010182F8CF11FF22AA7695F9B2
:10D260001B20511C0FD03C48FF2600EB021090F809
:10D27000CF21C2F34501013921EAE17161F3460290
:10D2800080F8CF21EE762A78022AD3D0324FD7F811
:10D29000E823B4EB422F4FEA42282CDCD7F8F063A6
:10D2A0001E407242A24226DCA2192869424513D3CD
:10D2B0002A7E12072BD5D7F86C23411C8A421CD337
:10D2C00000D100214344A4EB0808686108469B1B79
:10D2D00008EB060429616B600028ADD097F8A42103
:10D2E000032A33D080B24FF6F7729042A4D81A4680
:10D2F00014446C60A0E700209FE797F88C230ABBDA
:10D30000012387F88C3387F8A5316B68DAE701A928
:10D3100055F0EEFA0128EED16B68A4EB08042869F9
:10D320009844297868613444A8EB060301980229DF
:10D330001A466B602861CFD1D7F8F813B3EB412FB1
:10D34000D6D379E7012287F8A521BBE7034A9042AB
:10D350003FF672AFCBE700BFB8470024F7FFFF0FDF
:10D360002DE9F0474FF0010882B0044694F83830B8
:10D37000032B00F2A480DFE803F055170C02002015
:10D38000236C84F8280003B19847022002B0BDE85E
:10D39000F0870022236C84F828200BB120469847A0
:10D3A000012002B0BDE8F08723786768022B03D024
:10D3B000444BD3F8F0331F40C7F34F272046FFF705
:10D3C000D3FA404E3F1A0546BFB207EB050C0222C6
:10D3D00001A9002328461FFA8CF9FFF7E7FA012874
:10D3E0004FF400724FF00001D0D1019864F056F86C
:10D3F000E3694FF4007120460BB16368EBB1D6F8D6
:10D40000E833013B994547D20135FFF707FF002874
:10D41000DBD196F88C3313B9012386F88C3386F868
:10D42000A581D2E72046FFF72BFE012802D0022873
:10D4300045D1032084F8380098E7019B4FF0203253
:10D440004FF0100E4FF02E0C42F62E6AC3F801205A
:10D45000C3F80520A3F8092083F800C0D4F824C03D
:10D46000A3F820A083F80BE0C3F82220C3F82620FD
:10D4700083F82A20E26BA3F81AC02CFA0EFC5A8714
:10D4800022FA0EF2A3F814C083F82BE09A86D6F89D
:10D49000E833013B9945B7D3C3EBC3532046590248
:10D4A000FFF7BCFE28B996F88C3323B1012386F828
:10D4B000A5310220BEE7012386F88C33F6E7002071
:10D4C00064E700BFB8470024B1F904300F2B2DE901
:10D4D000F0410D4682B00446164634D02046FFF790
:10D4E00043FA94F91B80B8F1FF3F3DD05C4F07EB46
:10D4F0000813D3F8C031984212D097F88C33002B20
:10D5000070D0012387F8A5312378022B60D02269DF
:10D51000002A75D100230120336002B0BDE8F081FC
:10D52000D7F8BC1101EB4821002967D0AB88204611
:10D5300001331BB201EB4311AB803160FFF714FAEA
:10D5400028600120E9E74FF40071FFF767FE00282B
:10D5500044D04FF6FF732046AB80FFF705FA94F9ED
:10D560001B80B8F1FF3FC1D12378022B3ED0226946
:10D57000002ACFD03A4F97F8A431032B67D093B24B
:10D580004FF6F7718B4294BF00230123002BBFD1CC
:10D5900030B997F88C33002B4CD0012387F8A53194
:10D5A0000023112201A9FFF701FA012826D10199D0
:10D5B000D7F8BC31CB1A48BF03F2FF13B3F5B05F05
:10D5C0004FEA63222CD24FFA82F884F81B80ABE733
:10D5D000D7F8F8236368B3EB422F9BD2002002B048
:10D5E000BDE8F081012387F88C338AE71C4F63681C
:10D5F000D7F8F823B3EB422FCAD38BE7237884E71D
:10D6000097F8A431032B19D093B24FF6F7729342D7
:10D6100094BF00230123002B7FF47CAF0020DEE7C2
:10D6200097F88C3313B9012387F88C33012387F8DB
:10D63000A531CAE7012387F88C33AEE7094B9A423C
:10D6400094BF00230123002B7FF464AFE6E7054B72
:10D650009A4294BF00230123002B7FF459AF97E730
:10D66000B8470024F7FFFF0F2DE9F047044688B0C4
:10D6700094F83030042B11D8DFE803F04A135B0331
:10D680005400237E9A0640F1E2800023112205A96E
:10D69000E069FFF78BF9012800F0D98008B0BDE8F8
:10D6A000F087C64D01AE04F11C0705F564793246DA
:10D6B00039464846FFF708FF012800F0E1800228BC
:10D6C000ECD195F9AA335F1C0AD005EB0313FF21B7
:10D6D00093F8CF2185F8AA1322F0010283F8CF2115
:10D6E00095F9AB335E1C0FD005EB031393F8CF21F4
:10D6F000C2F34501013921EAE17161F34602FF21DC
:10D7000083F8CF2185F8AB13042384F83030AFE7DA
:10D71000AB485AF0CDF84FF6FF720123228484F80B
:10D720003030A5E70020E36A207008B0BDE8F0477C
:10D730001847A24D95F8B833002BAFD104F11C0760
:10D7400005F5647801AE324639464046FFF7BCFE27
:10D75000012840F0E780DDF80490B9F1000F00F0F7
:10D76000C08099F800300BB1E52BECD1D5F8BC3175
:10D77000B9EB030348BF03F2FF13B3F5B05F4FEA01
:10D78000632280F00E8112018E4B13449A7B042A8F
:10D790000CD0D5F870220132C5F870225A600422EC
:10D7A0009A73D5F874320133C5F8743295F9AA33F7
:10D7B000581C0AD005EB031393F8CF2122F0010285
:10D7C00083F8CF21FF2385F8AA3395F9AB33591C91
:10D7D0000FD005EB0313FF2193F8CF2185F8AB138E
:10D7E000C2F34501013921EAE17161F3460283F890
:10D7F000CF2120220021484663F050FED4F831208A
:10D80000D4F8353005A8C9F80020C9F8043094F8D8
:10D810003B30B4F8392089F80A30A9F80820637E33
:10D8200089F80B3001F01EFFBDF81430002B40F0DA
:10D83000FC8044F281720321A9F81020A9F80E306F
:10D84000A9F81820A9F8163084F8301010E72046FF
:10D850005AF02EF82369002B6BD0237E03F0F702D9
:10D8600013F00403227671D1122A00F08680002280
:10D87000E36A204684F8282008B0BDE8F04718473E
:10D88000DDF80480B8F1000F00F09E8098F80030B9
:10D89000002B00F0998098F80BA01AF0080F7FF485
:10D8A00006AF0B2204F13101404663F0E7FE002889
:10D8B0007FF4FDAE637E8AEA0303DF0640F1EB806E
:10D8C00095F9AA335E1C3FF40BAF05EB0313FF2160
:10D8D00093F8CF2185F8AA1360F3000283F8CF21D3
:10D8E000FEE695F890330922022B3FF40DAF95F830
:10D8F000B833002B7FF408AF85F8C833404685F86D
:10D90000C43385F8B823C5E9F333D5F8A433C5F893
:10D91000BC33D5F8EC33C5F8C033FFF721FD01283F
:10D920003FF411AF02287FF4B9AE042384F83030FD
:10D930009EE6237E1B079AD5204B93F87023002A7E
:10D940007FF4ACAE072283F8702390E70023A5682C
:10D950002046E66A294684F82830FFF75FFC002855
:10D9600040F0938094F82830002B7FF497AE022388
:10D97000C4E90B6584F8283090E6E06A0421626A05
:10D98000A063204684F83C3084F828106363636207
:10D99000C4E90B22C4E9023308B0BDE8F04759F0EE
:10D9A00087BF95F88C3313B9012385F88C33012395
:10D9B0006FF00F0285F8A531E6E600BFB8470024F6
:10D9C000484B00247849002495F9AA33591C0AD001
:10D9D00005EB0313FF2193F8CF2185F8AA1322F05A
:10D9E000010283F8CF2195F9AB335A1C0FD005EB18
:10D9F000031393F8CF21C2F34501013921EAE17104
:10DA000061F34602FF2183F8CF2185F8AB13237E13
:10DA1000DB067FF579AE3F4859F04AFF4FF6FF72BB
:10DA20000223228484F8303022E605A8B5F9705D1F
:10DA300001F032FD4FF47A72002360F0F1FD3C23D7
:10DA400092B205FB03014FF47A700023C1FB00235F
:10DA500002A801F05DFD9DF80A309DF80B209DF8AD
:10DA60000E1042EA4312BDF80830A3F2BC7342EA3A
:10DA700043229DF80D305B0192B243EA51039DF8B9
:10DA80000C1043EAC1239BB2D5E6002E3FF406AE4C
:10DA90002046334649E6B8F81420B8F81A3043EA6D
:10DAA0000243D5F8E82363625202D8F81C30B3FB76
:10DAB000F2F102FB1131A36009B113445B1AE36078
:10DAC00084F819A095F9AA33591C0AD005EB031361
:10DAD000FF2193F8CF2185F8AA1322F0010283F8E1
:10DAE000CF2195F9AB335A1C0FD005EB031393F8F4
:10DAF000CF21C2F34501013921EAE17161F3460208
:10DB0000FF2183F8CF2185F8AB13032384F830304D
:10DB1000AEE500BF484B002410B50378044690F8EA
:10DB200018C0023B012B02D91CF0060F5DD11CF07E
:10DB3000200F3CD194F91A20511C0AD0314BFF21FF
:10DB400003EB021393F8CF2122F0010283F8CF21D7
:10DB5000A17694F91B305A1C0FD02A4901EB03110E
:10DB600091F8CF31C3F34502013A22EAE27262F33F
:10DB70004603FF2281F8CF31E2761CF0080F0DD06A
:10DB8000204B93F87023072A05D093F88C23A2B377
:10DB9000012283F8A521002283F870230023E26A82
:10DBA000237084F82830FAB1BDE810401047164BB6
:10DBB0000022E069D9691033884206D001320B2A6D
:10DBC000B8D0D96910338842F8D10E4901EB02115F
:10DBD00091F8CF31C3F34502013A22EAE27262F3CF
:10DBE000460381F8CF31A5E710BD0121FFF774F995
:10DBF0000128F9D194F818C099E7012283F88C2301
:10DC0000C6E700BFB84700245C49002438B51A4C69
:10DC100094F8B8332BB970B190F828201AB118468F
:10DC200038BD002038BD0146442204F5647063F01D
:10DC3000D7FB012038BD04F564750146442228460F
:10DC400063F02CFC94F8A43103224FF6FF71022BF1
:10DC50002846A4F8AA1318BF1346D4F8F41384F87E
:10DC6000A823102284F89033C4F8B41384F8A923AD
:10DC700059F01EFEDDE700BFB8470024304A4FF0E0
:10DC8000FF3CF8B5A2F5D2700023644603E00133EF
:10DC900010320B2B14D092F82A100429F7D100EB84
:10DCA000031191F8CF11CE07F1D4651C116A01D090
:10DCB0008C45ECD91C4601338C4610320B2BEAD133
:10DCC000002C01DA0120F8BD1E4DA71C260105EB32
:10DCD0000713B3F8AC11D9B9AB19D5F8BC111A4A6E
:10DCE000D3F8C00101EB4421D5F8A0301C69002312
:10DCF000A047B0B1022809D1D5F8743205EB071757
:10DD00000122013B87F8AE21C5F874320020F8BD2E
:10DD100005EB0413D3F8C001D5F8A030DB689847B1
:10DD2000DAE7D5F8743205EB071703210122013B2E
:10DD300087F8AE1185F87822C5F87432E6E700BF9F
:10DD40005C490024B8470024658F04082DE9F041A0
:10DD500090F8283082B00446013B082B0BD8DFE84E
:10DD600003F0383C1F2305290A2E33000121FFF759
:10DD7000F1F8012802D002B0BDE8F081002223783A
:10DD8000216C84F82820002BF5D00322E162D4E92D
:10DD9000010384F82820834238BF03462046A3604D
:10DDA00002B0BDE8F041B7E6002102B0BDE8F041A5
:10DDB000FFF7D0B802B0BDE8F041FFF7CDB902B02F
:10DDC000BDE8F041FFF75CB902B0BDE8F041FFF7F4
:10DDD000C7BA02B0BDE8F04146E4DFF84C814268C2
:10DDE000D8F8F053036B1540D8F8E81390F800E02A
:10DDF000E8184E02B0EB412F41D34FF6F777BEF152
:10DE0000020F14D021690846002963D16068A36815
:10DE10000021E26A834284F8281038BF0346A360D9
:10DE2000002AA8D0204602B0BDE8F0411047D8F83B
:10DE3000F8136068B0EB412F34D22069217E0907C6
:10DE40003AD5D8F86C1300F1010C614530D298F83E
:10DE50008C1300294FD1012388F88C3388F8A53121
:10DE6000626894F800E0236B9B1B32442B44521BE6
:10DE700000259E4262602363C4E904C0BFD9BEF19D
:10DE8000020F0ED021690029C0D098F8A401032800
:10DE900043D089B24FF6F7708142B7D898186060C6
:10DEA000B5E76068D8F8F813B0EB412FF6D3AEE7CA
:10DEB000DAD14FF0000CD7E701A954F019FD012881
:10DEC0007FF459AF2069DDF804C094F800E062687F
:10DED000236BC9E798F8A4C1BCF1030F11D01FFA56
:10DEE00081FCBC4594BF4FF0000C4FF0010CBCF11D
:10DEF000000FC8D1A2E7012188F8A51194F800E02D
:10DF0000B2E7DFF820C0614594BF4FF0000C4FF03E
:10DF1000010CBCF1000FB6D190E7024881423FF6F8
:10DF200075AFBBE7F7FFFF0FB847002410B58C189B
:10DF3000A14215D001F1FF3E013C41F2210C1EF837
:10DF4000012F082380EA022002B24000002A8CEA56
:10DF5000420180B2B8BF88B2013BF5D17445EED121
:10DF600010BD00BF0823484041B240000029C0B2A4
:10DF7000B8BF5040013BF7D1704700BF30B50568CE
:10DF800004468D4218D901F1FF3E681E00231EF899
:10DF900001CF082183EA0C034FFA83FC5B00BCF13C
:10DFA000000FDBB2B8BF53400139F5D17045EED157
:10DFB0006A1C22602B7030BD00236A1C22602B700B
:10DFC00030BD00BF9FED067AF7EE007A60EE870A5B
:10DFD00060EE800A30EEA70A80EE800A704700BF2C
:10DFE000DB0FC94070EEA07ADFED263ADFED264A5E
:10DFF000F7EE006A9FED254A67EE807A9FED245A7E
:10E00000DFED245A9FED246AB8FE677A77EEC77A6F
:10E01000BDEEC77A17EE103A27EEA77ADA07E7EED9
:10E02000234AA7EE045AE7EE245AA7EE056A67EEE4
:10E03000A57AE7EE066A05D5B1EE677AF0EE667A64
:10E04000F0EE476A9B0703D5F1EE677AF1EE666A58
:10E0500087EEA67ADFED117A00230361C360F7EE45
:10E06000006AB0EE666A77EE277A80ED007AA7EE56
:10E07000276AC6EE867A27EE277AC0ED017A80ED10
:10E08000027A70474AD99E3DA04B25BF762FA7BC88
:10E0900000D8813E8E0FC93FCEE99DBFF304B53F46
:10E0A0002DE9F047002BDDF820A0884607460CBF7D
:10E0B0004FF020094FF030095646002A144616F852
:10E0C000011B23DD11B3334601E0002C05DD13F8FD
:10E0D000012B2546013C002AF7D1023D3CB14946BF
:10E0E0003846C047013DFAD29AF8001059B1384677
:10E0F000C047334616F8011B0029F8D1A4EB0A04E7
:10E100001819BDE8F0872046BDE8F087002C04F11F
:10E11000FF35E4DC00240029E9D1F4E703685A1C48
:10E1200002601970704700BF10B56FF000440246DE
:10E13000044404E0B3EB0E0015D1A24214D012F84F
:10E14000013BA3F14100192811F8010BA0F1410C8A
:10E1500098BF203300F1200EBCF1190FEAD91B1A29
:10E1600004D10028E9D110BD002010BD184610BD13
:10E17000884230B54FF001043AD301FB04F4B0FB00
:10E18000F4FC8C45F9D2BCB102BB06E0A14203F815
:10E19000015B11D81446B0FBF2FCBCF1090F0CF185
:10E1A00057050CF1300E04FB1C00B4FBF1F2EDDC62
:10E1B000A14203F801EBEDD900221A7030BDA14253
:10E1C00003F8015BF8D81446B0FBF2FCBCF1090F70
:10E1D0000CF137050CF1300E04FB1C00B4FBF1F21E
:10E1E000EDDCA14203F801EBEDD900221A7030BD3D
:10E1F0008446002AEAD1D0E7002870B503DA2D233F
:10E20000404201F8013B092886464FF0010307DD33
:10E2100003EB83035B00B0FBF3F2092AF8D89BB150
:10E220000F4CA4FB030CBEFBF3F2092A4FEADC0CF3
:10E2300002F1570602F1300503FB12EE07DD092B50
:10E2400001F8016B6346ECD800230B7070BD092BFD
:10E2500001F8015B6346E4D800230B7070BD00BF7A
:10E26000CDCCCCCC0378202B03D110F8013F202B50
:10E27000FBD0092BF9D02D2B00F0A9802B2B75D0CA
:10E28000B7EE000AA3F13002D1B2092977D8F2EE35
:10E29000046ADFED5F7A07EE102A10F8013FB8EE4E
:10E2A000C77AA3F13002D1B2A7EEA67A0929F0EE1F
:10E2B000477AF0D92E2B66D003F0DF03452B40F0D0
:10E2C000838010B442782D2A00F096802B2A00F02B
:10E2D0008380A2F130030130092B00F284800024F6
:10E2E000002303EB830302EB430310F8012FA2F199
:10E2F0003001303B0929F4D9B3F59A7F1A46B7EEBD
:10E30000007A28BF4FF49A72072B09D91346DFED24
:10E31000416A083B27EE267A072BFAD802F007025B
:10E32000DAB1F2EE046A012A27EE267A15D0022A23
:10E3300027EE267A11D0032A27EE267A0DD0042A5A
:10E3400027EE267A09D0052A27EE267A05D027EE71
:10E35000267A062A18BF27EE267A002C45D0C7EE6B
:10E36000877A5DF8044B20EE270A70474378B7EEB2
:10E37000000A0130A3F13002D1B2092987D92E2B2E
:10E38000DFED237A98D143780130A3F13002D1B286
:10E39000092991D8B2EE047AF0EE475A06EE902A97
:10E3A00010F8013FB8EEE66AA3F13002D1B2C6EE32
:10E3B000076A092927EE257A77EEA67AEED903F0C7
:10E3C000DF03452B3FF47DAF20EE270A70474378EB
:10E3D000BFEE000A013055E782780230A2F1300327
:10E3E000092B7FF67CAFB7EE007A67EE877A5DF88F
:10E3F000044B20EE270A704782780230A2F13003E6
:10E40000092B01D801246BE7B7EE007AA7E700BF1C
:10E410000000000020BCBE4C30B58588C38815F0D4
:10E42000050F9CB203D10C600389136030BD1BB291
:10E430000B60B0F90830F8E7F0B5868806F4E073B1
:10E44000802B03D185794FF0FF3406E0C02B4FF0CD
:10E450000105F8D1847905FA04F40023012006F0BF
:10E460000706AB4200D1F0BD052E0FD8DFE806F05D
:10E470000308101D242448B1C85CD75C78400FE025
:10E4800020B1C856D756C71B784278410133E8E718
:10E490000028FBD031F8130032F81370784080B2B6
:10E4A00020420CBF01200020F0E70028EED031F917
:10E4B000130032F91370E6E70028E7D051F8230083
:10E4C00052F82370DAE7838803F03803102B1CD04E
:10E4D00002D83BB980897047182BFBD0202B22D063
:10E4E00000207047174B808993F900305A1C0AD1DD
:10E4F000154B1B7803EB4302C3EBC20303EB83030F
:10E5000000EB43000BE0DBB2F4E70E4B808993F99C
:10E510000130591C05D10C4B5B7800EB431080B2E5
:10E520007047DBB2F9E7074B808993F902305A1C38
:10E5300006D1054B1B7C03EB830203EB4203DFE7B1
:10E54000DBB2F8E704080024D44C0024032870B59B
:10E5500019D80D4BC943C60003EBC00201F00101FD
:10E560001579527981EA0504A2420CD053F8302083
:10E570003AB14D1B106892886942694109018A408D
:10E58000826133445C7170BDCCA10024002370B55E
:10E59000934200DB70BDD0E90245A54208DB046967
:10E5A0004568AC4204DA661C05680661CE5C2E55EF
:10E5B000C46801330134C460EAE700BF092917D0F9
:10E5C000B1FA81F35B0999B1013903604A0001F0A6
:10E5D000030102F00802C1EB01119300C1EB01112C
:10E5E000A3EB92038900C3EB031381809B0043805C
:10E5F000704738B505460C4608465FF099FB214642
:10E6000002462846BDE83840C0E700BFB5EEC00A64
:10E61000DFED357A0023F1EE10FA30B5C8BF30EEE9
:10E62000270A87B0D8BF30EE670ADFED307A05469B
:10E6300003A9029320EE270ACDE90033FDEEC07A4C
:10E6400017EE904A84EAE470A0EBE47052F06CFE9E
:10E65000002C03A8B4BF2D2320238DF800305FF0D9
:10E6600067FB01282AD0022834D003281ED003A932
:10E67000684662F01BFF68465FF05AFB0446694635
:10E680002846033CE4B2224662F0AAFE0023284654
:10E690002B555FF04DFB2E22431C0DEB04012A5439
:10E6A000E81862F030FF284607B030BD302303A9D8
:10E6B00068468DF8013062F0F9FEDCE743F2300283
:10E6C000302303A96846ADF801208DF8033062F0CD
:10E6D000EDFED0E743F2300303A96846ADF8013000
:10E6E00062F0E4FEC7E700BF6F12033A00007A440D
:10E6F0000CF058BF38B5054660B159B14C1E14F83E
:10E70000011F284619B9BDE838400CF05FBF0CF076
:10E7100049FFF4E738BD38B5084B04461D6A5DB1C2
:10E7200028465FF005FB29460246204662F0A6FF18
:10E73000B0FA80F0400938BD0120FCE7CCA10024EC
:10E7400070B5054640894DF027F9064B044628462A
:10E7500093F82460FFF7B7FE16B1E368184470BD64
:10E76000A368FBE7CCA1002438B505460C46FFF7AB
:10E77000E7FFAA8802F0070302F4E072C02A29D159
:10E78000052B0CD8DFE803F0030B0F0B1B1BAA793A
:10E79000012393400278DBB214B11343037038BDF8
:10E7A00022EA0303FAE7AA790123934002889BB285
:10E7B00014B113430380F2E722EA0303FAE7AB79CB
:10E7C00001229A40036814B113430360E7E723EA88
:10E7D0000203FAE7052BE2D8DFE803F0030305059F
:10E7E00007070470DBE70480D9E70460D7E708B5C2
:10E7F000034640B1202162F068FE034618B11A7842
:10E800000130202AF9D0184608BD08B5CB0701D43D
:10E81000F5F79CF808BD2DE9F3410023124D04469D
:10E8200000EB8106114F05F8253FB44203D1104893
:10E8300002B0BDE8F081394628464FF0000862F08A
:10E8400035FE2146684662F05EFE2021684662F091
:10E850003CFE28B969462846043462F027FEE4E706
:10E8600080F80080F1E700BFCCA10024D4500C0850
:10E87000F1A1002410B58EB00C46694618F0A0FB3B
:10E88000089824B1431D0A22B3FBF2F3236060B160
:10E8900007EE900A9FED060AF8EE677A80EE270AE7
:10E8A0000EB0BDE8104061F0ADBA0EB010BD00BFB3
:10E8B0008096184B70EEA00A9FED284A9FED285ACB
:10E8C000F7EE007ADFED274A60EE800ADFED265A88
:10E8D0009FED266ADFED266AB8FE607A70EEC70A01
:10E8E000BDEEC77A17EE103A20EEA07ADA07A7EE4F
:10E8F000045AE7EE245AA7EE056AE7EE256A60EEB1
:10E90000860AE7EE267A05D5B1EE607AF0EE670A60
:10E91000F0EE477A9B0703D5F1EE600AF1EE677AD5
:10E92000F7EE006A002380EEA77AC3600361C6EEAB
:10E93000817AB0EE666A21EE071A80ED021A77EE50
:10E94000275A67EE277AA7EE256A86EE867A67EE63
:10E95000877A80ED007AC0ED017A70474AD99E3DF2
:10E96000A04B25BF762FA7BC00D8813E8E0FC93F94
:10E97000CEE99DBFDFED197A20EE270AF8FE407A36
:10E98000BDEEE77A30EE670A17EE103A60EE007AD5
:10E9900003F00202DB070DD59FED116ADFED116A6E
:10E9A0009FED117AE7EE866AA7EEA67A20EE070AB7
:10E9B00082B170479FED0D6AB7EE000ADFED0C6A79
:10E9C0009FED0C7AE7EE866AA7EEA67AA7EE870A95
:10E9D000002AEED0B1EE400A704700BF83F9223F13
:10E9E0004AD99E3DA04B25BF8E0FC93F762FA7BCAD
:10E9F00000D8813ECEE99DBFB0EEC07AF0EEE06A6D
:10EA0000F0EE407AC6FE875AF5EE405AF1EE10FA63
:10EA10003BD086FEC75A85EE256A9FED1D2A9FEDE5
:10EA20001D3A9FED1D4ADFED1D4ADFED1D2AF7EE71
:10EA3000005ADFED1C3A9FED1C5AA6EE423AE6EE74
:10EA4000223AA6EE034AE6EE235AE6EE044AA6EE82
:10EA5000245A85EE250AF4EEC76AF1EE10FA03D5C2
:10EA60009FED127A37EE400AF5EEC00AF1EE10FA89
:10EA700003D59FED0F7A37EE400AF5EEC07AF1EE3E
:10EA800010FA48BFB1EE400A70479FED070AE2E76F
:10EA900039094E3DE3B59E3E88FA163E45FE7F3F5E
:10EAA00099FB243F69A2163EA7DFA834DB0FC93FBC
:10EAB000DB0F49402DE9F04F884689B01E4611789A
:10EAC000531C0393002900F01681002514460746C5
:10EAD000A94609E038460135C047039C621C2178ED
:10EAE0000392002900F08F802529F3D16078A31CC0
:10EAF0003028CDE9033923D0A0F130034FF0000ACC
:10EB0000DBB2092B26D96C282AD078287FD8572841
:10EB100078D9A0F15803202B79D8DFE803F0BD782D
:10EB200078787878787878787882AF787878787824
:10EB300078787878AA787878789E788A7878BD001E
:10EB4000E31CA0784FF0010A0393A0F13003DBB27D
:10EB5000092BD8D804AA03A953F0E2FF6C28D4D11A
:10EB6000039B1A785C1C782A0394B7D8572A40F282
:10EB70008E80A2F15803202BB0D801A151F823F0C8
:10EB8000B7EC0408DDEA0408DDEA0408DDEA04085D
:10EB9000DDEA0408DDEA0408DDEA0408DDEA040829
:10EBA000DDEA0408DDEA0408DDEA040825EC0408CF
:10EBB000D3EC0408DDEA0408DDEA0408DDEA040811
:10EBC000DDEA0408DDEA0408DDEA0408DDEA0408F9
:10EBD000DDEA0408DDEA040875EC0408DDEA04084F
:10EBE000DDEA0408DDEA0408DDEA04085DEC040857
:10EBF000DDEA0408E3EC0408DDEA0408DDEA0408C1
:10EC0000B7EC040828B9284609B0BDE8F08F039C8A
:10EC100064E72528FBD1039C252138460135C047F0
:10EC20005CE7039C56F8041B38460135C9B2C0475F
:10EC300054E70DF1140B00220A2156F8040B5B4631
:10EC4000039CFFF795FA5346049A41463846CDF89F
:10EC500000B0FFF725FA054440E7039C56F8040B83
:10EC60000023049A414600903846FFF719FA0544FC
:10EC700034E7039C56F8043B1D602FE70DF1140B9D
:10EC800056F8040B039C5946FFF7B6FADBE7002A57
:10EC9000B9D0252AC0D021E7A0F158020DF1140BFC
:10ECA000102156F8040BB2FA82F25B465209FFF7C4
:10ECB0005FFA039CC7E7A2F158020DF1140B102173
:10ECC00056F8040BB2FA82F25B465209FFF750FA8B
:10ECD000B9E70DF1140B56F8040B5946FFF78CFAFF
:10ECE000B1E70DF1140B00220A2156F8040B5B4624
:10ECF000FFF73EFAA7E70D4685E7F8B5104C074643
:10ED00000D461646A06CA0B10E49FFF7F3FC39463C
:10ED1000A06CFFF7EFFC0C49A06CFFF7EBFC0B4974
:10ED200033462A46A06CFFF7C5FE0949A06CFFF7E1
:10ED3000E1FC94F84C3013B1012384F84D30F8BD58
:10ED4000CCA10024133D0C0840580C08F1E604083F
:10ED5000203D0C080EB400B584B0084905AB019005
:10ED600001A853F8042B0393FFF7A4FE0022019B94
:10ED70001A7004B05DF804EB03B070471DE104089D
:10ED80002DE9F04F914692881D4685B002F4E0735C
:10ED900007468846802B4CD10026344636E0B9F829
:10EDA000043003F00703013B042B04D8DFE803F031
:10EDB00006080B0E3E00AA5D5D490AE0AA57FBE774
:10EDC00035F81620F8E735F91620F5E755F826202E
:10EDD000584908F1FF3B6846FFF7BCFF8246A34550
:10EDE00008DDABEB040269468242A8BF024638192F
:10EDF00062F0F6FA99F806205444013AB24204DD72
:10EE0000A34501DD2C233B550134013699F806302A
:10EE1000B342C4DC08F1FF33A342A8BF2346002B52
:10EE200036DB984534DD0022FA5431E055F82620CF
:10EE3000C2E702F00702052A49D8DFE802F003180A
:10EE40002D2F3246402B2A784DD049D9C02B64D083
:10EE5000B3F5807F41D1284699F8071062F033FC62
:10EE6000354B002812BF044601241D464DE095F99C
:10EE70000020C02B51D0EBD893B3402B2DD1002ACA
:10EE800031DAB8F1000F01DD00233B704FF0FF34A1
:10EE9000204605B0BDE8F08F2A88EAE7B5F90020E2
:10EEA000E7E72968402B0A46E9D0CFD821496846D0
:10EEB000FFF750FF08F1FF32044669468242A8BFBF
:10EEC0000246384662F08CFAA4E72A68D1E7C02BE4
:10EED00022D0BDD81BB1402B04D000249AE71A469B
:10EEE0001349E4E7002299F80610144B03EBC10024
:10EEF00000799042C5DD53F8313053F82250002D8F
:10EF0000BFD028465EF014FF044608F1FF322946C0
:10EF1000A242A8BF2246D4E7002299F80630084D45
:10EF2000DA40084B12F0010F18BF1D46E9E700BF99
:10EF30004F660C081F410C086D5F0C0814430B084A
:10EF40005C660C0887410C08F7B5114E0746002394
:10EF50000C46304615460F494E3600F84E3F04EB3E
:10EF600045050D4B002F18BF19460C4F62F09EFA55
:10EF7000AC4202D10A4803B0F0BD394634F8022B46
:10EF80006846FFF7E7FE6946304662F08FFAEFE722
:10EF9000CCA100242D3D0C08243D0C08363D0C0866
:10EFA0001AA20024F7B500230B4E044600EB4105DE
:10EFB0000A4F06F87F3FAC4202D1094803B0F0BDCA
:10EFC000394634F8022B6846FFF7C4FE69463046DE
:10EFD00062F06CFAEFE700BFCCA100244E660C088B
:10EFE0004BA20024F8B54E1E054601F11F04054F43
:10EFF00016F8012F284639460235FFF7ABFEA64228
:10F00000F6D1F8BD3B3D0C0803685A1C026019702C
:10F01000090A03685A1C026019707047D0E900326F
:10F02000934201D3002070475A1C02601878704741
:10F0300010B50446FFF7F2FF01462046FFF7EEFF4A
:10F0400041EA002080B210BD70B50446FFF7E6FF2C
:10F0500005462046FFF7E2FF06462046FFF7DEFFA3
:10F06000014620460904FFF7D9FF41EA062129435A
:10F0700041EA006070BD00BF70B50B4616460546FC
:10F08000D0E900141846641A24EAE4749442A8BF34
:10F090001446224662F0A4F9A64203DC2B682344FE
:10F0A0002B6070BD321B0021204462F0F7F92B6801
:10F0B00023442B6070BD00BFA0F13003092B07D99A
:10F0C00020F02000413819288CBF00200120704713
:10F0D00001207047303809288CBF0020012070477C
:10F0E000413819288CBF0020012070476138192849
:10F0F0008CBF00200120704720280BD0092809D0A0
:10F100000A2807D00D2805D00B3801288CBF002015
:10F110000120704701207047A0F14103192B98BFCF
:10F1200020307047A0F16103192B98BF2038704739
:10F1300002B3844610B5841803E0981A15D1A4458B
:10F1400014D01CF8013BA3F14100192811F8010B60
:10F15000A0F1410E98BF203300F12002BEF1190F3B
:10F16000EBD91B1A04D10028E9D110BD002010BD35
:10F17000184610BD104670472DE9F84306460D4667
:10F180000024DFF838804FF00E0909FB04F32A460B
:10F19000304658F803703946FFF7CAFF38B9384689
:10F1A0005EF0C6FDA84202D1A0B2BDE8F8830134EA
:10F1B000B4F5257FE9D12046F7E700BF98530B0847
:10F1C00070B5044608460D465EF0B2FD064602E004
:10F1D00014F8013F43B1324629462046FFF7A8FF05
:10F1E0000028F5D1204670BD1C46204670BD00BFEA
:10F1F0002DE9F043064686469EF800C074460EF19F
:10F20000010EBCF1200FF7D0BCF1090FF4D0BCF116
:10F210000A0FACF10B00EFD0ACF10D05B5FA85F596
:10F220006D09002DE8D10128E6D9BCF12B0F3DD0A6
:10F23000BCF12D0F39D0102A3ED04FF0FF3E904642
:10F24000BEFBF2FE02FB0EF7FF43FFB2002014F8F4
:10F2500001CBBCF1390F4CF02009ACF1300C0DD8CA
:10F260005FFA8CFC944510DA7045264602D819D115
:10F27000674517D21D404FF0FF30E8E7A9F1570C62
:10F28000B9F1600F5FFA8CFCECD801B10E6003F0AD
:10F290000103D5B9002803DA002B18BF6FF0004036
:10F2A000BDE8F08300FB08C0D1E70125102A94F8DF
:10F2B00001C004F10104C0D1BCF1300F10D06FF0D7
:10F2C000704E0F274FF01008C0E7B0F1004F04D97F
:10F2D0001BB14FF00040BDE8F0834042BDE8F08331
:10F2E00060786FF0704E0F274FF01008A0F14106C4
:10F2F000192E04F1010698BF203078280CBF023483
:10F300003446A3E72DE9F0470E46B4B015468146D2
:10F31000002862D00378002B5FD08F79322F5CD821
:10F3200004464FF000084FF0150A2378ABB323468C
:10F330001C4613F8012B202AFAD072B32C2A4CD089
:10F3400047454ADDB38803F007032AFA03F3DB07D6
:10F350001CD52D2A41D000230A2201A92046FFF7FF
:10F3600047FF019BA34238D002AB0199002243F82A
:10F3700028000B780C460131202B09D002B10194F2
:10F380002C2B07D108F101080134CEE70123E3E774
:10F390000122EEE70BBB08F1010847451DD14C45A2
:10F3A00003D914F8013C2C2B17D002A800210446E5
:10F3B0008F4204DC00239F421ADC01200EE0B28859
:10F3C00054F8043B02F00702032A0FD8DFE802F0EA
:10F3D00003020B098033FF2B08D9002034B0BDE8AD
:10F3E000F08703F50043B3F5803FF6D20131DFE744
:10F3F000B28802F00702052A06D8DFE802F003030C
:10F4000008080C0C0268EA5401330430D3E70268A0
:10F4100025F81320F8E7026845F82320F4E700BF39
:10F4200001230A220021E3E670B50D461446FFF7DA
:10F43000DEF90646A0B1FFF7F3FF40F634031922C8
:10F440009842A8BF1846B0F5617FB8BF4FF461700D
:10F45000A0F56173B3FBF2F32B70237801332370B3
:10F460003046FFF7C4F90646A0B1FFF7D9FF40F6D2
:10F47000340319229842A8BF1846B0F5617FB8BF7F
:10F480004FF46170A0F56173B3FBF2F36B702378F6
:10F4900001332370304670BD038800211A4A30B50D
:10F4A00003F0030E90F802C0184CA3F5FA630EEBBC
:10F4B0004E0E0CF1FF3C40F2B5550CEB8E0C04EBFC
:10F4C0004C044FEA930CB4F8F831847905FB0C3303
:10F4D00090F803C022444FF47A740CF1FF3C63446B
:10F4E00090F804C003EB43030CEBC30C4379008991
:10F4F000CCEB0C1C03EB8C03C3EB031302EB83027A
:10F50000C2FB040130BD00BF80436D3814430B08BB
:10F51000F8B516461F46404D0446394630464FF46E
:10F520007A7200235FF07CF83C4B05443C4F3D4E23
:10F5300083FB0510E9172844C1EB601183FB01032D
:10F54000C8170B44C0EB631087FB003CC317C3EB29
:10F55000AC0386FB03764FEAE37ECEEBE61EC1EBFF
:10F560000116A5EB860CC0EB00154FEA8E0684F859
:10F5700006C0A1EB8501617103EB4301A0EBC10063
:10F5800040F2B55101FB1E332071B3F5896F37DAB4
:10F5900040F2DA218B4239DCB3F5B77F2249B4BFA0
:10F5A0004FF0000E4FF0010E0EEB4E0075464FEA85
:10F5B0004E0701EBC001B1F80E021C4907EB0E0C1F
:10F5C00001EBCC0C0B210CF1160C01E03CF8020D08
:10F5D000984212DD0139F9D17744134901EBC70193
:10F5E000B1F8F801012106F5FA6E0133A1707544F6
:10F5F0001B1A22812580E370F8BD0131C9B2F2E700
:10F60000032540F296500627AE46D6E7022540F283
:10F6100029400427AE46D0E780BC92C789888888F5
:10F62000ABAAAA2A73B06D1614430B080C450B083D
:10F6300070B5054608461446FFF72EFF4FF47A7260
:10F6400000235EF0EDFF3C23014692B2284604FB06
:10F6500003114FF47A740023C1FB0423BDE870400A
:10F6600056E700BF0D4B10B5D3E9004354EA03023F
:10F670000AD10146002340F2011218460B80C1F85E
:10F6800002208B710B8110BD054A1268121943F1DB
:10F690000003FFF73DFF012010BD00BF20550024EF
:10F6A0006C3500242DE9F041044615460846944285
:10F6B000B4FBF2F607D205FB1644134B1B5D00F8B2
:10F6C000013BBDE8F0819642B6FBF2F70CD20E4B3F
:10F6D00005FB176705FB1644DA5D1B5D00F8012B7F
:10F6E00000F8013BBDE8F081BA42B7FBF2F807D958
:10F6F00005FB1878044B13F8082000F8012BE7E706
:10F700004046FFF7CFFFF3E748C60B086B4B9A88DC
:10F71000B2F57A7F10B582B002D94FF47A729A802E
:10F72000DA88B2F57A7F02D94FF47A72DA80B3F8C8
:10F7300008C0BCF57A7F03D94FF47A7294461A81D7
:10F740005889B0F57A7F02D9002210465A819A89E9
:10F75000B2F57A7F0BD94FF47A72D98991429A81A6
:10F760000BD900228445DA810DD81A810BE0D989A2
:10F77000B1F57A7F01D90021D98184455FD99142C1
:10F7800001D300229A81598B9A8B914201D9002290
:10F790005A834B4B1B88F3B14A4CA278062A51D9A5
:10F7A0002179002940F083809FED477A474A07EE90
:10F7B000903AA3791178F8EEE77A06EE901AB8EE4F
:10F7C000E66AC6EE276A0BB137EE077AB4EEE67A40
:10F7D000F1EE10FA4EDC3E4B597803292BD83D4A06
:10F7E00002EB411293F800C03B49BCF1030FC1F892
:10F7F00004251BD801F59470E6220CFB02001A7C4C
:10F80000364C022A20600AD802EB8200344B02EB0D
:10F81000400203EB4202C1F8082502B010BD0020EF
:10F820002F4A1874C1F8082502B010BD002201F556
:10F8300094701A70E3E70021264A5970D2E700203D
:10F8400018819CE72749207901EB820191ED967A96
:10F850000028ABD0042ABED8002ABCD0B7EE000ADC
:10F8600080EE070A60F0CEFA2388834228BF034661
:10F870002380B0E767EE877ABCEEE77A8DED017AF8
:10F880009DF8043007EE103AB8EEC77AF4EEC77A66
:10F89000F1EE10FA01DD0133DBB26BB1102BA8BF22
:10F8A0001023DBB28B4238BF0B46137093E7082A54
:10F8B00091D99FED057AD1E70123F2E71058002492
:10F8C0000C220020783400246F1203385057002493
:10F8D000D44C002474A20024CCA100245857002446
:10F8E0008CA6002414430B082DE9F04FA54B83B0E0
:10F8F0001B7800AFA3F11702022A00F2CC82A24EBD
:10F90000A24C4FF0000A04F5A86994F8143504F5E8
:10F91000B768CB467B60B14619E09BF90420142AF6
:10F920002FD0284662F0C8F8AA031ED5012828D097
:10F93000082826DC16B1964B1D4204D1796828466A
:10F940005BF05EFBE8B10BF10C0BD84513D0DBF894
:10F95000005015F00106E0D028460AF1010A62F0D5
:10F96000ABF8AA035FFA8AFAE0D40128E0DC0BF1D5
:10F970000C0BD845EBD10AF1FF324E46022A05D9CD
:10F9800000E04E46834984484CF01CF800230220D6
:10F9900084F8BC3512F0A2FB94F8C0357F4A023BD4
:10F9A0001568022B00F21D8358B190F904904FF0B6
:10F9B000FF0A01E080F808A0484612F07FFB00280B
:10F9C000F8D1DFF8F091764B4FF47A7A94F813C6B9
:10F9D0004FF0000E03F5667B4FF06408C7F804C0D3
:10F9E00033F8082CB2F57A7FB3F8462088BF23F8A5
:10F9F00008ACB2F57A7F33F8062C88BFA3F846A08E
:10FA0000B2F57A7F33F8042C88BF23F806ACB2F540
:10FA10007A7F02D9002223F804EC33F8061C9142C5
:10FA2000B3F85610B3F8582098BF23F806EC91426B
:10FA300093F8672003F1610102F1FF3288BFA3F858
:10FA400056E0632A93F8682002F1010288BF83F828
:10FA50006780D2B2092A4FF0000288BF83F868E0BD
:10FA600013F83200013211F801CF844538BF81F814
:10FA700000E0032AF4D17A68E633012A18BF03F8BC
:10FA800065EC5B45ACD1DFF830A19AF80230042B6D
:10FA900000F0E3822BB9BAF80030B3F5F07F00F242
:10FAA0000F82FFF733FE3F4894F82016FEF786FDDD
:10FAB000103094F83F16FEF781FD103094F84F1681
:10FAC000FEF77CFDB4F85E26B4F85C361343B4F858
:10FAD000602613431BB213B10123A4F86236324BE4
:10FAE0002B40002B00F0E782EB0700F198826804BE
:10FAF00000F12082290740F15D822C4A274B1540F6
:10FB00001D60D9F800301340C9F800302B0440F1D3
:10FB10003582002384F81B3584F82B35E80440F146
:10FB2000388294F86F36012B02D9012384F86F369E
:10FB3000DFF87C80434608F1780B02E006339B45F2
:10FB40000CD01A780A2AF9D19978DA78914202D33E
:10FB50005A79002AF2D00A2021F07AFE00234FF4CD
:10FB6000806084F8BC3512F0B9FA002800F08A826F
:10FB70000F490D467960687960B3297839B34346F7
:10FB80001FE000BFB055002414430B08CCA1002493
:10FB9000BC0202000CA7002454B80C08745C0024BA
:10FBA000FEA20024FCA7002409600002FC9FFFFDC8
:10FBB00040A80024345500247834002406339B45A3
:10FBC00008D01A788242F9D15A79002AF6D008462C
:10FBD00021F03EFE0635AB45CDD19AF8028079681A
:10FBE000B8F1080F00F00D8294F81336D9F8000030
:10FBF000A3F10103C0F3C032B3FA83F384F8EF2614
:10FC00005B0984F8EC3694F81436A3F10103B3FAD7
:10FC100083F35B0984F8F236B14B5A78032A01D991
:10FC200000225A70AF4DB04A2B6813400240AF48D3
:10FC30002B60807BC9F80020002800F00482AC4DC6
:10FC4000AB88002B40F0F581AA4A1368B3F5000F8A
:10FC500001D3002313609368A748184010B140F205
:10FC6000022393601379013B042B01D90123137103
:10FC7000A8F10508A14BB8F1030F93F8009040F2EA
:10FC80007481B9F1000F28D00025DFF89C827D60D7
:10FC90003E6045464E46894606E0A8F10608A8EBB8
:10FCA0000A039E4240F24881A84615F8010F002839
:10FCB000F3D00CF059FA0028EFD083799B07ECD5EC
:10FCC0007D6849463E6801223DB19AF8113053B92A
:10FCD0009AF80530012B00D02AB19AF8063013B1FA
:10FCE00000238AF80630864BDA8802F00F000428D9
:10FCF00003D8C2F30312022A02D94FF42062DA8039
:10FD00001A8902F00F00042803D8C2F30312022A52
:10FD100002D940F601221A8194F8050794F81127B8
:10FD200094F80437904205D9002284F8052753B18E
:10FD3000A4F8082794F810279A4204D2002384F8E4
:10FD40000437A4F8083794F8062794F8FA379A424B
:10FD500002D9002384F80637DFF8D0C10CF1800AFD
:10FD6000634613F8032D02EB4202324492F84C939F
:10FD700092F84D8392F84EE313F8015F98794D4560
:10FD8000DA78A8BF4D464045A8BF404672451D7071
:10FD9000A8BF72469C459871DA70EDD10CF1200C29
:10FDA000E245DDD1D4F83825002A00F03A8100255B
:10FDB000012002E006318B450ED00B782C2BF9D1B7
:10FDC0004B78043300FA03F31342F3D0063122EAEE
:10FDD000030201258B45F0D10DB1C4F83825494EF9
:10FDE0006D4606F10808334602E0434500F0A9805D
:10FDF00013F8012F072AF8D988B02022FF2168467E
:10FE000061F04CFB002306F8013F0133082BFAD1C7
:10FE10003D4B4FF00008DFF818C1AD463B4E03F1F3
:10FE200042054FF00A0E59881A88914205D29888E7
:10FE3000824202D3814240F2C280C3F800C05E60B9
:10FE40009A7A1633182A13F80B2C88BF03F80C8CF7
:10FE5000642A88BF03F80BECAB42E4D12C4BFF22A1
:10FE60002C4D03F1780084F82C2813F9082C142A5F
:10FE700005D053F80C1C35EA010100F0EB800C337F
:10FE80009842F2D1244B5A79022A00F0A0800C3714
:10FE9000BD46BDE8F08F214A12F83310A9B9DB0046
:10FEA0001A441F4E5278002A3FF42AAD334493F887
:10FEB0007432002B7FF424AD18231A4A13701FE507
:10FEC0004FF4F073AAF80030EBE502EBC301DB005E
:10FED00049680029E4D1172112480170E0E700BF0A
:10FEE00010580024745C0024BDD77718D44C00242B
:10FEF0004456002460570024FDFDFFFF501C0020E5
:10FF0000405B00248A3400248CA600245E019A0100
:10FF100018A7002401000200004D002404300B0843
:10FF200014430B08B05500247F34002479A2002428
:10FF3000AE014A01644AE1E57D6849463E68002217
:10FF4000C2E688B02022FF21E946484661F0A6FAC1
:10FF50005E4A12F8013F59F8231001317FF452AF85
:10FF6000424549F82330F4D152E700238AF804309F
:10FF7000B9F1000F00F09D80012586E694F81B354D
:10FF8000002B00F090800023E80484F82B353FF527
:10FF9000C8AD29067FF5C5AD4D4B1A78182A04D88F
:10FFA0004C4BD340DA073FF5BCADDFF8408108F198
:10FFB000780BD3E5AA047FF5A9AD474A9EE5D98819
:10FFC00088423FF63AAF8A42FFF437AF38E7434AF8
:10FFD0001279002A7FF45BAF0C375A71BD46BDE839
:10FFE000F08F00287FF4EDAC3D4B25F08005DFF865
:10FFF00000911D60D9F8003023F08003C9F800306B
:020000040805ED
:10000000E1E49AF80630002B3FF4EEAD9AF8113097
:10001000012B7FF4E9AD02238AF81130E4E5314A7F
:100020006CE52C20796021F013FCD4F83825796830
:10003000BDE6287879600CF097F8796800287FF49D
:1000400003AEA88000E62848034302432B60C9F8AA
:100050000020F4E584F82C2814E7214B25F4805582
:100060001D60D9F8003023F48053C9F80030BAF885
:100070002030B3F57A7FBFF414AD4FF47A73AAF849
:1000800020300EE59AF802300A2B3FF471AD144A85
:10009000136823F000631360D9F8003023F0006385
:1000A000C9F8003064E542F201031D427FF46BAFF2
:1000B00034E54A4609E6D9F8003045F0080543F032
:1000C0000803C9F8003018E5F4DFFFFD8A34002486
:1000D000B055002400410001F4BFFFFD084D00248D
:1000E000745C0024F59FFFFD0004050040A8002477
:1000F000345500242DE9F04FDFF8989283B099F839
:100100003038013B012B40F205818D4F8D4BFA6851
:10011000DFF8848202F2DC524345FA6080F00C8101
:100120009B46894B0122894D9E1C0192864B598822
:10013000002900F0D780052906EB010240F2D280A9
:10014000AA4280F0CF80BBF800003446C0F30B0019
:100150000BE0138814461A44002B00F0C380AA4217
:1001600080F0C080052B40F2BD8063888342F0D1CF
:1001700063799B07EDD123885846DBF8081094F883
:1001800004A000934BF01EFCBBF80010BAEB113F2B
:1001900000F0AE8000230193BBF804100BF11C0BA0
:1001A0005BF8140CC1F30B015BF8044C52F05AFDE0
:1001B000C3452060BAD3664A664B1268664E1A6021
:1001C000FFF792FB654BE6223178654C01FB02326A
:1001D00071782260A3F1800203F5667302EB41128D
:1001E000C9F80425327C022A00F28C8002EB8201DD
:1001F00002EB410203EB4203C9F808351DF0BCFADB
:10020000584B9FED596A5B68DFED586A07EE903AEC
:10021000574A584DF8EE677A2468204686EE277ACA
:1002200067EEA67AC2ED007A82ED017A4FF0FF32D6
:100230006A60514A1360514A136028F00BFD204652
:1002400027F0CEFF21F04AFB4D4B03F1780102E08D
:100250000633994259D01A78002AF9D19C78D87877
:10026000844202D358790028F2D099F86C362A7269
:1002700003EB8303B9F8702603EB83039B00642B25
:10028000B8BF64237B60642303FB02F20023642A6B
:100290007B61BB84B8BF642287F82630C7E903338B
:1002A000BA603A62374AC7E90633374B93622EF099
:1002B0002FFC99F87618B9F8740823F059FA3FF032
:1002C000F7F916F0E1FB99F83038013B012B2BD9F7
:1002D0002E4B012201981B6887F82520FB6003B094
:1002E000BDE8F08FDBF8081058464BF06BFB51E788
:1002F000009BA11D58469A1F4BF09AFB00287FF4E3
:100300004BAF47E70022327476E7F27B003A18BF22
:100310000122AAE7F5F7BCFC1D4B0222034489F831
:100320007028C9F86C38F0E6F5F7B2FC0223C9F87A
:100330006C0889F87038CBE7012301933BE700BFD5
:100340007457002480B40C08000002080000040860
:10035000745C002434550024D44C0024F4A20024FE
:10036000585700240C22002000247449BD378635DC
:10037000C426002004080024C026002050070024C2
:1003800040A80024B429002028A800246C350024AB
:1003900060E31600CCA1002454BF0C0838B501223C
:1003A0001C4B032804461A7005D9601CBDE8384070
:1003B000C0B212F0A3B8184BE6229FED186A5B6832
:1003C000DFED176A07EE903A164D1749F8EE677A97
:1003D00000FB0255154A0870284686EE277A144914
:1003E0000B6067EEA67AC2ED007A82ED017A114ABF
:1003F0001560114A136028F02DFC284627F0F0FE06
:1004000026F054F926F05AFA601CBDE83840C0B214
:1004100012F074B84C1C00200C22002000247449F7
:10042000BD378635F4A20024D44C0024C426002015
:100430005007002458570024C0260020044A0120F9
:100440000449136881F8780843F400131360704777
:100450004C570024CCA10024F8B5164D6B78BE2B68
:1004600026D1AC1C144F022229464FF6FF70FDF72F
:100470005DFD22884AB1A618BE4219D2052A17D9B5
:1004800021463446FDF752FDF3E721460222FDF7EF
:100490004DFD0222A1180634FDF748FD074B641BF1
:1004A000A3F87A4841F60F53C31A58425841F8BD91
:1004B0000020FCE70000020800000408CCA1002492
:1004C00070B5046886B005460E46C4F3100343BBFE
:1004D00001220393CDE901332023CDE9042304F164
:1004E0007843B3F5801F1AD3A4F10163B3F5801FDD
:1004F00010D2A4F58013022203F17843694601A8C3
:1005000002925B0C03934CF073FB50B14FF0FF3041
:1005100006B070BD052053F00DFB53F025FF2346B8
:10052000EAE73146204652F0FFFE18B92B68203327
:100530002B60EDE76FF00200EAE72DE9F0416B4E2A
:1005400090B03378B22B7ED1FFF786FF80F00104A4
:10055000E4B2674B04F00104664DB3F85B33664FB9
:10056000ADF80030BD4270D3002C00F0BC802822D2
:10057000002106A860F092FF604B04969B1B059338
:100580005F4BDA68D40770D45D4BD3F80C21D007E9
:1005900074D44FF480730222694604A8ADF83C304D
:1005A0005CF00AFB022269464FF6FF70514DFDF7E1
:1005B000BDFC4FF000080446BD4269D3002502226D
:1005C00001A904A8ADF804505CF0F6FA022201A9D2
:1005D0002046FDF7ABFC40BA022202A9C043ADF8A9
:1005E000080004A85CF0E8FA0E9888B106ABC0F1E8
:1005F00020022946184460F051FF9DF93C0018B9CB
:1006000006A904A8FFF75CFF00238DF83C000E93B9
:100610009DF83D307BB13A4BDA6842F00102DA6076
:10062000DA68D20707D5D3F80C2142F00102C3F8EB
:100630000C21D3F80C319DF93C00B0FA80F0400950
:1006400010B0BDE8F081012483E7AB691C3535F8B3
:10065000181CD3F8008055F8140CC1F30B0152F0AC
:1006600001FB804518BF01247CE7264A5A6002F14D
:1006700088325A60DB68D90786D58AE7214AC3F8F1
:10068000042102F18832C3F80421D3F80C3180E749
:10069000AE8802A904A88DF80D80C6F30B061C35A0
:1006A000B31DADF8083035F81C3CC3F30B021B0B2F
:1006B000ADF80A2006228DF80C305CF07DFA062297
:1006C00002A92046FDF732FC044655F8141C3246B8
:1006D00004A85CF071FA204655F8141C3246FDF768
:1006E00025FC044668E70120AAE700BF00000208D5
:1006F00014430B0880B40C0854BF0C080000040815
:100700000020005223016745F8B5274DFFF7ECF8AC
:1007100095F83038013B012B33D9244E01220324B4
:10072000234FF36885F87C2803F2DC53F360FFF76E
:1007300004FF58B13B78B22B08D1FFF78DFE013C86
:100740000BD060B9FFF7F9FE0028F3D1013CEED1E0
:10075000052053F0EFF953F007FE0028F8D095F884
:1007600030380022013B85F87C28012B13D9114B2E
:10077000012100221B6886F8251085F87D28F3608A
:10078000F8BDF5F785FA0C4B0222034485F8702872
:10079000C5F86C38C1E7F5F77BFA0223C5F86C0899
:1007A00085F87038E3E700BFCCA10024745700241B
:1007B000000002086C35002460E3160010B5074AFB
:1007C0000124074B14709C73FFF79EFFFFF792FC08
:1007D0002046BDE8104011F091BE00BF4C1C002027
:1007E000D44C002490F88D30B7EE007ADFED6A6AC1
:1007F000014607EE903A90F89130684AB0EE476AA9
:1008000005EE103A90F88F30F8EEE77A04EE903A61
:1008100090F89030B8EEC55A05EE903A90F89330C3
:1008200067EEA67A04EE103A25EE265AF8EEE44A70
:10083000F8EEE55AB8EEC44A25EE275A64EEA64A09
:1008400065EEA65A24EE264A64EE854A65EEA75A5E
:1008500024EE274AB0EE473AF0B590F88C7000F1DC
:100860006B0602F11A050024137807EE903AF8EEB1
:10087000E77A67EE857A67EE867AFDEEE77A17EE1D
:10088000903AFA2BA8BFFA2323EAE3730B7253784A
:1008900007EE903AF8EEE77A67EEA47A67EE867A8A
:1008A000FDEEE77A17EE903AFA2BA8BFFA2323EA77
:1008B000E3734B72937803EE903AF8EEE33A63EE0B
:1008C000A57A67EE877AFDEEE77A17EE903AFA2B73
:1008D000A8BFFA2323EAE3738B72938807EE903A5A
:1008E000F8EEE77A67EE847A67EE867AFDEEE77ACD
:1008F00017EE903AD5ED007AB3F57A7FF8EEE77A05
:10090000A8BF4FF47A7323EAE3738B812B68002B23
:100910003FDD90F89230B0EE436A02EE903AF8EE86
:10092000E22AA2EEE66A63EE863A83EEA76AA2EEB8
:10093000A66A65EEA77A013467EE877A67EE867A53
:10094000FDEEE77A17EE903AFA2BA8BFFA23BC42E5
:1009500023EAE37306F8013F00DDF0BD012C13D15B
:1009600090F88E3007EE103A90F8963006EE103A76
:10097000B8EEC77AB8EEC66A27EE267A26EE266A61
:100980000435083208316FE7B7EE007AB0EE476AF7
:10099000F6E7B7EE006ACCE70AD7233C72460B08AD
:1009A00090F88C3003B11DE7704790F894306BB32A
:1009B000B0F860308BB190F89520642102EB82038F
:1009C000C3EB0313B3FBF1F3A0F86030962312FBE3
:1009D00003F3B3FBF1F3A0F8623043884BB190F816
:1009E0009530642203EB8303C3EB0313B3FBF2F3F1
:1009F0004380B0F850304BB1962290F8953013FBFD
:100A000002F36422B3FBF2F3A0F85030704790F881
:100A100021304BB3438B83B190F82230FA2264210A
:100A200013FB02F203EB8303B2FBF1F2B3F57A7F1F
:100A30004283A8BF4FF47A738383838843B1FA2239
:100A400090F8223013FB02F36422B3FBF2F38380AD
:100A5000C3884BB190F8223003EB8303B3F57A7F60
:100A6000A8BF4FF47A73C380704770B5074D002458
:100A7000074E28460134FFF793FFE635FFF795FF51
:100A80003046FFF7C4FF042CF3D170BDF4A200245C
:100A90001058002410B5064C4FF48072002104F663
:100AA0007E0060F0FBFC0023C4F8803910BD00BF5D
:100AB000CCA10024034BD3F8840908B10AF086BD09
:100AC000704700BFCCA1002408B50B46054902467B
:100AD000D1F8840928B10449FDF7ECFFBDE80840CE
:100AE000E8E708BDCCA10024F1E60408024B01466A
:100AF000D3F88409FDF7FEBDCCA100240048F5E73A
:100B0000F34C0C080CB4C30607B500D561B905A9B0
:100B100004980191FFF7D8FFFFF7F0FF012003B021
:100B20005DF804EB02B070470020F8E708B5FFF766
:100B3000DDFFBDE80840E1E710B504460348FFF7D4
:100B4000D5FF2046BDE81040F0E700BF403D0C084F
:100B500010B508460749FDF7E7FA002815BF01243C
:100B6000002405480548FFF7E7FF2046BDE8104090
:100B700009F0D2BD453D0C084E3D0C08753D0C08F2
:100B8000034B0146D3F8840908B10AF00BBD704746
:100B9000CCA100240CB407B510F020000BD079B91B
:100BA0002320FFF7EDFF05A904980191FFF78CFFC3
:100BB000FFF7A4FF012003B05DF804EB02B070471B
:100BC0000020F8E70FB407B504A951F8040B019110
:100BD000FFF77AFF03B05DF804EB04B0704738B557
:100BE00004460D46FDF797FD38B12A4621460348D5
:100BF000FFF7E8FFBDE8384080E738BD913D0C08BD
:100C00000EB417B50446FDF786FD50B121460748DE
:100C1000FFF7D8FF06A905980191FFF755FFFFF7E9
:100C20006DFF03B0BDE8104003B07047973D0C085E
:100C300030B52A4885B0FFF759FF294B1B7923B9F6
:100C4000284805B0BDE8304070E7FBF76BFE08B9F7
:100C50002548F6E7FBF77EFE08B92448F1E7244B68
:100C60001B68DB6998470028F7D0FBF753FE026842
:100C70000446037D81795208407CE51D0C340290C6
:100C800020790190E08800901A48FFF79BFF15F843
:100C9000010BFFF775FFAC42F9D1174C1748FFF76E
:100CA00025FF6378022B06D007D9032B0ED11448F9
:100CB000FFF71CFF0AE01348FAE71348FFF716FF97
:100CC00094F8E831022B05D0032B05D005B0BDE820
:100CD000304013E70D48EBE70D48E9E79B3D0C0872
:100CE000084D0024A53D0C08B43D0C08C23D0C087D
:100CF00058480024D13D0C085C490024FF3D0C08F5
:100D0000053E0C080B3E0C08183E0C081E3E0C0855
:100D1000373E0C08F8B5164B1B6843B30025154F3A
:100D20001548FFF703FFFFF7C5FEFBF729F8FBF7B0
:100D300061F8044640B1132011F034FBFFF7DEFEEA
:100D40000E48BDE8F840F1E6FBF7ACF83846FFF78F
:100D500039FF792D05F1010602D12646FFF7CEFEB7
:100D6000FFF7A8FE64203546F6F7C6FADFE7F8BDC0
:100D7000C04700241A5E0C08493E0C08633E0C086C
:100D80002DE9F04F8FB00B4611F8012B202AFAD035
:100D9000002AB14CB1494FF0000508BF0023B0480C
:100DA000B04E04F519682362FFF719FFAE492F46CC
:100DB000AE48FFF714FFAE49AE48FFF710FFAE494B
:100DC000AE48FFF70CFFAE49AE48FFF708FFAE494B
:100DD000AE48FFF704FFAE49AE48FFF700FFAE494B
:100DE000AE48FFF7FCFEAE49AE48FFF7F8FEAE494D
:100DF000AE48FFF7F4FEAE49AE48FFF7F0FEAE4B4B
:100E0000AE491A68AE4BAF48DFF87093B2FBF3F20D
:100E1000FFF7F6FEB4F88829A849AB48FFF7F0FEC3
:100E2000B4F98A29A949AA48FFF7EAFEA94AA749BD
:100E3000A948FFF7E5FEA94AA949AA48FFF7E0FE3D
:100E4000A94BAA489B7B06EB8303D3F88413FFF7D7
:100E5000C6FEB4F87A289D49A548FFF7D1FEA54BF8
:100E6000A54A9A49D21AA548FFF7CAFE94F88C29D8
:100E70009649A348FFF7C4FE94F88D299349A148E9
:100E8000FFF7BEFEA04B91491A88A04892B2FFF727
:100E9000B7FE99F81F3005F1010A2B41DA070ED58C
:100EA0009B49524606A80137FDF754FF98F80030D9
:100EB00006A806EB8303D3F88C13FFF790FEBAF174
:100EC000020F08F101084FF00105E2D13A467B49D3
:100ED0009048AA46FFF794FE8F4FD4F89439DFF874
:100EE000A0B201930AFA05F3019A13421CD0D7F875
:100EF000088015F80B903A7BB8F1000F14D091459B
:100F000012D2864A06A8864952F82520FDF722FF0C
:100F100006AA5F2012F8011B002940F0718158F8E1
:100F2000291006A8FFF75BFE01350837062DD9D139
:100F3000DFF850827B4FD8F800307B4D13F0800FE4
:100F40007A480CBF39462946FFF749FED8F80030E9
:100F50001B061DD594F8B4197548032994BF39466A
:100F60002946FFF73CFE94F8B4197248042994BF4F
:100F700039462946FFF733FE94F8C439002B00F0B8
:100F8000448106EBC303D3F844146B48FFF727FEF4
:100F90006A4B6B481D686B4B1B7806EB8303D3F8D9
:100FA0007814FFF71CFE4DB16A7A44496648FFF792
:100FB00027FE2A7A41496548FFF722FEFAF7ACFE80
:100FC000026905464AB162496248FFF719FEAA68FC
:100FD0003A49120D6048FFF713FE604B60481A68EB
:100FE0004FF47A733549B2FBF3F2FFF709FE03A819
:100FF000FEF738FB38B103A906A85BF0B9FF06A9D4
:101000005848FFF7ECFD02A90220FDF733FC94F8E5
:10101000C85980462DB1544B93ED050A5EF0F2FE9F
:10102000054600210846FDF725FC504B0746274999
:101030001A884F48642AA8BF6422FFF7E1FD029A8C
:1010400022494C48FFF7DCFD424620494A48FFF759
:10105000D7FD2A4698E000BFCCA10024713E0C08C1
:101060007C3E0C0814430B088A3E0C08933E0C0887
:10107000A43E0C08AE3E0C08DB4C0024B53E0C0828
:10108000C63E0C08D23E0C08DD3E0C08E63E0C08BD
:10109000F13E0C08FC3E0C08093F0C080E3F0C0802
:1010A0001E3F0C08233F0C08333F0C08433F0C083D
:1010B0004E3F0C085A3F0C08880300241F410C08BF
:1010C00040420F005E3F0C08663F0C084F660C085C
:1010D0006E3F0C08000800007A3F0C08F8FF012062
:1010E000704D0C08853F0C08D44C0024903F0C0830
:1010F0009D3F0C080000020800000408A93F0C08EE
:10110000B93F0C08C33F0C08BC280024CD3F0C0895
:10111000D83F0C08E33F0C080C470B083C470B0872
:10112000EE3F0C085C660C0887410C08F43F0C0885
:1011300000400C080E400C081D400C08BC5B00244D
:1011400029400C08B85B002434400C083D400C08D2
:10115000E1410C0846400C0855400C086C35002451
:1011600063400C086C400C0804080024F02900209F
:1011700079400C0886400C0894400C081058002454
:1011800010080024345500242B492C48FFF738FD63
:101190003A4629492A48FFF733FDB4F8CC3964218F
:1011A0002848B3FBF1F201FB123327499BB2FFF74A
:1011B00027FD94F8DC2920492448FFF721FD94F805
:1011C000DD39234806EB8303D3F89014FFF707FDBE
:1011D0002048FDF7A0FA054668B11F484FF0010806
:1011E000FFF784FC1D4BDFF87C901E68DFF878A0C9
:1011F0006EB9FFF783FC002323620FB0BDE8F08FC8
:101200002D2908BF02F8010C84E61549BDE696FABF
:10121000A6F7B7FA87F708FA07F726EA070615B917
:101220004846FFF763FC3846002510F0A7FC01464E
:101230005046FFF7C7FCDBE74F660C08A1400C08DF
:10124000AC400C08BB400C08BD430C08C5400C0862
:10125000D3400C08E1400C08F6400C084C57002421
:10126000693E0C08D4500C08FD570C080FB407B5A4
:1012700004A951F8040B0191FFF726FCFFF73EFC8F
:1012800003B05DF804EB04B070472DE9F8438388A0
:1012900003F4E072802A4AD009D822BB03F0070386
:1012A000052B1BD8DFE803F0171A171A0A10C02AFB
:1012B00044D0B2F5807F3DD0BDE8F883D0F8061069
:1012C0002048BDE8F843D1E7D0F8062051421E4837
:1012D000BDE8F843CAE70289C188F8E7B0F90820F9
:1012E000B0F90610F3E785790024184E1848FFF787
:1012F000FDFB012306EBC50292F80480A04503D84C
:10130000BDE8F843FFF7FABB56F835704FEA840999
:1013100057F824204AB113B90E48FFF7E7FB57F8F6
:1013200009100D48FFF74EFC00230134E6E78179F0
:101330000A48C6E7C27981790948C9E70948BDE882
:10134000F84393E70C410C0822410C0814430B08A6
:1013500039410C0875430C08FD570C084A410C082C
:101360005B410C0872410C082DE9F04385B0224E18
:10137000FAF7D2FC026983890025018804460292AB
:101380008268DFF8888001924288DFF884901B4FE2
:10139000009242681A48FFF769FF15B91948FFF72C
:1013A000C5FBD8F800309D4212DA3378052B20D8DF
:1013B00009EB8303D3F8A424B388294601353846C2
:1013C0000093063636F8043CFFF750FF062DE4D1B3
:1013D00051F0CEFB4288838864689B1A03FB044467
:1013E000FAF744FD02460848214605B0BDE8F0433F
:1013F0003CE70022E0E700BF10500024F4410C0855
:101400008A410C08E8410C0803420C0834500024BF
:1014100014430B080249034801F500610EC925E792
:1014200000E0F11F20420C0870B50024144E96F81D
:101430002330651C2341DB071CD5E4B22946114843
:10144000FFF714FF752120462EF050F901460E4893
:10145000FFF70CFF1A2120462EF048F901460B48F1
:10146000FFF704FF1B2120462EF040F901460848F3
:10147000FFF7FCFE022D4FF00104D8D170BD00BF74
:101480001058002434420C0840420C0853420C0807
:1014900066420C08B74BB8491A68B84B2DE9F04FB3
:1014A00095B0B74CB74E0025079004F5196BB648B8
:1014B000B64FDFF88883B946DFF884A3B2FBF3F2B6
:1014C000FFF780FBB4F888294FF47A730A20B2FB47
:1014D000F3F103FB1122B4F98A3992B2B2FBF0F2B4
:1014E000AB48FFF7C3FEAB4AAB49AC48FFF76AFB1A
:1014F000FFF704FBAA4BAB4A997BAB4B06EB810190
:10150000AA48D31AB4F87A28D1F88413FFF7AEFEAC
:10151000FFF7F4FAA648FFF7E9FA94F88C19A54802
:10152000FFF750FBA448FFF7E1FAA44B94F88D199C
:101530001A88A34892B2FFF745FBFFF7DFFAA149EB
:10154000A148FFF73FFB2B4698F81F202A41D00700
:101550002FD513B19D48FFF7C9FA691C5046FFF714
:1015600031FB15F80B309A4806EB8303D3F88C1344
:10157000FFF728FB99F88A342B41D90702D5954803
:10158000FFF720FB97F82031032B09D09248FFF793
:1015900019FB97F82031012B02D19048FFF712FB7D
:1015A000FB6C2BB15B7B012B02D98D48FFF70AFB4B
:1015B000012307F5D277002D00F0C481002B40F005
:1015C000C3818848FFF7B2FAD4F894894FF0010933
:1015D000854FDFF870A209FA05F313EA080F19D056
:1015E000BB6815F80A20397BA3B18A4212D253F89E
:1015F00022207E4B7E4853F82510FFF7E3FA012D99
:1016000006D17C4B93F8211011B17B48FFF7DAFA31
:10161000FFF774FA01350837062DDCD17748FFF75C
:1016200065FA774B1B681A0640F1E68194F8B439E5
:10163000032B8CBF73487448FFF758FA94F8C035F1
:101640009A1E022A00F2838106EB8303D3F8BC04BE
:10165000FFF74CFA94F8B439052B7FD1FFF74EFA17
:1016600094F8101A6948FFF7ADFA002294F8285A46
:1016700013461146664F954200F2B08123B165488A
:10168000B1FBF3F1FFF79EFAB4F8EE2942B16423FF
:101690006148B2FBF3F103FB112292B2FFF792FA19
:1016A000B4F8F02942B164235C48B2FBF3F103FBC8
:1016B000112292B2FFF786FA94F8AC3A9B0740F1F8
:1016C0009781D4F8E4094FF06409554F5549D4F88F
:1016D000E859D4F8E03937EA200B28BF8B460028B8
:1016E00083EAE37CB8BF404237EA250A28BF8A462E
:1016F000002DACEBE37C4C4BB8BF6D42B0FBF3FE6E
:10170000B5FBF9F803FB1E0009FB1855BCFBF3F20F
:10171000CDE90485CDE9020ACDE900BED4F8E0099F
:1017200003FB12C311EA200138BF39463F48FFF7D7
:1017300049FA94F8263A8BB194F8223A3C4802933D
:1017400094F8213A019394F8203A009394F81F3AC0
:1017500094F81E2AB4F81C1AFFF734FAFFF7CEF9F2
:10176000344B1A78002A74D0334A1278002A00F0D9
:10177000478169E0880300244E3F0C0840420F0077
:10178000CCA1002414430B0879420C080C22002041
:101790008B420C08F8FF012000080000AD420C0845
:1017A000D44C00240000040800000208BF420C08CA
:1017B000D6420C08E8420C08F0420C08BC28002471
:1017C000F2420C0806430C080B430C0875430C0846
:1017D00094430C08EB570C0815430C081D430C08E8
:1017E00022430C082A430C080C470B083C470B0803
:1017F0002E5C0C08F02900202F430C0833430C0802
:101800003455002439430C0845430C0898430C0810
:10181000F8AB0024A3430C08B5430C08C5430C08DF
:10182000F54C0C086D5F0C0880969800D5430C08A9
:101830000F440C08E83700242C37002410580024EB
:1018400010430C08100800249A7859787648FFF75E
:101850000DFD764B76481D68764B1B7806EB8303AF
:10186000D3F87814FFF7AEF925B12A7A697A72486D
:10187000FFF7A8F9FFF742F970490798FFF7D8F981
:10188000FAF74AFA016921B182686D48120DFFF733
:10189000EDFCFFF733F96B4B6B4819684FF47A7323
:1018A000B1FBF3F1FFF78EF909A8FDF7DBFE38B1C4
:1018B00009A90CA85BF05CFB0CA96448FFF782F94E
:1018C000FFF71CF908A90220FCF7D4FF94F8C859C7
:1018D00007462DB15E4B93ED050A5EF093FA05467F
:1018E00000210846FCF7C6FF5A4B089A19883B4668
:1018F0006429CDE90050A8BF64215748FFF7B6FC22
:10190000B4F8CC29642355480125B2FBF3F103FB5D
:10191000112294F8DD3906EB830692B2D6F89034A2
:101920004F4E009394F8DC39FFF7A0FC4D48FFF7C9
:10193000DDF84D4B1C68002C66D1FFF7DFF815B0C1
:10194000BDE8F08F0125FFE5FFF7D8F83CE602205F
:1019500010F0E2FB0546C8B94448FFF7C7F894F811
